:020000040800F2
:20300000481F002001310008170D010811B40008150C01080D4500087D4A010800000000A1
:20302000000000000000000000000000E3280108E16300080000000079100108F13601086E
:203040001B3100081B3100081B3100081B3100081B3100081B3100081B3100081B310008D0
:203060007D6900081B3100081B310008695400081B3100081B3100081B3100081B310008A5
:203080001B3100081B310008E53D00081B310008B54601081B3100081B3100081B3100080A
:2030A0001B3100081D3801081B3100081B3100081B3100081B3100081B3100081B31000866
:2030C0001B3100081B3100081B3100081B3100081B3100081B3100081B310008C94501088D
:2030E000716900081B3100081B310008DFF80CD000F028FE00480047C13D0008481F002061
:203100000648804706480047FEE7FEE7FEE7FEE7FEE7FEE7FEE7FEE7FEE7FEE7C53701080E
:20312000ED3000082DE9FF1F002000210022002300240025002600275FF000085FF000096B
:203140005FF0000A5FF0000B5FF0000C002001210222032304240525062607275FF00808CA
:203160005FF009095FF00A0A5FF00B0B5FF00C0C00281DD101291BD1022A19D1032B17D167
:20318000042C15D1052D13D1062E11D1072F0FD1B8F1080F0CD1B9F1090F09D1BAF10A0FDA
:2031A00006D1BBF10B0F03D1BCF10C0F00D101E003F0BCBEBDE8FF1F7047000073B40020F6
:2031C00000210124002501262046A04226D1A94224D12846A84221D1A9421FD14FEA440498
:2031E00006F10106202EEFDD5FF0FF305FF0FF317FF000445FF0FF3501262046A0420DD137
:20320000A9420BD12846A84208D1A94206D14FEA740406F10106202EEFDD01E003F086BE13
:2032200073BC7047E7B40021002000220125002601272946A94230D1B0422ED1B2422CD1F9
:203240003146B14229D1B04227D1B24225D14FEA450507F10107202FEBDD5FF0FF315FF0CE
:20326000FF305FF0FF327FF000455FF0FF3601272946A94211D1B0420FD1B2420DD13146E8
:20328000B1420AD1B04208D1B24206D14FEA750507F10107202FEBDD01E003F047BEE7BC84
:2032A00070472DE9CE01002200210023012600275FF001083246B24233D1B94231D1BB42FC
:2032C0002FD13A46BA422CD1B9422AD1BB4228D14FEA460608F10108B8F1200FEADD5FF014
:2032E000FF325FF0FF315FF0FF337FF000465FF0FF375FF001083246B24212D1B94210D1E0
:20330000BB420ED13A46BA420BD1B94209D1BB4207D14FEA760608F10108B8F1200FEADD79
:2033200001E003F003BEBDE8CE0170472DE99C0300230022002401275FF000085FF00109D7
:203340003B46BB4233D1424531D144452FD1434643452CD142452AD1444528D14FEA470740
:2033600009F10109B9F1200FEADD5FF0FF335FF0FF325FF0FF347FF000475FF0FF385FF09B
:2033800001093B46BB4212D1424510D144450ED1434643450BD1424509D1444507D14FEA0A
:2033A000770709F10109B9F1200FEADD01E003F0BDBDBDE89C0370472DE9381C00240023F1
:2033C00000255FF0010A5FF0000B5FF0010C5446544533D15B4531D15D452FD15C465C45FA
:2033E0002CD15B452AD15D4528D14FEA4A0A0CF1010CBCF1200FEADD5FF0FF345FF0FF335D
:203400005FF0FF357FF0004A5FF0FF3B5FF0010C5446544512D15B4510D15D450ED15C46D1
:203420005C450BD15B4509D15D4507D14FEA7A0A0CF1010CBCF1200FEADD01E003F076BDAA
:20344000BDE8381C70472DE9701C0025002400265FF0010A5FF0000B5FF0010C5546554566
:2034600033D15C4531D15E452FD15D465D452CD15C452AD15E4528D14FEA4A0A0CF1010CF1
:20348000BCF1200FEADD5FF0FF355FF0FF345FF0FF367FF0004A5FF0FF3B5FF0010C5546C7
:2034A000554512D15C4510D15E450ED15D465D450BD15C4509D15E4507D14FEA7A0A0CF1BA
:2034C000010CBCF1200FEADD01E003F02FBDBDE8701C70472DE9E01C0026002500275FF0C1
:2034E000010A5FF0000B5FF0010C5646564533D15D4531D15F452FD15E465E452CD15D45A2
:203500002AD15F4528D14FEA4A0A0CF1010CBCF1200FEADD5FF0FF365FF0FF355FF0FF374D
:203520007FF0004A5FF0FF3B5FF0010C5646564512D15D4510D15F450ED15E465E450BD1AA
:203540005D4509D15F4507D14FEA7A0A0CF1010CBCF1200FEADD01E003F0E8BCBDE8E01CF0
:2035600070472DE9C01D002700265FF000085FF0010A5FF0000B5FF0010C5746574533D1B0
:203580005E4531D1D8452FD15F465F452CD15E452AD1D84528D14FEA4A0A0CF1010CBCF12B
:2035A000200FEADD5FF0FF375FF0FF365FF0FF387FF0004A5FF0FF3B5FF0010C57465745AF
:2035C00012D15E4510D1D8450ED15F465F450BD15E4509D1D84507D14FEA7A0A0CF1010C2A
:2035E000BCF1200FEADD01E003F0A0BCBDE8C01D70472DE9801F5FF0000800275FF0000934
:203600005FF0010A5FF0000B5FF0010CD046D04533D15F4531D1D9452FD1D846D8452CD16F
:203620005F452AD1D94528D14FEA4A0A0CF1010CBCF1200FEADD5FF0FF385FF0FF375FF040
:20364000FF397FF0004A5FF0FF3B5FF0010CD046D04512D15F4510D1D9450ED1D846D845C9
:203660000BD15F4509D1D94507D14FEA7A0A0CF1010CBCF1200FEADD01E003F057BCBDE804
:20368000801F70472DE970075FF000095FF000085FF0000A012400250126A146A14530D100
:2036A000A8452ED1AA452CD1A946A94529D1A84527D1AA4525D14FEA440406F10106202EC4
:2036C000EBDD5FF0FF395FF0FF385FF0FF3A7FF000445FF0FF350126A146A14511D1A84594
:2036E0000FD1AA450DD1A946A9450AD1A84508D1AA4506D14FEA740406F10106202EEBDD14
:2037000001E003F013BCBDE8700770472DE9700E5FF0000A5FF000095FF0000B012400254A
:203720000126A246A24530D1A9452ED1AB452CD1AA46AA4529D1A94527D1AB4525D14FEADA
:20374000440406F10106202EEBDD5FF0FF3A5FF0FF395FF0FF3B7FF000445FF0FF35012618
:20376000A246A24511D1A9450FD1AB450DD1AA46AA450AD1A94508D1AB4506D14FEA740403
:2037800006F10106202EEBDD01E003F0CFBBBDE8700E70472DE9701C5FF0000B5FF0000A88
:2037A0005FF0000C012400250126A346A34530D1AA452ED1AC452CD1AB46AB4529D1AA45C5
:2037C00027D1AC4525D14FEA440406F10106202EEBDD5FF0FF3B5FF0FF3A5FF0FF3C7FF06B
:2037E00000445FF0FF350126A346A34511D1AA450FD1AC450DD1AB46AB450AD1AA4508D106
:20380000AC4506D14FEA740406F10106202EEBDD01E003F08BBBBDE8701C70472DE970187B
:203820005FF0000C5FF0000B012400250126A446A44526D1AB4524D1AC46AC4521D1AB45EE
:203840001FD14FEA440406F10106202EEFDD5FF0FF3C5FF0FF3B7FF000445FF0FF3501266F
:20386000A446A4450DD1AB450BD1AC46AC4508D1AB4506D14FEA740406F10106202EEFDD7F
:2038800001E003F053BBBDE8701870472DE9F0030024002546594E51445105F10405182DF9
:2038A000F8DB04255FF0000801245FF0010944514659B4425FD105F10407C659B0455AD19D
:2038C0002F1FC659B04556D140F805804659B04551D105F10407C659B0454CD12F1FC6594D
:2038E000B04548D14FEA440409F10109B9F1200FDDDD05F10405142DD6DB5FF0FF3400250A
:20390000445105F10405182DFADB04255FF0FF387FF000445FF0010944514659B4422AD119
:2039200005F10407C659B04525D12F1FC659B04521D140F805804659B0451CD105F10407E9
:20394000C659B04517D12F1FC659B04513D14FEA740409F10109B9F1200FDDDD05F10405DE
:20396000142DD5DB00254E59465105F10405182DF9DB012000E00020BDE8F00370472DE955
:20398000F00300240025445105F104058D42FADB00255FF0000801245FF001094451465985
:2039A000B44268D1002D03D02F1FC659B04562D105F104078F4202DAC659B0455BD140F81D
:2039C00005804659B04556D1002D03D02F1FC659B04550D105F104078F4202DAC659B04562
:2039E00049D14FEA440409F10109B9F1200FD5DD05F104058D42CEDB5FF0FF3400254451EA
:203A000005F104058D42FADB00255FF0FF387FF000445FF0010944514659B4422BD1002DF9
:203A200003D02F1FC659B04525D105F104078F4202DAC659B0451ED140F805804659B04559
:203A400019D1002D03D02F1FC659B04513D105F104078F4202DAC659B0450CD14FEA7404E6
:203A600009F10109B9F1200FD5DD05F104058D42CDDB012000E00020BDE8F0037047202A87
:203A800004DB203A21FA02F00021704721FA02F3D040C2F12002914008431946704740EAB7
:203AA00001039B0703D009E008C9121F08C0042AFAD203E011F8013B00F8013B521EF9D249
:203AC0007047D2B201E000F8012B491EFBD270470022F6E710B513460A4604461946FFF7AF
:203AE000F0FF204610BD10B5044604E00B7800F8013B03B1491C521EF8D2204610BD421C16
:203B000010F8011B0029FBD1801A704730B505460020034600E05B1C934205D2EC5CC85C33
:203B2000201A01D1002CF6D130BD2DE9F0410546002090460E46044600E0641C44450BD2AD
:203B4000285D00F04AF80746305D00F046F8381A02D1295D0029F0D1BDE8F0810EB5C10F68
:203B600080EAE0700844CA07002140F233438DE80E000A460B4600F045F803B000BD70B5BF
:203B8000C1F30A5201F000450024C1F3130140F2FF3341F480119A4201DA002070BD40F293
:203BA00033439A42A2F2334203DC5242FFF767FF00E090402C43F1D0404270BD202A04DB23
:203BC000203A00FA02F1002070479140C2F1200320FA03F3194390407047A0F14101192918
:203BE00000D82030704710B5141E73F1000408DA401C41F1000192185B411A4301D120F091
:203C0000010010BD2DE9F04D92469B4611B1B1FA81F202E0B0FA80F220329046FFF7CEFF01
:203C200004460F4640EA0A0041EA0B0153465A46084313D0114653EA010019D0C8F140029A
:203C40005046FFF71CFF05460E46504659464246FFF7B4FF084305D0012004E020463946AE
:203C6000BDE8F08D0020054346EAE0762C4337430A986305E40AA0EB08000022FD0A44EA69
:203C800047540A3002D500200146E9E7010510196941DDE9084500196941BDE8F04DA2E727
:203CA0002DE9F04D00231A461B1A8A4103DB00200146BDE8F08DC1F30A52C1F3130141F4BA
:203CC00080154FF0000BD10702D100186D41521E0027044640F2FF11384601EB620A3E4617
:203CE0008046024600204FF48011FFF7C8FEC2197141BB1846EB0100B4EB030C75EB000C5A
:203D000004D3E41A65EB000517460E46241908F101006D4180463428E3DDF91946EB0600B8
:203D2000091BA84103D24FF0FF32134601E0002213461BEB070046EB0A51BDE8F04DFFF70B
:203D400052BF0000064C074D06E0E06840F0010394E8070098471034AC42F6D3FFF7CAF934
:203D6000547E0108747E010870B58C1810F8015B15F0070301D110F8013B2A1106D110F801
:203D8000012B03E010F8016B01F8016B5B1EF9D12B0705D40023521E0DD401F8013BFAE763
:203DA00010F8013BCB1A921C03E013F8015B01F8015B521EF9D5A142D8D3002070BD000074
:203DC00010B572B606480079AA2801D00EF08AFC00200349087162B611F0F6FA10BD00004D
:203DE0000030024010B5024804F00CF810BD00009C13002070B5044600252068806800F0BA
:203E00000100F0B12068806820F001002168886005F060FC05460EE005F05CFC401B0228B2
:203E200009D9A06A40F01000A062E06A40F00100E062012070BD2068806800F001000028C0
:203E4000EAD10020F6E770B505466C6AA06A00F05000E0B9A06A40F40070A0622068806861
:203E600000F46020B0F5602F0DD1E06858B9A06A20F48070A062A06A00F4805018B9A06AAA
:203E800040F00100A062204603F01CFE03E0206A016B2846884770BD70B505466C6AA06AE9
:203EA00040F04000A062E06A40F00400E062204603F0A7FF70BD70B50446656A284603F005
:203EC0009FFF70BD38B504460025002000902068806800F0010080BB2068806840F00100CE
:203EE00021688860164800681649B0FBF1F0009002E00098401E009000980028F9D105F029
:203F0000E9FB054613E005F0E5FB401B02280ED9A06A40F01000A062E06A40F00100E06235
:203F200000BF002084F8240000BF012038BD2068806800F001000028E5D00020F6E70000F2
:203F40000000002040420F0070B505460E4605F0C1FB22490968401A02283DD3002418E0AF
:203F60001F4850F824001F4931F81410C0EB81201B4951F8241001EBE010194941F82400F1
:203F8000084650F82400C0F38F2025F81400601CC4B2092CE4DB002418E0134850F824000B
:203FA000124931F81410C0EB81200F4951F8241001EBE0100C4941F82400084650F82400F0
:203FC000C0F38F2026F81400601CC4B2032CE4DB05F080FB0149086070BD000034040020C6
:203FE000101400204813002034140020E003002010B5154803F02AFA144803F027FA124894
:2040000004F0B6F8114804F0B3F8104803F02EFC09220F490C4804F043F90B48006A006865
:20402000006820F004000849096A09680860094806F099FB0C21074806F00CFE0C21054896
:2040400006F0B2FA10BD00006C1300209C1300204813002088120020014600226648814274
:204060000DD1664848604A68824201D000207047634848604A68824201D00020F7E76148AD
:2040800081420DD1604848604A68824201D00020EDE75E4848604A68824201D00020E6E772
:2040A00040F2555048614A69824201D00020DEE740F6AA2048614A69824201D00020D6E785
:2040C00040F2555088618A69824201D00020CEE740F6AA2088618A69824201D00020C6E785
:2040E00040F25550C861CA69824201D00020BEE740F6AA20C861CA69824201D00020B6E785
:2041000040F2555008620A6A824201D00020AEE740F6AA2008620A6A824201D00020A6E780
:2041200040F2555048624A6A824201D000209EE740F6AA2048624A6A824201D0002096E780
:2041400040F2555088628A6A824201D000208EE740F6AA2088628A6A824201D0002086E780
:204160002B48C862CA6A824201D000207FE72948C862CA6A824201D0002078E72648086397
:204180000A6B824201D0002071E7244808630A6B824201D000206AE71F4848634A6B8242C0
:2041A00001D0002063E71D4848634A6B824201D000205CE71A4888638A6B824201D0002010
:2041C00055E7184888638A6B824201D000204EE700204860C860086148618861C8610862FB
:2041E00040F6FF70486200208862C86208634863886301203BE700000024014055554500A4
:20420000AAAA8A000028014055554000AAAA800055555500AAAAAA0055555515AAAAAA2A60
:2042200055551500AAAA2A0088B001460022086800904868019088680290CB6803930B69A0
:2042400004934B690593552008600A68552A02D0002008B07047AA2008600A68AA2A01D003
:204260000020F6E745F2555048604A68824201D00020EEE74AF6AA20486048684AF6AA2312
:2042800000EA03021846824201D00020E1E745F2555088608A68824201D00020D9E742F6F1
:2042A000AA2088608A68824201D00020D1E745F25553CB60CA681846824201D00020C8E7EF
:2042C00042F6AA23CB60CA681846824201D00020BFE745F255530B610A691846824201D012
:2042E0000020B6E742F6AA230B610A691846824201D00020ADE745F255534B614A691846DA
:20430000824201D00020A4E742F6AA234B614A691846824201D000209BE7009808600198CB
:20432000486002988860039BCB60049B0B61059B4B6101208DE70246002004E0002322F815
:204340001030431C98B28842F8DB7047F0B50346002640F2FE34601E534F07EB800042884C
:20436000154652480088401C504F3880384600880A2801DC0020F0BD4C4800880F2801DCFB
:204380000A20F8E749480088142801DC1920F2E746480088192801DC2D20ECE74348008869
:2043A0001E2801DC4120E6E740480088232801DC5520E0E73E48007801281FD100203C4F76
:2043C0003870002110E00A2093FBF0F0364F37F82170B84205DB344800EB81004088151A8E
:2043E00004E00025481C81B2A142ECDB00BF64206843B0FBF2F02F4F387051E02E48C07BF0
:204400002E4F3870384600782A4F38702C48006818442B4F38602B480078401C294F3870AF
:204420003846007819283BDB254800681927B0FBF7F086B20020224F3860224F38700021ED
:2044400010E00A2096FBF0F0174F37F82170B84205DB154800EB81004088151A04E0002508
:20446000481C81B2A142ECDB00BF64206843B0FBF2F0104F387038460078104F3F78B84273
:204480000EDD0C4807780D4800781E30874207DA084800785A2803DA08480078054F3870AE
:2044A0000448007867E70000046B0108DA020020E3020020E102002038060020E20200200C
:2044C000DC020020E002002038B504460B48012300220A2100900A4807F086F90948012314
:2044E00000220A210090084807F07EF903480078044909780840207038BD00008E03002012
:20450000E81100208F030020FC11002000BFFEE700B58BB0002006900790012008904CF2CB
:2045200020000190002002904CF2E01003904FF6FF700490002005900120099001A9154899
:2045400003F06EFF20B140F2271113A010F0F4FC0120069000200790012008904FF4604013
:204560000190002002904CF2E01003904FF6FF700490002005900120099001A9054803F096
:204580004FFF20B14FF49E7103A010F0D5FC0BB000BD00007C1800202E2E5C436F72655C6D
:2045A0005372635C63616E2E630000002DE9F04104460D46002700260DB9666B00E0A66BFB
:2045C000206800F5D87000EB0510006800F00400B060B06858B9206800F5D87000EB0510BC
:2045E000006840F2FF7101EA505030600AE0206800F5D87000EB051000686FF0604101EA94
:20460000D0007060206800F5D87000EB0510006800F00200F060206800F5D87000EB0510C6
:20462000406800F00F0030613562206800F5D87000EB05104068C0F30720F061206800F596
:20464000D87000EB051080683075206800F5D87000EB05108068010A7175206800F5D87022
:2046600000EB05108068010CB175206800F5D87000EB05108068000EF075206800F5D8703A
:2046800000EB0510C0683076206800F5D87000EB0510C068010A7176206800F5D87000EBBD
:2046A0000510C068010CB176206800F5D87000EB0510C068000EF0764DB920202168C86031
:2046C0002068406920F00A002168486108E02020216808612068406920F050002168486180
:2046E00094F83C70222F01D0322F05D12068406920F40F4021684861CDB994F83C004228AB
:2047000004D0622806D072280CD107E0122084F83C000BE0322084F83C0007E0522084F853
:204720003C0003E0012084F83C0000BF19E094F83C00522804D0622806D072280CD107E0F5
:20474000122084F83C000BE0222084F83C0007E0422084F83C0003E0012084F83C0000BF0E
:2047600000BF204604F032F90020BDE8F08100002DE9F34F83B0044660790B287EDB002164
:20478000204610F001FD00906449009808700121204610F0F9FC8246604981F801A00098C8
:2047A00055286CD1BAF1AA0FFBD12088000A88702078C8700221204610F0E6FC064657493E
:2047C0000E71112E03D0162E01D00C2E7ED10321204610F0D9FC8046504880F805800521CA
:2047E000204610F0D1FC83460421204610F0CCFC0BEB00201FFA80F94FEA192047498871C7
:2048000081F807900521204610F0BEFC0546A8EB0500022872D1617908F10900814217DA62
:20482000207C012804D104F055FFE0600020207404F050FFE168411A0498814205D96179A4
:20484000204610F05DFC0120207405B0BDE8F08F0120207400270EE0B81DC1B2204610F093
:2048600093FC2F49C8550846C15D07F108002B4A1154781C87B2AF42EEDB01E04CE047E013
:20488000A81DC1B2204610F07FFC4FEA006BE81DC1B2204610F078FC0BEB004B05F10800CA
:2048A000C1B2204610F070FC0BEB002B05F10900C1B2204610F068FC0BEB0001019105F1D7
:2048C0000801164800F038F9029000E01BE0DDE90110081A0CD12088114B4A46314600F012
:2048E0004BFE08F10900C1B2204610F009FCACE70121204610F004FC0EE0FFE70121204618
:2049000010F0FEFB08E00121204610F0F9FB03E00121204610F0F4FB00BF96E7C7090020B4
:20492000C808002030B50A4600211CE00F4B5B6B14335B5CC57884686355C3785B1CDBB2F7
:20494000C3708478A34201DB0023C37043795B1CDBB243718478A34203DD83784371012309
:2049600083714B1CD9B29142E0DB30BD7C1800202DE9F047824688461446002C5FDD204617
:20498000E11704EB5171C910A4EBC1018FB237B90827E11704EB5171C1F3CF0907E0204662
:2049A000E11704EB5171C910491C1FFA81F92548006BC0F800A000202249096BC8602149BC
:2049C000096B886000261CE008201E49096B086100250AE0082000FB065018F800101948E4
:2049E000006B14304155681C85B2082DF2DB0A21144804F05BF8012801D10BF0FBFE701C6C
:204A000086B2A9F10100B042DEDC0E48006B076100250AE0082000FB065018F800100948F5
:204A2000006B14304155681C85B2BD42F2DB0A21044804F03BF8012801D10BF0DBFEBDE898
:204A4000F08700007C18002010B504462068406920F001002168486194F83C00122805D1D0
:204A60002068406920F40F402168486194F83C00422804D0522806D072280CD107E022207A
:204A800084F83C000BE0322084F83C0007E0622084F83C0003E0012084F83C0000BF00BF0E
:204AA000204604F05BF9002010BD000010B5014600224C69CB69552008600A68552A01D0A5
:204AC000002010BDA82008600A6802F0A802A82A01D00020F5E70A4848614A69824201D0C9
:204AE0000020EEE7074848614A69824201D00020E7E74C61CB614FF4004008600120E0E7E7
:204B0000550501002A8A020030B503460C460021002200BF09E0985C80EA1120C0B2054DC6
:204B200035F8100080EA0121521CA242F3D388B230BD000054610108F0B502460B4600254C
:204B4000681E00210FE0565C7040002407E0060E064F57F8265000026840661CB4B2042C62
:204B6000F5DB4E1CB1B29942EDDBF0BD5463010800B585B000BF1848806940F00400164903
:204B800088610846806900F00400009000BF00BF00BF0846806940F00800886108468069A5
:204BA00000F00800009000BF00BF08200190002002900120039001A9084804F0EBFB4FF4B9
:204BC00000400190002002900120039001A9044804F0E0FB05B000BD00100240000C0140C8
:204BE000000801402DE9F84F04460D4616461F4600F0FAF8009000F0F7F8804600F0F4F8BE
:204C000081460098404504D1C84502D16A4880F800906A48007830B96748007866494870A0
:204C20000120664908706448007863494978884238D0614840786049097801F00301604A9F
:204C4000515C884209D1002060705E4908805E4908806068401C606024E0574840785649D7
:204C6000097801F00301594A515C88420DD155480088401C5349088008460088042811DB33
:204C800001206070002008800CE04F480088401C4D490880084600880A2803DD012060701D
:204CA000002008804FF0020A4348007800F001004149497801F0010188422DD004F00AFD0D
:204CC00043490968401A4FF47A71B1FBF0F04149088004F0FFFC3E49086017B94FF0010AB9
:204CE00000E0B246607858B93B480078401C3A49087008460078504504DB0120A07001E055
:204D00000020A07035490888012110F06FFD208104F0E0FC32490860324800682D4909888A
:204D2000C0EB81202F49096801EB20202D49086008460068C0F3872020704FF0640B254879
:204D40000088142802DA4FF496700DE021480088282801DD642007E01E48008800EB80009A
:204D60004FF4FA71A1EB40001FFA80FB0BFB05F0642190FBF1F085B204F0ACFC1849096894
:204D8000401AA84211D90020A070022060700020207010490880134908600F4908700F4946
:204DA0000888002110F022FD20810348007802494870BDE8F88F0000180300201A03002018
:204DC0001C7B01081C0300201E030020207B010820030020280300202A030020EE03002023
:204DE0002C0300202403002070B54FF40041084804F05EFC05462C460821064804F058FC5A
:204E0000064644EA4600C4B204F0030070BD000000080140000C014000BF084A1268526A5B
:204E200091B201EB810292004FF47A7392FBF3F202800022014B1B685A627047C8120020AC
:204E400010B54FF4FA710948FFF792FC4FF4FA710748FFF78DFC4FF4FA710648FFF788FC18
:204E60004FF4FA710448FFF783FC10BD5C040020700400208404002098040020F0B58DB09C
:204E800007460E46154618A103C9CDE90B0118A103C9CDE9070109AB002231460BA810F08C
:204EA000DDF905AB0022314607A810F0D7F9002405E009A8005D01A90855601CC4B2082C10
:204EC000F7DB002407E005A8015D01AA04F108001154601CC4B2082CF5DB294601A801F0DE
:204EE00086FA0DB0F0BD000039FF6C063454333029270957FFFFFFFF30B502460B460021E8
:204F0000002400BF0EE0481C84B207E0505C155DA84201D1002030BD601C84B29C42F5DBF8
:204F2000481C81B29942EEDB0120F4E731B581B0BDF80400ADF80000BDF9040044F6E615D6
:204F400000FB05F1C913BDF9060000FB05F2D2130C4613466042C01AC01A00B2ADF8020097
:204F600000983CBD70B504460AB9084670BD081B800290FBF2F086B2934202DD0D46284634
:204F8000F4E706FB03F004EBA02085B22846EDE710B590B01022694626480CF0CFFC0446B5
:204FA00024B9102269462448FEF779FD10226946204814300CF0C2FC04462CB91022694605
:204FC0001D481030FEF76BFD20226946194828300CF0B4FC044624B9202269461748FEF70D
:204FE0005EFD1022694613484C300CF0A7FC044624B9102269461248FEF751FD1022694679
:205000000C4860300CF09AFC044624B9102269460C48FEF744FD10226946064874300CF0B9
:205020008DFC044624B9102269460748FEF737FD10B010BD08FC010858060020B007002078
:20504000D0070020E0070020F007002010B50446574B0C220421204602F08CF9401C28B91D
:20506000534B0C220421204602F084F9514B20221221204602F07EF9401C28B94D4B202273
:205080001221204602F076F94B4B04223421204602F070F9401C28B9474B04223421204694
:2050A00002F068F9454B10223A21204602F062F9401C28B9414B10223A21204602F05AF9CC
:2050C0003F4B30224C21204602F054F9401C28B93B4B30224C21204602F04CF938480068DB
:2050E000401C374908600B4630224C2120460DF0B4FF401C28B9324B30224C2120460DF06A
:20510000ACFF304B1022EC21204602F033F9401C28B92C4B1022EC21204602F02BF92A4BC2
:2051200018227E21204602F025F9401C28B9264B18227E21204602F01DF9244B08229821D9
:20514000204602F017F9401C28B9204B08229821204602F00FF91E4B1022A221204602F046
:2051600009F9401C28B91A4B1022A221204602F001F9184B1022D621204602F0FBF8401C11
:2051800028B9144B1022D621204602F0F3F8124B2022B421204602F0EDF8401C28B90E4B1C
:2051A0002022B421204602F0E5F8002010BD00003408002020070020520100206007002019
:2051C00070070020A00700205C11002057010020B8080020A8080020400700201CB521491A
:2051E000214801F079FB102220491F4808300DF0D3FE10221D4910311B481C300DF0CCFE8A
:2052000020221B49184830300DF0C6FE10221949154854300DF0C0FE1022174912486830B3
:205220000DF0BAFE102215490F487C300DF0B4FE1348007800061249497800EB01401049FD
:20524000897800EB01200E49C9780844009004210B48FFF771FC019002226946024801F053
:205260000DFD1CBDFFFF010800FC010858060020B0070020D0070020E0070020F0070020D5
:20528000247B010838B5054600240FF017FE0FF0EFFD284601F0CCF9284601F085F91F48A3
:2052A000008800909DF800200021284601F08AFA401C28B99DF800200021284601F082FA2F
:2052C0009DF801200121284601F07CFA401C28B99DF801200121284601F074FA022168466E
:2052E000FFF712FC044622120221284601F06AFA401C20B922120221284601F063FAE2B26A
:205300000321284601F05EFA401C20B9E2B20321284601F057FA002038BD0000287B010854
:2053200010B5094A0949A2F10C00FFF7A7FD064B0C22042106480DF090FE0648006820F483
:2053400000100449086010BD34080020570100207C0300204401002070B5054600263948CC
:205360000078C8B9002404E03748C0880644601C84B20A2CF8DB0A20B6FBF0F033490880A1
:2053800004F0A8F93249086004F0A4F93149086001202C4908704FE004F09CF92D49096875
:2053A000401AB0F5FA7F03D904F094F9284908602868C0F3804000283ED104F08BF9244920
:2053C0000968401AB0F5FA6F36D9002404E01E48C0880644601C84B20A2CF8DB0A20B6FB4F
:2053E000F0F01A49088008460088B0F57A7F05DB0846008840F6B831884219DD286820F435
:20540000802000F5802028600720134948800F4800888880084601F033FB00200F49087040
:205420000F484089401C0E49488102200D49087004F050F90649086004F04CF905490860FD
:2054400070BD000040000020481300200404002044000020480000207C100020EC02002096
:20546000A00700205601002010B5024803F0F8FC10BD0000CC1300203FB504460025206841
:20548000009060680190A0680290E06803900020206045F2555020602568854202D000206C
:2054A00004B030BD0020206042F6AA2020602568854201D00020F3E70020206045F255508E
:2054C000606005200DF0FEF9656845F25550854201D00020E4E74AF6AA20606005200DF0DB
:2054E000F1F965684AF6AA20854201D00020D7E74FF05530A060A568B5F1553F01D0002079
:20550000CEE74FF0AA30A060A568B5F1AA3F01D00020C5E74FF05530E060E568B5F1553FF9
:2055200001D00020BCE74FF0AA30E060E568B5F1AA3F01D00020B3E7019860600298A06024
:205540000398E060009820600120A9E730B590F840500124AC40C56B6C60046863604468C2
:20556000102C04D10468A2600468E16003E00468A1600468E26030BD2DE9F84306460F4622
:2055800015461C4605F0FF0940F23171701A8E4272D00ADCA6F2516000286BD0CF280DD07B
:2055A000D0280CD0DF287DD165E00F287BD010287AD01F2879D02028F5D10BE300BF41F2FB
:2055C0000C61681A8D4236D00BDCA5F58050A0F1100070B1B0F53E7F23D0B0F5806F45D1F5
:2055E00023E0B0F5807F2CD0A0F5C850F93878BB2FE04A462146F848FEF751FAF648407A79
:20560000F649C8730020F649887604F063F8F449C8610020F349087004F05CF8F149486000
:2056200025E001200BF048FE21E04A462146EE48FEF735FA1BE04A462146EC48FEF72FFA6D
:2056400015E04A462146E9480C30FEF728FA0EE00CE04A462146E6A0FEF758FA28B9E6482D
:20566000007820F00100E449087000E000BF00BFAEE201E0E5E300BFB5F54C5F73D01FDC13
:2056800043F20201A5EB01008D4242D010DCA5F58050A0F1080058B3B0F5017F2CD0B0F5A0
:2056A000417F03E0EEE36CE16CE192E277D129E0A0F20310F0B3A0F203100028F6D160E0FB
:2056C00043F20561681A8D426AD008DCA5F54050A0F5816000287DD0F828E7D1A5E0A0F2BC
:2056E000FB20002877D0A0F205100028DED1EBE001200BF0E1FD42E14A462146BF48FEF7C7
:20570000CEF93CE14A462146BC480C30FEF7C7F935E1BB48007878B94A462146B948FEF70A
:20572000BEF9B8480078C043B7490870B5484078C04300E018E04870B2480078A74948735A
:20574000B048407888730B464FF481520C214FF4E2600DF019FD0020AC49087003F0BAFF39
:20576000AA4948600BE11CE04A462146A0A0FEF7CDF928B9A048007820F002009E49087002
:20578000FDE04A462146A248FEF789F9A1A345F203320C2140F213700DF0F6FCEFE0EDE0B7
:2057A0004CE09D4B202212219C4801F0E3FD9A48007B207098484078607097480079A070EE
:2057C0009548C07EE070234645F208420C2140F2137001E003E04EE00DF0D6FCCFE020788A
:2057E00040B28D49C876084690F91B000A2801DD0A20C876884890F91B0010F10A0F02DACF
:20580000F6208549C8766078834948700B462022122182480DF021FC7EA345F203320C21A6
:2058200040F213700DF0B0FCA9E07D4B41F210520C214FF4E2600DF0A7FCA0E04A4621465B
:2058400078A0FEF763F9A8B9002075498860C8600B461022D62171480DF0FFFB6DA345F21F
:2058600003320C2140F213700DF08EFC00205B490883488383E06D48007820BB10226C491E
:205880006C480CF05BF8102269491031694814300CF054F80C216848FFF74EF98046644817
:2058A000C0F82C8003464FF492520C214FF4E2600DF06AFC614B4FF4B9520C214FF4E26053
:2058C0000DF062FC00BF5AE04A46214655A0FEF71DF9002851D152480068B0F5FA7F44D2FD
:2058E0000922574957A0FEF711F9E8B100204C498860C860086048600B2255A15048FEF7C9
:20590000F2F8002055490870454B1022D62143480DF0A3FB00203149088348830FF0A8FAF7
:205920003E4800F041FE20E04548807A35281CDA00203B498860C860086048604048807A92
:20594000401C3F498872002044490870344B1022D62132480DF081FB0020204908834883CA
:205960000FF086FA2D4800F01FFE2AA345F203320C2140F213700DF007FC00E000BF00BFAD
:2059800076E600BFB5F5445F6CD010DCA5F58050A0F58670C8B1B0F5807F64D0B0F57F7F8E
:2059A00067D0A0F5F050F43800287CD169E0A5F54850083878B1FD2876D0B0F5FC7F74D087
:2059C000A0F2FD200028F0D1E1E04A4621462448FEF765F8FBE09CE0B80600203806002026
:2059E0009C02002084010020E0060020C8060020524541445900000048010020F00600205C
:205A0000C8000020CA000020CC000020740100204901002041434B00200700207C03002014
:205A2000A8080020434C4541520000009A0100205806002008FC01082808002098060020DB
:205A4000D0070020434C4541525F4F444F000000434C4541525F4F444F5F310075030020D7
:205A6000080700203AE04A462146F648FEF717F8ADE00020F449087003F02CFEF249486042
:205A8000A5E0F248007840BB1022F149F1480BF055FF1022EE491031EE4814300BF04EFF74
:205AA0000C21ED4802E091E05AE067E0FFF744F88046E748C0F82C8003464FF492520C2188
:205AC0004FF4E2600DF060FBE44B4FF4B9520C214FF4E2600DF058FB00BF78E0E04B2022E6
:205AE0001221E04801F046FCDD48007B2070DC4840786070DA480079A070D948C07EE070E2
:205B0000234647F208320C2140F214700DF03CFB5DE0207840B2D249C876084690F91B0080
:205B20000A2801DD0A20C876CD4890F91B0010F10A0F02DAF620CA49C8766078C849487036
:205B40000B4620221221C7480DF087FAAFF23C1347F203420C2140F214700DF015FB36E07E
:205B60004A462146AFF27810FDF7D0FF28B9BE48007820F00400BC49087028E0BB4B41F211
:205B800010520C214FF4E2600DF0FEFA1FE04A462146AFF27010FDF7B9FFB0B90020B349B4
:205BA0008860C8600B461022D621AE480DF055FAAFF2A01347F203420C2140F214700DF067
:205BC000E3FA0020AA490883488300BF00BF00BFF0E300BFB5F5045F7BD03DDC41F61001F7
:205BE000A5EB01008D4275D01CDC41F21041A5EB01008D426FD00CDCB5F5805F7CD0A5F58E
:205C000088500838F0B3F82867D0B0F5FC7F70D1D5E0F0286ED0B0F5007F6CD0B0F53C7F46
:205C2000F5D130E1B0F5A06F75D00BDCF12873D0B0F5F87F71D0B0F5447F6FD0B0F57C7FAD
:205C4000E5D185E1B0F5BE6F69D0B0F5DE6F67D0B0F5FE6FDBD1BFE142F60121681A8D42EB
:205C600076D023DC42F20561A5EB01008D4270D012DCA5F50050A0F5047000286AD0B0F5BD
:205C8000807F00E04DE07CD0B0F5047F7AD0A0F2F5200028BBD1F3E1A0F20310002872D0FC
:205CA000FA2871D0B0F5FC7FB1D168E240F2FF42811A904269D011DCA0F20110002865D08F
:205CC000FF2878D0A0F20620002875D0F8289ED108E393E1E5E081E00EE03CE0B1F5807F6D
:205CE0006BD0B1F5087F69D0A1F6092100298ED12EE342E384E092E05E4B08229821594881
:205D000001F038FB5B4B4AF208420C2140F215700DF03AFA32E32AE1D5E0F1E0FFE03BE17D
:205D20004BE14A4621465348FDF7B9FE514B082298214C480DF091F9AFF228334AF603120F
:205D40000C214FF4E2600DF01FFAFFF7E9FA15E31EE2B0E15BE13D48007858BB10223C4916
:205D60003C480BF0EBFD102239491031394814300BF0E4FD0C213848FEF7DEFE8046344866
:205D800005E058E16AE1BBE1D4E1B4E219E2C0F82C8003464FF492520C214FF4E2600DF035
:205DA000F3F92E4B4FF4B9520C214FF4E2600DF0EBF900BFE2E224E227E2A5E2B3E21022BD
:205DC0002D4924484C300BF0B9FD2B4B4AF210620C2140F215700DF0D7F9CFE24A46214637
:205DE0002548FDF75CFE002024490870AFF2DC334AF603120C214FF4E2600DF0C5F9BDE2D2
:205E000010221F49134860300BF098FD1C4B4AF210720C2140F215700DF0B6F9AEE24A4698
:205E200021461748FDF73BFE002014490870AFF21C434AF603120C214FF4E2600DF0A4F9D9
:205E40009CE29DE2140700207C0100209A0100205806002008FC0108280800209806002019
:205E6000200700207C03002048010020A80800203806002057010020D0070020750300209E
:205E8000E007002095E21022F949FA480BF056FDF74B4AF610020C2140F215700DF074F99E
:205EA0006CE24A462146F248FDF7F9FD0020F2490870AFF2A0434AF603120C214FF4E2601B
:205EC0000DF062F95AE22078EC49087008460078C043EB490870E948007801280FD1E94891
:205EE000006820F48060E74908600846006820F4805008600846006820F4006008603DE2FB
:205F0000E14B20221221E14801F034FADE4B4AF220020C2140F215700DF036F92EE24A4661
:205F20002146D948FDF7BBFDD74B20221221D7480DF093F8D449487B0EF0BAFCAFF22C533B
:205F40004AF603120C2140F215700DF01DF915E2CF4B10223A21CD4801F00CFACC4B4AF2F8
:205F600010120C2140F215700DF00EF906E24A462146C748FDF793FDC54B10223A21C348FD
:205F80000DF06BF8AFF274534AF603120C2140F215700DF0F9F8F1E1BE4B4AF230220C217C
:205FA00040F215700DF0F0F8BB4B4AF610420C2140F215700DF0E8F8E0E12022B749AD48F4
:205FC0004C380BF0BBFCB54B4AF220520C2140F215700DF0D9F8D1E1234618227E21AB4844
:205FE00001F0C8F9AE48C08AE082AD4B4AF218320C2140F215700DF0C7F8BFE1A94B41F268
:2060000001420C214FF4E2600DF0BEF8B6E14A462146A548FDF743FD002097490870AFF210
:206020000C634AF603120C214FF4E2600DF0ACF8FFF776F9A2E14A4621469B481030FDF753
:206040002EFD00208C490870AFF238634AF603120C214FF4E2600DF097F88FE14A46214672
:206060008E48FDF71CFD002083490870AFF25C634AF603120C214FF4E2600DF085F87DE19A
:206080004A46214689A0FDF741FD98B9AFF27C634AF603120C2140F215700DF075F800201A
:2060A0000BF00AF9642003F02FF801200FF01CF803F032FC62E14A462146AFF29860FDF728
:2060C00025FDE0B9FF2304220021704800F03EFA784968487C3800F0FFFB7749774800F03E
:2060E000FBFBAFF2D0634AF603120C2140F215700DF04AF801200EF0F7FF03F00DFC3DE12F
:206100004A4621466EA0FDF701FD90B90EF0D6FE5E4800F08DFAAFF204734AF603120C21B6
:2061200040F215700DF030F801200EF0DDFF03F0F3FB23E14A4621466448FDF7B0FC6348B5
:206140000078C0436249087060484078C043487000206049087003F0BDFA5E4948605B48A9
:2061600000785D4948735948407888730B464FF481520C214FF4E2600DF006F8FEE0574B5E
:206180004AF604220C2140F215700CF0FDFFF5E04A4621465148801CFDF781FC4F4B04228B
:2061A00034213A480CF059FFAFF298734AF603120C214FF4E2600CF0E7FF55204749C870E2
:2061C000DCE04648C078552803D04448C078AA2816D1AA204149C8704A4621463F48FDF772
:2061E0005EFC3E4B0422342128480CF036FFAFF2DC734AF603120C214FF4E2600CF0C4FFEA
:20620000BCE0207836490870B8E000BF20790006617900EB0140A17900EB0120E17908448B
:2062200021780906627801EB0241A27801EB0221E2781144401A00F1010820780006627809
:2062400000EB0240A27800EB0220E2788118424604F10800FDF723FC4AF60830404482B22F
:2062600023460C2140F215700CF08EFF00BF85E0F00700207CFC010875030020C80000200C
:20628000C900002044010020200700207C0300206007002070070020A0070020B00700200E
:2062A0005C11002048010020580600205245534554000000FFFF0108FFF3010800F00108EC
:2062C0005245434F5645525900000000CA000020CC00002074010020380600205201002013
:2062E0006B010020354B41F210520C214FF4E2600CF04AFF42E0324B41F208620C214FF45A
:20630000E2600CF041FF39E02E4B2022B4212E4801F030F82B4B4AF620520C2140F21570BB
:206320000CF032FF2AE04A4621462648FDF7B7FB244B2022B42124480CF08FFEAFF62C13BC
:206340004AF603120C2140F215700CF01DFF15E04A4621461DA0FDF7D9FB68B90EF088FDD7
:20636000194800F021F9AFF654134AF603120C2140F215700CF008FF00E000BF00BF19E013
:20638000A5F51450053820B1A0F5F840063828B900E000BF02201049087000E000BF00BF15
:2063A0002B463A4640F251610C4800940CF038FF00E000BF00BFBDE8F8830000A80800209F
:2063C0008C010020400700207C0300204C4F4720434C4541520000005D000020BC04002044
:2063E000704700BF0100A0F10100FBD1704710B50246002016E0135C041D145D63400B54EB
:20640000031DD35C00F10804145D6340041D0B55231DD35C0834145D634000F108040B557F
:20642000431CD8B20428E6DB10BD00001FB54FF460400090112001900220039069461948EB
:2064400002F0A8FF4FF4E060009011200190022003906946144802F09DFF00224FF480712A
:20646000114803F031F900224FF400710E4803F02BF900224FF480610B4803F025F9002297
:206480004FF40051074803F01FF900224FF48041044803F019F900224FF40041014803F0B5
:2064A00013F91FBD000C01400008014010B500210D4804F0EFFB04210B4804F0EBFB0821CA
:2064C000094804F0E7FB0021074804F083F80421054804F07FF80821034804F07BF80C21D1
:2064E000014804F0B7FB10BD88120020F8B50446002000906A460021204600F00DF90DF154
:2065000001020121204600F007F902216846FEF7FBFA06466A460221204600F0FDF80DF1DD
:2065200001020321204600F0F7F89DF801009DF8001000EB012085B2A81B03D12046FEF77F
:2065400085FDF8BD2046FEF79DFEFAE72DE9F04780460C4616461F46301B00F0FF0900259F
:2065600007E06019C1B23A46404600F02BF9681CC5B24D45F5DBBDE8F08700001FB5044697
:20658000022000900120019003906946054802F001FF01220221034803F096F8204604F0AA
:2065A00063FF1FBD000C014010B504461C4B30224C2120460CF051FD401C28B9184B302279
:2065C0004C2120460CF049FD164B1022EC2120460CF043FD401C28B9124B1022EC21204625
:2065E0000CF03BFD104B1022D62120460CF035FD401C28B90C4B1022D62120460CF02DFD06
:206600000A4B1022A22120460CF027FD401C28B9064B1022A22120460CF01FFD10BD0000DC
:2066200070070020A0070020A8080020B808002010B50446314B0C22042120460CF00DFD02
:20664000401C28B92D4B0C22042120460CF005FD2B4B0822982120460CF0FFFC401C28B9DB
:20666000274B0822982120460CF0F7FC254B2022122120460CF0F1FC401C28B9214B202251
:20668000122120460CF0E9FC1F4B2022B42120460CF0E3FC401C28B91B4B2022B42120469E
:2066A0000CF0DBFC194B10223A2120460CF0D5FC401C28B9154B10223A2120460CF0CDFC8E
:2066C000134B0422342120460CF0C7FC401C28B90F4B0422342120460CF0BFFC0D4B1822FB
:2066E0007E2120460CF0B9FC401C28B9094B18227E2120460CF0B1FC10BD00003408002042
:2067000057010020200700204007002060070020520100205C1100202DE9F04106460F46E4
:2067200015460024304604F012FFA021304604F053FF00BF00BF601C84B240F6B8308442CE
:2067400003DD4FF0FF30BDE8F081304604F06CFE0028F0D13946304604F03EFF002400BF0F
:20676000601C84B240F6B830844202DD4FF0FF30E9E7304604F058FE0028F1D1304604F052
:20678000E6FEA121304604F027FF002400BF601C84B240F6B830844202DD4FF0FF30D2E744
:2067A000304604F041FE0028F1D12946304604F078FE304604F0A8FE304604F0E8FE002077
:2067C000C1E700002DE9F04106460F461546002400220221294802F077FF304604F0B7FE6D
:2067E000A021304604F0F8FE00BF00BF601C84B240F6B830844203DD4FF0FF30BDE8F08100
:20680000304604F011FE0028F0D13946304604F0E3FE002400BF601C84B240F6B8308442D3
:2068200002DD4FF0FF30E9E7304604F0FDFD0028F1D12946304604F0CFFE002400BF601CE8
:2068400084B240F6B830844202DD4FF0FF30D5E7304604F0E9FD0028F1D1304604F097FEDC
:206860000A2002F051FC01220221044802F02CFF034802F05DFF0020C0E70000000C014053
:2068800004060020F8B50E480468001D0568200E8DF80000200C8DF80100200A8DF80200BF
:2068A000E0B28DF8030004216846FEF745F90646701B02D1FEF76CFB01E0FEF78FFCF8BD9C
:2068C00000FC010810B50446207818B9FEF786FC0120207010BD000038B504460D4600209C
:2068E0000C49086008468460281B401C800AC86002F0D8FC00BF34200749C86000BF694699
:20690000044802F015FC02F06BFC642002F0FCFB38BD0000D81100200020024010B590B0FD
:20692000042269460E480BF009F80446ACB9042269460CA0FDF7EAF878B9282269460848B0
:2069400008300AF0FBFF04463CB9282269460748FDF7A5F8002010B010BD0120FBE7000043
:2069600000E80108464C4147000000000008002010B54FF4805002F0FFFC10BD10B5042069
:2069800002F0FAFC10BD00001FB54FF4604000900220019003906946064802F0FBFC4FF48C
:2069A000E06000900220019003906946024802F0F1FC1FBD000C01400008014010B5002191
:2069C000104804F047F904210E4804F043F908210C4804F03FF90C210A4804F03BF900210F
:2069E000084803F0E1FD0421064803F0DDFD0821044803F0D9FD0C21024803F0D5FD0AF0C2
:206A0000E1FC10BD881200202DE9F04107460C46207860BB384600F057F846B2701C48B13F
:206A20001448402101FB06054022394628460CF0E7FA1AE00F49491E0F48FFF74DFFF02202
:206A40000C4940310C4800F019F90C490948FFF743FFF0220849074800F010F9074D3F3DC1
:206A60004022394628460CF0CBFA01202070BDE8F081000000F0010800EC0108FFF3010856
:206A800010B504460B480068A0600B484068E06020220A4904F11000FDF701F808480168B1
:206AA00021634068606307480168A1634068E06310BD000044010020700700203806002019
:206AC0008C010020CE00002010B50246002116E00F4C04EB811003884FF6FF7083420CD13B
:206AE00011B90120108006E04020C0EB8110084C035B581C1080084610BD481C41B2102938
:206B0000E6DB04480388581C10804FF0FF30F3E700F00108C0F301080021074AD1610749E8
:206B2000096941F00401054A11611146096941F040011161704700001806002000200240E8
:206B40000021074AD1610749096941F00201054A116111464861096941F0400111617047CD
:206B600018060020002002400022054BDA61054A126942F00102034B1A61018070470000C8
:206B8000180600200020024000201E49C96801F0100139B11C49C96941F002011A4AD16150
:206BA00040F010001749C96801F0040139B11649C96941F00101144AD16140F00400114942
:206BC000C96901F0010169B10F49C96941F004010D4AD16100BF0B49C96921F00101094A82
:206BE000D16100BF00BF40F20111884206D10549C96921F00101034AD16101E00149C8609B
:206C000000BF7047002002401806002070B5044602F060FD054609E0601C38B124B102F040
:206C200059FD401BA04201D9032070BD1248C06800F001000028EFD10F48C06800F02000AD
:206C400020B100BF20200C49C86000BF0A48C06800F0100048B90848C06900F0010020B96A
:206C60000548C06800F0040018B1FFF78DFF0120DBE70020D9E70000002002402DE9F041F4
:206C800004460E461746002502F00CFB00BF0FE056F825C0624600232146022002F0AAFA10
:206CA00008B9241D03E002F09BFABDE8F0816D1CBD4202D203488442EAD902F091FA00BFE6
:206CC000F3E70000FBFF0108022005490870002004490880488004490880488070470000DE
:206CE00030000020280000202C0000200120014908707047300000202DE9FF4705460E46CB
:206D000017464FF0000A0CF099F803900398FEF70DF9029039B202980AF068F9009071485C
:206D200000990160B0F900006F490968C1EB80206D49096801EBA0206B4908600846006896
:206D4000801200B2694908806648B0F9020068490968C1EB80206649096801EBA020644975
:206D6000086008460068801200B2624908806248007C002849D161480078042845D160480B
:206D8000408840F6EC01884210DA5E4805605E48006810F1040F05DA5B480068001D5A497D
:206DA000086042E00020584908603EE05448408840F6BE11884221DA51484088A0F6EC00F1
:206DC00000EB800040F21A41081A5049086008460068854201DA284601E04C480068494963
:206DE000086049480068801E474908600846006810F5D27F19DA4648086016E00020414907
:206E000008604348404908600FE03E4805603E48006810F1040F05DA3B480068001D3A4948
:206E2000086002E00020384908603A4A2F48B0F900103448008800B20AF098F80446364843
:206E40000068C0EB44203449096801EBE0003249086032484088B7214843C0F3CF1947F6A1
:206E600098107043B9F57A7F02DA4FF47A7100E0494690FBF1FA284800680AEB602447F693
:206E80009810844200DD00E02046044620B224490880244A1748B0F900101B48008800B22D
:206EA0000AF064F8804620480068C0EB48201E49096801EBE0001C4908600846006840125A
:206EC00000B21749488008460AF07EFD1448006800900AF09FFD019001980BF003FDBDE861
:206EE000FF870000280000200400002018000020080000201A000020BC100020CE0000202C
:206F000048130020200000201C000020240000205CFEFFFF100500201000002060070020F2
:206F20002C000020340500201400002004F0A2FB09F0A8FC09F048FD62B60020124981F800
:206F40003C0009F057FC72B609F01EFD0AF042FAFFF76CFA00200D4908600846006820F433
:206F6000005000F5005008600DE0084B41F204120C214FF4E2600CF007F9C8200BF092FC6C
:206F8000034802F0D5FBF0E77C180020440100200406002070B505460E46049CAC4204DA9A
:206FA000281B7043C0F5806108E0944202DA4FF4806103E0A01A5843C0F58061002901DCB3
:206FC000002000E00846014688B270BD87B0014600220868009048680190C86803903D488C
:206FE00081423AD04FF0553008600A68B2F1553F02D0002007B070474FF0AA3008600A689C
:20700000B2F1AA3F01D00020F4E74FF0553048604A68B2F1553F01D00020EBE74FF0AA30E7
:2070200048604A68B2F1AA3F01D00020E2E745F25550C860CA6890B245F25553984201D0AE
:207040000020D7E74AF6AA20C860CA6890B24AF6AA23984235D00020CCE700986FF30B00E8
:2070600000F2555008600A68C2F30B0040F25553984201D00020BDE700986FF30B0000F69B
:20708000AA2008600A68C2F30B0040F6AA23984201D00020AEE7039820F00700C01DC86072
:2070A000CA6802F00700072801D00020A2E7039820F00700C860CA6802F0070008B100201E
:2070C00098E700980860019848600398C860012090E70000001401402DE9F04104460E465B
:2070E000154629480078012812D1284801780078401C264A1070264820F8116010460078CE
:20710000322810DB002020490870114608700AE032221F49304609F0E3FD643087B22088F0
:20712000B84200DD00BF2888C0F3C03050BB208840F2DC51884203DC02F0CCFA154908602D
:2071400002F0C8FA13490968401A42F21071884218D9286820F4004000F500402860012022
:207160000D494880208888800846FFF789FC00200A4908700A488088401C0949888002205B
:2071800008490870BDE8F081C7030020C803002024120020CC0300207C100020EC0200203C
:2071A000A007002056010020B1F5967F03DA0122044B1A7002E00022024B1A7001F16402CA
:2071C00002807047C603002038B5044601234FF47A720A210248009404F006FB38BD000010
:2071E0001012002030B503460024002204E033F812502C44551CAAB28A42F8DBB4FBF1F5F7
:20720000A8B230BD70B505462A480078012811D100202849087002F05DFAB0F5E16F05D99D
:2072200002F058FAC8302449088003E04FF4FA602149088002F04EFA1F490988884236D99F
:207240001E480078012832D11D48007858B11D480088C82807DC40F2C270854207DD40F639
:207260003E00854203DA00201749C8721CE001201549C872002415E0144830F81400A84222
:207280000EDB092212A11548FCF72DFC1448015D1248203880F8271000200849087070BD7D
:2072A000601CC4B2092CE7DB00200449087000BFF5E70000D2030020D00300209A010020C2
:2072C0006C01002068010020BC100020387E010854544B5A303139412E00000078060020F9
:2072E0004A7E010810B502460B460020002107E032F81140844201DD32F811004C1CA1B222
:207300009942F5DB10BD10B502460B464FF6FF70002107E032F81140844201DA32F8110084
:207320004C1CA1B29942F5DB10BD00000246002108E0064830F81100904201DC084670478E
:20734000481CC1B2C829F4DB0020F8E72A7B01080246002108E0064830F81100904201DC62
:2073600008467047481CC1B2BF29F4DB0020F8E7BA7C01082DE9F047C2B082460D46144608
:207380001F4600260FE002A88219A819C1B25046FFF7C2F9401C20B94FF0FF3042B0BDE879
:2073A000F087701CC6B2A642EDDB214602A8FDF7ABFB81462819C1B201AA5046FFF7ACF9A0
:2073C0002819401CC1B20DF105025046FFF7A4F99DF805009DF8041000EB01201FFA80F88F
:2073E000B8EB090006D1224602A93846FCF757FB0020D3E74FF0FF30D0E72DE9FC5F8046FE
:2074000089464FF0000A002549464046FFF7EAFE8346002407E038F81400ABEB000505FB89
:2074200005AA601C84B24C45F5DB5046FCF796FB06460F46304639460EF0B2F9CDE900017A
:20744000FCF79DFB05462846BDE8FC9FF8B5044600260020009000BF94F82400012801D171
:207460000220F8BD012084F8240000BF2046FCF7C1FC0646002E62D1A06A20F4885040F0CC
:207480000200A062022002F069FA30490968B1FBF0F04000009002E00098401E009000982B
:2074A0000028F9D12046FCF70DFD2068806840F008002168886002F00DF9054611E002F038
:2074C00009F9401B0A280CD9A06A20F0020040F01000A06200BF002084F8240000BF01207B
:2074E000BFE72068806800F008000028E7D12068806840F004002168886002F0EBF8054669
:2075000011E002F0E7F8401B0A280CD9A06A20F0020040F01000A06200BF002084F824005A
:2075200000BF01209DE72068806800F004000028E7D1A06A20F0020040F00100A06200BF95
:20754000002084F8240000BF30468AE70000002038B50246002300200090906800B100BF35
:2075600000BF92F82400012801D1022038BD012082F8240000BF906890B94868012809D11A
:207580001068806B6FF315000C6840EAC4301468A06338E0906A40F020009062012332E076
:2075A0000C694868A0421ED84C680869001BC0F1030000EB80041F20A04040F4401410684C
:2075C000806BA0434D680C69641BC4F1030404EB84050C68AC400D8A6D1E44EA0554204394
:2075E0001468A0630FE04C680869001BC0F1030000EB80041F20A04040F440141068806BB0
:20760000A0431468A0631068806800F0010040B91068806847F20104A043CC692043146829
:20762000A060886901280FD1C869B0F5E04F06D11068406840F480601468606004E0906A26
:2076400040F0200090620123486901280DD1886930B91068406840F480501468606004E0EE
:20766000906A40F020009062012308680A2812D31068C0680C780A3C04EB44050724AC406A
:20768000A0430D780A3D05EB45058C68AC4020431468E0600FE0106800690C7804EB440576
:2076A0000724AC40A0430D7805EB45058C68AC402043146820610868102802D008681128AE
:2076C00005D11068806840F400001468A0604868012806D002280DD0032814D004281BD1E7
:2076E0001BE0106840696FF30B00CC682043146860611BE0106880696FF30B00CC682043CD
:207700001468A06112E01068C0696FF30B00CC6820431468E06109E000BF1068006A6FF3AC
:207720000B00CC6820431468206200BF00BF0868102802D00868112827D1174C1068A04253
:207740001ED11068806800F40000F0B91068806840F400001468A0600868102815D10F4848
:2077600000680F4CB0FBF4F000EB80004000009002E00098401E009000980028F9D104E0A6
:20778000906A40F020009062012300BF002082F8240000BF1846E9E600240140000000209B
:2077A00040420F0010B504460121204600F044F84FF6FF7101EA00101A4948800221204611
:2077C00000F03AF84FF6FF7101EA0010154988800321204600F030F84FF6FF7101EA00101F
:2077E00010490880104800880988401A00B20F4908800D4840880B494988401A00B20B49A9
:2078000048800948808807498988401A00B2074988800749054809F031FC012005490870D8
:2078200010BD0000E0030020F2030020F8030020FE030020EC0300200246002001290FD0A7
:20784000022909D0032904D0042908D11368986C09E01368586C06E01368186C03E000BFF0
:207860001368D86B00BF00BF7047000070B50446002500BF94F82400012801D1022070BDC8
:20788000012084F8240000BF2046FCF71BFB0546002D5BD1A06A42F20101884340F4805046
:2078A000A0622E492068884208D12D48006800F4702008B9012002E0002000E0012020B10D
:2078C000A06A20F48010A06203E0A06A40F48010A062A06A00F4807008B90020E06200BF75
:2078E000002084F8240000BF401F216808602068406840F08000216848602068406800F484
:20790000806010BB2068806800F4E040B0F5E04F15D112492068884208D11148006800F443
:20792000702008B9012002E0002000E0012030B12068806840F40210216888600BE0206857
:20794000806840F400402168886004E000BF002084F8240000BF284691E7000000280140E9
:207960000424014038B5024600230020009000BF92F82400012801D1022038BD012082F87C
:20798000240000BF4868072812D21068406B0C79641E04EB84051F24AC40A0430D796D1E7C
:2079A00005EB85050C68AC4020431468606327E048680D2812D21068006B0C79E41F04EB21
:2079C00084051F24AC40A0430D79ED1F05EB85050C68AC4020431468206311E01068C06AAB
:2079E0000C790D3C04EB84051F24AC40A0430D790D3D05EB85050C68AC4020431468E06264
:207A000008680A2812D31068C0680C780A3C04EB44050724AC40A0430D780A3D05EB45053D
:207A20008C68AC4020431468E0600FE0106800690C7804EB44050724AC40A0430D7805EB4C
:207A400045058C68AC402043146820610868102802D00868112827D1174C1068A0421ED1D5
:207A60001068806800F40000F0B91068806840F400001468A0600868102815D10F480068AC
:207A80000F4CB0FBF4F000EB80004000009002E00098401E009000980028F9D104E0906AF1
:207AA00040F020009062012300BF002082F8240000BF184661E700000024014000000020F9
:207AC00040420F0070B50646B4480068401CB349086008460068B0F5967F01D900200860AE
:207AE000AF480078012805D14120AE4948758875C87599E0AC48C07A012808D1AB480078B5
:207B0000012804D10020A949087008F039FDA8480088A84909680844A6490860A44880883E
:207B2000A54909680844A4490860A148C089A34909680844A1490860A1480088401CA04962
:207B400008800846008840F6B83188426CDB9648C07A012822D197480068B0FBF1F085B259
:207B60002846FFF7F5FB8F4948759348006840F6B831B0FBF1F085B22846FFF7E9FB8949DD
:207B800088758E48006840F6B831B0FBF1F085B22846FFF7DDFB8349C8753CE08548006832
:207BA00040F6B831B0FBF1F085B22846FFF7BEFB7C4948758048006840F6B831B0FBF1F069
:207BC00085B22846FFF7B2FB764988757D48007801280ED10846407D7B49087077480068EE
:207BE00040F6B831B0FBF1F0784908800020754908707248006840F6B831B0FBF1F07349B2
:207C00000988081A00EB400080016F49097801EBA0206449C87500206949088065490860C6
:207C200065490860654908606148408868490968C1EB80206649096801EB60206449086098
:207C400008460068801244F2CE714843C0F38F205449C8800846C1880089C01101EBC000F8
:207C60005049C8805B48007803280BD10846C088A0F5F850A43840F27A514843C0F38F20C8
:207C80004849C8804848C07A012809D14848C08851490988401A49F619214843841208E05F
:207CA0004348C0884C490988401A4CF250314843C412002C01DC002005E04CF250308442BF
:207CC00000DB00E02046044644480068C0EB84204249096801EB60204049086008460068E7
:207CE000C0F38F202F4908813D48C078AA2811D02F4800893B49C98A401A642148433849EF
:207D0000897890FBF1F4002C01DC002000E02046044607E0334AD18A254A1089304A0CF0FC
:207D200033F9044630490C8030480078D8B9204880892F490988441A002C01DC002000E066
:207D4000204604462B480068C0EB84202949096801EB20202749086008460068C0F38F204A
:207D60002149488002E000201F4948801048408921490968C1EB80201F49096801EB602012
:207D80001D49086008460068C0F38F201B4908800749488809F052FA70BD00000804002053
:207DA0009A01002038060020BC10002030040020481300201C04002018040020200400202F
:207DC000140400202404002025040020260400200C0400209401002004040020100400204F
:207DE000520100205C110020EE030020C6030020C4030020280400202C040020980100204D
:207E00007047704710B504462068406800F0200020282FD12068006800F00200022829D157
:207E2000A06A00F0100018B9A06A40F40070A0622068806800F46020B0F5602F13D1E06873
:207E400088B92068406820F0200021684860A06A20F48070A062A06A00F4805018B9A06A97
:207E600040F00100A0622046FFF72CFE6FF01200216808602068406800F0800080283BD193
:207E80002068006800F00400042835D1A06A00F0100018B9A06A40F40050A06220688068F1
:207EA00000F4E040B0F5E04F0DD02068406800F48060D0B92068806800F46020B0F5602F58
:207EC00013D1E06888B92068406820F0800021684860A06A20F48050A062A06A00F4807066
:207EE00018B9A06A40F00100A0622046FFF75AFC6FF00C00216808602068406800F0400006
:207F000040280FD12068006800F0010050B1A06A40F48030A062204600F0A8F86FF00100F1
:207F20002168086010BD00002DE9F0410446002700250026A84614B90120BDE8F081A06886
:207F400010B1606900B100BFA06A30B90020E06284F82400204600F08BF82046FBF74AFFB8
:207F60000746A06A00F01000002873D1002F71D1A06A20F4885040F00200A062E169606891
:207F80000843E16840EA41000643A068B0F5807F02D0A068012802D14FF4807000E00020E4
:207FA00005436069012811D1E06838B9A069401E4FF4006141EA4030054307E0A06A40F05D
:207FC0002000A062E06A40F00100E0622068406820F469402843216848602068806821495F
:207FE0000840304321688860A068B0F5807F02D0A068012802D14FF4807000E00020B0F5FB
:20800000807F03D1208A401E4FEA00582068C06A20F4700040EA08002168C8622068806869
:2080200011490840B04208D10020E062A06A20F0020040F00100A06211E0A06A20F0020015
:2080400040F01000A062E06A40F00100E062012705E0FFE7A06A40F01000A062012738463C
:208060006BE70000FDF7E1FFFE0E1FFF7047000010B586B004463249206888423CD100BF1B
:208080003048806940F400702E4988610846806900F40070019000BF00BF1F2002900320DD
:2080A000039002A9284801F075F9A02002900320039002A9254801F06DF9254825490860F9
:2080C000002048600021234881608021C1604900016189004161202181610021C16100F07D
:2080E0008DFF20B14FF48B711BA00CF025FF00BF18482062446221E01C49206888421DD11C
:2081000000BF1048806940F480600E4988610846806900F48060019000BF00BF0E20029031
:208120000320039002A9094801F034F901221146122001F09EFB122001F08EFB06B010BD0A
:208140000024014000100240001001400008014008000240CC1300202E2E5C436F72655CE8
:208160005372635C6164632E630000000028014070B50446002500BF94F82400012801D15B
:20818000022070BD012084F8240000BF2046FBF799FE0546002D77D1A06A40F20121884338
:2081A00040F48070A0623C492068884208D13B48006800F4702008B9012002E0002000E0B6
:2081C000012078B1A06A20F48010A0622068406800F4806000B3A06A20F4005040F480507C
:2081E000A06219E0A06A40F48010A0622B49091F2068884203D028492068884204D12748EC
:20820000006800F4806000E0002028B1A06A20F4005040F48050A062A06A00F4805020B136
:20822000E06A20F00600E06201E00020E06200BF002084F8240000BFC01E216808602068C4
:20824000806800F46020B0F5602F16D112492068884208D11148006800F4702008B90120FA
:2082600002E0002000E0012038B12068806840F4A000216888600CE006E02068806840F4E7
:2082800080102168886004E000BF002084F8240000BF284675E7000000280140042401401F
:2082A0002DE9F04104460D461646002757492068884203D056492068884205D15348001D13
:2082C000006800F4702000E0002000287ED100BF94F82400012802D10220BDE8F081012077
:2082E00084F8240000BF2046FBF7ECFD0746002F6DD1A06A40F60161884340F48070A06291
:2083000043492068884209D14048001D006800F4702008B9012002E0002000E0012078B106
:20832000A06A20F48010A0622068406800F4806000B3A06A20F4005040F48050A06219E069
:20834000A06A40F48010A06230492068884203D02F492068884205D12C48001D006800F422
:20836000806000E0002028B1A06A20F4005040F48050A062A06A00F4805020B1E06A20F0D7
:208380000600E06201E00020E06200BF002084F8240000BF1F48216A88621F48216AC8621C
:2083A0001E48216A08636FF00200216808602068806840F4807021688860226802F14C0140
:2083C00033462A46206A00F051FE01E01AE014E02068806800F46020B0F5602F06D12068A5
:2083E000806840F4A000216888600CE02068806840F480102168886005E000BF002084F87F
:20840000240000E00127384667E700000024014000280140473E0008B73E0008993E00082D
:2084200030B5024600230C7D012000FA04F31068D0F8000220F47C5001254C6A45EA0424FC
:2084400020431468C4F800021068D0F81C0298431468C4F81C02C869E8B91068D0F80C02D0
:2084600098431468C4F80C02888880B28C8940EA0444106800F510704D6940F83540088832
:2084800080B20C8940EA0444106800F510704D6900EBC5004460C86901281DD11068D0F824
:2084A0000C0218431468C4F80C02888880B20C8840EA0444106800F510704D6940F8354075
:2084C000888980B20C8940EA0444106800F510704D6900EBC5004460886938B91068D0F839
:2084E000040298431468C4F8040206E01068D0F8040218431468C4F80402086938B91068BE
:20850000D0F8140298431468C4F8140206E01068D0F8140218431468C4F81402086A0128D4
:2085200006D11068D0F81C0218431468C4F81C021068D0F8000220F001001468C4F80002C8
:20854000002030BD0168496941F0020102685161704700002DE9F0410446002500260027E9
:20856000A8462068C068C0F3001520684069C0F3C0062DB126B148F4007810202168C860A1
:2085800020680069C0F3001520684069C0F380162DB126B148F48068102021680861206825
:2085A000406900F0010000283BD0206880687A490840884201D1012000E0002005462068E3
:2085C000806876490840884201D1012000E0002006462068806872490840884201D1012073
:2085E00000E0002007460DB906B9D7B120688068C0F3400520688068C0F3402620688068C0
:2086000000F001070DB906B91FB12046FCF71CFA01E048F40068206880686249084321682A
:2086200088602068C06800F0030520684069C0F3400625B11EB100212046FBF7B7FF206824
:20864000006900F0030520684069C0F3001625B11EB101212046FBF7A9FF206C40EA08003A
:2086600020642068806900F0010520684069C0F3002620684069C0F3C0372DB126B11FB1A5
:20868000206C40F00100206420688069C0F3400520684069C0F3402620684069C0F3C0370B
:2086A0002DB126B11FB1206C40F00200206420688069C0F3800520684069C0F38026206838
:2086C0004069C0F3C0372DB126B11FB1206C40F0040020642068806900F0700008B90120CB
:2086E00000E00020054620684069C0F3C02620684069C0F3C03795BB8EB387B3206880694E
:2087000000F07005402D1BD006DC102D09D0202D0CD0302D24D10EE0502D16D0602D1FD15B
:2087200018E0206C40F0080020641AE0206C40F01000206415E0206C40F02000206410E06A
:20874000206C40F0400020640BE0206C40F08000206406E0206C40F48070206401E007E00C
:2087600000BF00BF2068806920F0700021688861206C78B1042021684860012084F83C0035
:208780002068406948F65B718843216848612046FFF7D8FEBDE8F08101000004000100084B
:2087A00000000110090501002DE9F041044600270026002514B90120BDE8F08194F83C00CA
:2087C00028B9002084F83D00204600F0A5F8022084F83C002068006820F00200216808601F
:2087E0002068006840F001002168086000F072FF06460EE000F06EFF801B0A2809D903209D
:2088000084F83C0000BF002084F83D0000BF0320D2E72068406800F001000028EAD02068E2
:20882000406800F00100002867D0A069012802D145F0800501E025F08005E069012802D1C1
:2088400045F0400501E025F04005206A012802D145F0200501E025F02005606A012802D1A2
:2088600045F0100501E025F01005A06A012802D145F0080501E025F00805E06A012802D112
:2088800045F0040501E025F004052068006820F0FC00284321680860D4E9020108432169AE
:2088A0000843616908436168491E08432168C8612068006820F001002168086000F00AFF40
:2088C00006460EE000F006FF801B0A2809D9032084F83C0000BF002084F83D0000BF032065
:2088E0006AE72068406800F001000028EAD12068406800F0010000B90127012F06D10020FA
:208900002064012084F83C00002055E7042084F83C00012050E7000010B586B004462449B8
:208920002068884242D100BF2248C06940F000702049C8610846C06900F00070019000BF27
:2089400000BF8815029000200390049002A91A4800F020FD4FF400700290022003900320AB
:20896000059002A9144800F015FD00BF1349486820F4C04040F0E06040F48040486000BFAF
:2089800001221146142000F074FF142000F064FF0B4820630B486063FBF7BAFD0A480068F0
:2089A000406940F0020008490968486106B010BD0064004000100240000C0140000001406A
:2089C000401400205C1400207C18002010B50446606B806810B9606B006940B92E48006849
:2089E000406940F002002C490968486110BD606B006840F23172811A904214D009DCA0F270
:208A0000516080B3CF2818D0D02817D0DF2837D108E00F291CD010291BD01F2924D02029F0
:208A20002ED122E000BF606B00881C490880606B017C1A48FBF776FF23E000BF606B008810
:208A400017490880606B017C1548FBF76BFF18E000BF606B008813490880606B017C11489E
:208A6000FBF760FF0DE001E000BF00BF606B00880D490880606B017C0B48FBF753FF00E069
:208A800000BF00BF04480068406940F0020002490968486100BFA9E77C1800205C040020E1
:208AA0007004002084040020980400202DE9F04104460E46042500272068806800F0806049
:208AC000B0F1806F0DD02068806800F00060B0F1006F06D02068806800F08050B0F1805FD3
:208AE0007ED100BF94F83D00012802D10220BDE8F081012084F83D0000BF94F83C002228C0
:208B000004D0322806D062280CD107E0422084F83C000BE0522084F83C0007E0722084F8DF
:208B20003C0003E0122084F83C0000BF00BF2068806800F0806008B1002507E02068806839
:208B400000F0006008B1012500E00225206800F5C07000EB0510006800F00101206800F55B
:208B6000C07000EB05100160206B806898B9206800F5C07000EB05100068216BC968226B41
:208B8000128841EA42510843216801F5C07101EB0511086015E0206800F5C07000EB051076
:208BA0000068216B8968226B526841EAC201226BD26811430143206800F5C07000EB05108F
:208BC0000160206B007C00F00F00216B0861206800F5C07000EB0510406820F00F0100E0E4
:208BE000B1E0206800F5C07000EB05104160206800F5C07000EB05104068216B09690843F8
:208C0000216801F5C07101EB05114860206BC07D0106206B807D41EA0041206B407D41EAC4
:208C20000020216B097D0843216801F5C07101EB05118860206BC07E0106206B807E41EA99
:208C40000041206B407E41EA0021206B007E0143206800F5C07000EB0510C160206800F5A6
:208C6000C07000EB0510006840F00101206800F5C07000EB0510016000F02CFD074620E0B6
:208C8000701CF0B126B100F025FDC01BB04218D9032084F83C001DB980202168886009E055
:208CA000012D03D1E8032168886003E04FF400002168886000BF002084F83D0000BF032045
:208CC00015E74DB92068806821490840884201D1012016E0002014E0012D09D12068806831
:208CE0001C490840884201D101200AE0002008E02068806818490840884201D1012000E062
:208D000000200028BCD094F83C00422804D0522806D072280CD107E0222084F83C000BE0E6
:208D2000322084F83C0007E0622084F83C0003E0012084F83C0000BF00BF00BF002084F873
:208D40003D0000BFD3E6042084F83C000120CEE6010000040001000800000110704710B512
:208D600004460CB9012010BD607920B900202071204600F005F8012060710020F3E7000054
:208D800008B5094A016891420DD100BF0749496941F04001054A51611146496901F040013A
:208DA000009100BF00BF08BD003002400010024070B50446002594F82100022803D00420B9
:208DC000A063012548E02068006820F00E00216808602068006820F00100216808601F49E9
:208DE0002068884201D1012026E01C4914312068884201D110201FE018492831206888421F
:208E000001D1801518E015493C312068884201D1801411E0114950312068884202D14FF43C
:208E2000803009E00D4964312068884202D14FF4801001E04FF0807008490839486001204B
:208E400084F8210000BF002084F8200000BF606B10B12046616B8847284670BD08000240C9
:208E600070B50446E06B05682068066894F84010042088402840002846D006F00400002845
:208E800042D02068006800F0200028B92068006820F004002168086057492068884201D126
:208EA000042027E0544914312068884201D1402020E0514928312068884201D1001519E0FC
:208EC0004D493C312068884202D14FF4804011E0494950312068884202D14FF4802009E072
:208EE000454964312068884202D14FF4800001E04FF08060404908394860E06A00287AD039
:208F00002046E16A884776E094F84010022088402840A0B306F0020088B32068006800F0E7
:208F2000200040B92068006820F00A0021680860012084F8210030492068884201D10220A0
:208F400028E02D4914312068884201D1202021E0294928312068884201D140151AE026493C
:208F60003C312068884202D14FF4005012E0224950312068884203D14FF400300AE017E074
:208F80001D4964312068884202D14FF4001001E04FF0007018490839486000BF002084F829
:208FA000200000BFA06A30B32046A16A884722E094F84010082088402840E0B106F00800E0
:208FC000C8B12068006820F00E002168086094F8401001208840E16B48600120A06384F8C0
:208FE000210000BF002084F8200000BF206B10B12046216B884770BD080002400146002229
:2090000009B901207047184B0868C01A1423B0FBF3F08000086414480838C863022081F8F6
:2090200021000868026843F6F0708243D1E901031843CB6818430B6918434B6918438B695E
:209040001843CB69184302430868026000208862C862086348638863012081F821000020FF
:2090600081F8200000BFCDE7080002402DE9F04104460D4616461F464FF0000800BF94F863
:209080002000012802D10220BDE8F081012084F8200000BF94F8210001282CD1022084F88F
:2090A00021000020A0632068006820F00100216808603B46324629462046FCF747FAE06A2E
:2090C00030B12068006840F00E00216808600BE02068006820F004002168086020680068C0
:2090E00040F00A00216808602068006840F001002168086006E000BF002084F8200000BF13
:209100004FF002084046BFE770B5044600F0E2FA06462546681C10B104480078054400BFD7
:2091200000F0D8FA801BA842FAD370BD580000202DE9F04104460E460127002500BF264817
:20914000007E012802D10220BDE8F08101202249087600BF2068022813D14CF25030FDF74C
:2091600055FD90BB0120FDF7D7FC4CF25030FDF74DFD07461948006920F00400174908617A
:2091800023E04CF25030FDF741FDF0B94FF0FF303060A56812E02846FDF7D2FC4CF2503048
:2091A000FDF734FD07460D48006920F002000B4908610FB1356007E005F58065D4E90210C6
:2091C00001EB8020A842E6D800BF00BF00200249087600BF3846B7E7180600200020024079
:2091E0000348006940F080000149086100207047002002402DE9FE4F05468B461746984665
:20920000012600240020029000BF2448007E012802D10220BDE8FE8F01202049087600BF91
:209220004CF25030FDF7F2FC064686BB012D02D10120029006E0022D02D10220029001E0D0
:209240000420029000241EE02201B946C24648465146FAF714FC80B20190022000FB04B052
:2092600000900199FDF780FC4CF25030FDF7CEFC06460B48006920F001000949086106B14D
:2092800004E0601CC4B202988442DDDB00BF00BF00200249087600BF3046BBE71806002064
:2092A0000020024000200849096901F0800151B10649054A5160064951601146096901F0EC
:2092C000800101B1012070470020024023016745AB89EFCD10B50446042C3BD1002021498C
:2092E000C8700846807840B900F0F4F91D494860601F88600120887011E000F0EBF9194965
:209300004968401A17498860084680684B2802D215480068886000F0DDF9124948601148AE
:209320008068114908600F4880684B2818D30F480068401C0D4908600D48007E08B9012058
:2093400001E00B48007E09490968B1FBF0F00549C86005E0B4F5805F02D10120054908706F
:2093600010BD00003C0300205804002054040020200700206002002010B504460448006841
:20938000204020B1024804602046FFF7A3FF10BD140401402DE9F8470346002400200025C3
:2093A0008446002700226EE14FF0010808FA02F4D1F8008008EA0400A0427DD1DFF8D0A253
:2093C000D1F80480A8EB0A09D0453AD014DCB8F1030F50D009DCB8F1000F31D0B8F1010F59
:2093E0001CD0B8F1020F49D120E0B8F1110F18D0B8F1120F42D11EE0B9F5881F25D006DCF5
:20940000B9F5803F20D0B9F5801F37D11AE0B9F5001F18D0B9F5041F30D117E0D1F80CC08D
:209420002DE0D1F80C8008F1040C28E0D1F80C8008F1080C23E0D1F80C8008F10C0C1EE0F0
:2094400000BF00BF00BF00BF00BF00BFD1F80880B8F1000F02D14FF0040C0BE0D1F808802B
:20946000B8F1010F03D14FF0080C1C6102E04FF0080C5C6103E04FF0000C00E000BF00BF11
:20948000FF2801D8984601E003F104084646FF2802D84FEA820803E0A2F108084FEA88086E
:2094A0004746D6F800804FF00F0909FA07F928EA09080CFA07F900E088E048EA0908C6F805
:2094C0000080D1F8048008F08058B8F1805F7DD100BFDFF8C081D8F8188048F00108DFF8C2
:2094E000B491C9F81880C846D8F8188008F00108CDF8008000BF00BF4FEAB9384FEA920996
:2095000058F829504FEA82784FEA18794FF00F0808FA09F825EA0805DFF87C81434502D1E1
:209520004FF0000816E0DFF87481434502D14FF001080FE0DFF86881434502D14FF002082C
:2095400008E0DFF86081434502D14FF0030801E04FF004084FEA82794FEA197908FA09F898
:2095600048EA0505DFF840814FEA920948F82950D1F8048008F48038B8F5803F0AD1DFF86B
:209580002C81D8F8008048EA0008DFF82091C9F8008009E0DFF81481D8F8008028EA00080C
:2095A000DFF80891C9F80080D1F8048008F40038B8F5003F10D1DFF8F48008F10408D8F88C
:2095C000008048EA0008DFF8E49000E05AE009F10409C9F800800DE0DFF8D08008F104080B
:2095E000D8F8008028EA0008DFF8C09009F10409C9F80080D1F8048008F48018B8F5801F65
:209600000ED1DFF8A88008F10808D8F8008048EA0008DFF8989009F10809C9F800800DE0A1
:20962000DFF8888008F10808D8F8008028EA0008DFF8789009F10809C9F80080D1F8048060
:2096400008F40018B8F5001F0ED1DFF8608008F10C08D8F8008048EA0008DFF8509009F14C
:209660000C09C9F800800DE0DFF8408008F10C08D8F8008028EA0008DFF8309009F10C09F3
:20968000C9F80080521C102AFFF48EAEBDE8F887000011100010024000080140000C014085
:2096A00000100140001401400800014000040140024693680B400BB1012000E00020704754
:2096C000C2684A40C26070470AB1016101E00B0403617047014800687047000050000020FD
:2096E00070B504460CB9012070BD4CF6CC402168086045F2555021680860D4E90010486067
:209700002168A0688860FFF7E5FF054606E0FFF7E1FF401B302801D90320E5E72068C068C3
:209720000028F4D14AF6AA20216808600020DBE701464AF6AA200A68106000207047000055
:2097400003480068034909780844014908607047500000205800002010B50848006840F03F
:20976000100006490860032000F0C2F8002000F007F800F02BF8002010BD000000200240E4
:2097800070B504460E4800784FF47A71B1FBF0F00C490968B1FBF0F5284600F075FE08B1F1
:2097A000012070BD102C07D200222146501E00F060F80548046001E00120F2E70020F0E784
:2097C00058000020000000205400002008B500BF1F48806940F001001D49886108468069FA
:2097E00000F00100009000BF00BF032000F080F8002211466FF00B0000F03BF80022114660
:209800006FF00A0000F035F8002211466FF0090000F02FF800221146501F00F02AF80022AE
:209820001146101F00F025F800221146901E00F020F800221146501E00F01BF800BF05496F
:20984000486820F0E06040F00070486000BF08BD001002400000014000BF00F01F020121B7
:2098600091404209920002F1E022C2F8001100BF70472DE9F05F80460D461646002707F00C
:209880004BFA074639462A46334601F00700C0F1070ABAF1040F02D94FF0040A01E0C0F19C
:2098A000070AD14600F1040ABAF1070F02D24FF0000A01E0A0F1030AD4464FF0010A0AFABC
:2098C00009FAAAF1010A0AEA020A0AFA0CFA4FF0010B0BFA0CFBABF1010B0BEA030B4AEA9F
:2098E0000B042146404607F01FFABDE8F09F000000BF00F00702064B19684FF6FF031940FE
:20990000044B0B4343EA0221014B196000BF70470CED00E00000FA0500BF00BF00BF00BF4B
:2099200000BFBFF34F8F00BF00BF00BF0948006800F4E06008490843001D0649086000BF7F
:2099400000BF00BFBFF34F8F00BF00BF00BF00BF00BFFDE70CED00E00000FA052DE9F04339
:2099600085B006463DA30FCB01AC0FC43FA0006800904FF00008002500270024A146012E88
:2099800030D0022E58D0102E61D139484468006800F0807000B301A8C4F38341475C04F418
:2099A000803070B132484068C0F340401DF8008004F4803040B12F48B0FBF8F000FB07F552
:2099C00002E02D4807FB00F52948406800F48000B0F5800F01D1A94603E068000321B0FB9D
:2099E000F1F935E02248046A04F44070B0F5807F05D104F0020010B14FF400491BE004F438
:209A00004070B0F5007F07D11948406A00F0020010B149F640490EE004F44070B0F5407F1A
:209A200007D11348006800F4003010B14FF2244901E04FF000090BE000F0A0F90C49496855
:209A4000C1F38131491C4900B0FBF1F900E000BF00BF484605B0BDE8F08300000203040596
:209A6000060708090A0B0C0D0E0F1010010200000010024000127A0000093D00F8B504463F
:209A800000260025207800F0010000286BD000274348C06900F0805070B900BF4048C0695B
:209AA00040F080503E49C8610846C06900F08050009000BF00BF01273A48006800F48070BB
:209AC000B0B93848006840F4807036490860FFF701FE064606E0FFF7FDFD801B642801D912
:209AE0000320F8BD2F48006800F480700028F2D02B48006A00F440752DB3A08800F44070AF
:209B0000A84220D02648006A20F44075012026490860002008602248056205F0010090B142
:209B2000FFF7D8FD064608E0FFF7D4FD801B41F28831884201D90320D3E71948006A00F09C
:209B400002000028F0D01648006A20F440706168084313490862012F04D10846C06920F029
:209B60008050C86100BF207800F00200022807D10B48406820F44040A168084308494860C5
:209B8000207800F01000102807D10548406820F48000E1680843024948600020A1E7000065
:209BA00000100240007000404004424270B504460D4600266248006800F00700A8420ED220
:209BC0005F48006820F0070028435D4908600846006800F00700A84201D0012070BD207898
:209BE00000F00200022807D15648406820F0F000A168084353494860207800F001000028E2
:209C00005DD06068012806D14E48006800F4003090B90120E2E76068022806D14948006838
:209C200000F0007040B90120D8E74648006800F0020008B90120D1E74248406820F0030024
:209C4000616808433F494860FFF744FD06466068012810D108E0FFF73DFD801B41F28831CC
:209C6000884201D90320B9E73648406800F00C000428F0D123E06068022810D108E0FFF7BA
:209C800029FD801B41F28831884201D90320A5E72C48406800F00C000828F0D10FE008E0E4
:209CA000FFF718FD801B41F28831884201D9032094E72448406800F00C000028F0D120486F
:209CC000006800F00700A8420ED91D48006820F0070028431A4908600846006800F007008D
:209CE000A84201D0012079E7207800F00400042807D11448406820F4E060E1680843114952
:209D00004860207800F00800082808D10D48406820F46050216940EAC1000A49486000F0E1
:209D20003DF808494968C1F30311074A515CC840064908600020FFF723FD00204EE70000DC
:209D40000020024000100240385901080000002001480068704700000000002000B5FFF762
:209D6000F7FF04494968C1F30221034A515CC84000BD0000001002404859010800B5FFF7B2
:209D8000E7FF04494968C1F3C221034A515CC84000BD00000010024048590108F0B585B0B3
:209DA0000FF26C0C9CE8E01001A8A0E8E0101CA52D68009500210022002300240020194D9A
:209DC000696801F00C05F5B1042D02D0082D19D101E0154819E001ADC1F38346AC5D01F488
:209DE000803555B10F4D6D68C5F340451DF805200D4D6543B5FBF2F302E00C4D04FB05F337
:209E0000184602E000BF084800BF00BF05B0F0BD02030405060708090A0B0C0D0E0F10107C
:209E2000010200000010024000127A0000093D00F8B504460025207800F00100002878D0E6
:209E4000F848406800F00C0004280CD0F548406800F00C00082811D1F248406800F480309D
:209E6000B0F5803F0AD1EF48006800F4003000285FD0606800285CD10120F8BD00BF60680F
:209E8000B0F5803F06D1E748006840F48030E549086028E0606858B9E248006820F480303F
:209EA000E04908600846006820F4802008601AE06068B0F5A02F0BD1DA48006840F48020CF
:209EC000D84908600846006840F4803008600AE0D448006820F48030D2490860084600688C
:209EE00020F48020086000BF606888B1FFF7F2FB054606E0FFF7EEFB401B642801D90320AF
:209F0000BBE7C848006800F400300028F2D010E0FFF7E0FB054606E0FFF7DCFB401B642873
:209F200001D90320A9E7BF48006800F400300028F2D1207800F00200022857D1B948406891
:209F400000F00C0050B1B748406800F00C00082818D1B448406800F4803098B9B14800684E
:209F600000F0020020B12069012801D0012084E7AC48006820F0F800616940EAC100A94904
:209F8000086033E02069E8B10120A7490860FFF7A1FB054606E0FFF79DFB401B022801D9FB
:209FA00003206AE79F48006800F002000028F2D09C48006820F0F800616940EAC100994917
:209FC000086013E0002098490860FFF783FB054606E0FFF77FFB401B022801D903204CE7F3
:209FE0009048006800F002000028F2D1207800F0080008282DD1A069B8B101208B490860B7
:20A00000FFF768FB054606E0FFF764FB401B022801D9032031E78348406A00F00200002838
:20A02000F2D0012007F0F2F913E000207F490860FFF750FB054606E0FFF74CFB401B0228E4
:20A0400001D9032019E77748406A00F002000028F2D1207800F00400042873D100267148E2
:20A06000C06900F0805070B900BF6E48C06940F080506C49C8610846C06900F0805000908B
:20A0800000BF00BF01266A48006800F48070B0B96748006840F4807065490860FFF71AFB58
:20A0A000054606E0FFF716FB401B642801D90320E3E65F48006800F480700028F2D000BF1F
:20A0C000E068012806D15748006A40F001005549086227E0E06858B95248006A20F0010081
:20A0E000504908620846006A20F00400086219E0E06805280BD14B48006A40F0040049491A
:20A1000008620846006A40F0010008620AE04548006A20F00100434908620846006A20F0D2
:20A120000400086200BFE068A0B1FFF7D3FA054609E0FFF7CFFA401B41F28831884202D9B7
:20A1400003209AE622E03748006A00F002000028EFD012E0FFF7BEFA054608E0FFF7BAFA1B
:20A16000401B41F28831884201D9032085E62D48006A00F002000028F0D1012E05D1294836
:20A18000C06920F080502749C86100BFE069C8B32448406800F00C00082860D0E0690228B7
:20A1A00048D1002020490866FFF794FA054606E0FFF790FA401B022801D903205DE6194834
:20A1C000006800F000700028F2D1206AB0F5803F07D11448406820F40030A1680843114910
:20A1E0004860D4E9080108430E49496821F4741108430C49486001200B490866FFF76AFA7F
:20A20000054607E02DE0FFF765FA401B022801D9032032E60348006800F000700028F2D013
:20A220001FE000000010024000004242800442420070004000200C490866FFF74BFA054628
:20A2400006E0FFF747FA401B022801D9032014E60648006800F000700028F2D101E0012062
:20A260000BE6002009E600000000424200100240042808D14FF0E021096941F004014FF0DC
:20A28000E022116107E04FF0E021096921F004014FF0E022116170470EB55F480078012826
:20A2A00000D10EBD5D48407E08B9022001E05B48407E02465948418801235948FAF792FC84
:20A2C0005848007830B9584A1188584A1088584A04F02CF8574858490978CDE90010574828
:20A2E0000278524800680290554803784D480078029903F0F7FD4F480078C0435149087085
:20A300004C488079C04388714A48B0F90200C04348804848B0F90400C04388804A4800785A
:20A3200038B94A4882784A480189414B494809F05BFD4948007828B9454881893C4A474880
:20A34000FCF7CAFE46494748F9F7FEFD464805F0B7FF46480088401C4449088008460088A3
:20A36000052801DB0020088041480088401C40490880084600880A2826DB0020088028488D
:20A38000407890B9264800783A490968C1EB80203849096801EBE01036490860084600682B
:20A3A000C0F387202049887204E000201E498872304908601C48807A0A2801DC002001E02C
:20A3C0001948807A184988722B480088401C2A49088008460088322804DB0020088027484F
:20A3E000FAF71AFD26480088401C2549088008460088642801DB0020088022480088401CD9
:20A400002049088008460088B0F57A7F01DB0020088000BF45E700005C00002020070020A5
:20A420000C030020C800002038060020EE03002044010020CE0000208D030020CA000020A9
:20A440008C030020D600002068030020520100204813002072110020C6030020C40300206B
:20A46000E60300205A130020400800205E000020600000206800002062000020680100204D
:20A48000640000206600002070B504462546681EB0F1807F01D301200FE0681E4FF0E02108
:20A4A00048610F214FF0FF3006F03EFC00204FF0E021886107200861002070BD10B5FFF744
:20A4C000EBFE10BD7047704710B50346002200BF93F83C00012801D1022010BD012083F81C
:20A4E0003C0000BF22F0FF00CC6840EA040222F440708C6840EA040222F480604C6840EA2E
:20A50000040222F400600C6840EA040222F480500C6940EA040222F400504C6940EA040245
:20A5200022F480408C6940EA040222F400408C6940EA04021868426400BF002083F83C00E9
:20A5400000BF00BFC9E7024600BF92F83C00012801D102207047012082F83C0000BF022074
:20A5600082F83D001068406820F0700013685860106840680B6818431368586010688068D0
:20A5800020F0800013689860106880684B68184313689860012082F83D0000BF002082F8A6
:20A5A0003C0000BF00BFD5E770B504460D4604222946206809F082F92068406C40F400402A
:20A5C000216848642068006840F0010021680860002070BD70B504460D460022294620680C
:20A5E00009F06CF900BF2068006A41F21111084050B92068006A8910084028B92068406CBE
:20A6000020F400402168486400BF00BF2068006A41F21111084050B92068006A89100840C8
:20A6200028B92068006820F001002168086000BF002070BD10B504460CB9012010BD94F8ED
:20A640003D0028B9002084F83C00204600F00CF8022084F83D00211D206809F0E7F8012010
:20A6600084F83D000020E9E710B586B0044632492068884233D100BF3048806940F4006067
:20A680002E4988610846806900F40060019000BF00BF8814029000200390049002A9284830
:20A6A000FEF778FE4FF46040029002200390059002A92348FEF76EFE4FF470600290022032
:20A6C0000390059002A91F48FEF764FE012211461920FFF7CEF81920FFF7BEF829E0206804
:20A6E000B0F1804F25D100BF1448C06940F001001249C8610846C06900F00100019000BF43
:20A7000000BF00BF0846806940F0040088610846806900F00400019000BF00BF012002907A
:20A720000020039004900220059002A90548FEF731FE06B010BD0000002C014000100240BD
:20A74000000C0140000801400146022081F83D000868006840F001000A681060012081F8BF
:20A760003D000020704701460868C06840F001000A68D0600868006840F001000A68106028
:20A78000002070472DE9F04104460D46002600BF94F83C00012802D10220BDE8F0810120FC
:20A7A00084F83C0000BF022084F83D002068866826F0770626F47F462068866028685028E9
:20A7C0003BD00CDC202860D004DC002853D0102865D155E030285DD0402860D141E0602879
:20A7E00035D070280DD0B0F5805F03D0B0F5005F55D115E02068806820F007002168886071
:20A800004EE0D5E902136A68206809F065F82068866826F0770646F07706206886603FE03E
:20A82000D5E902136A68206809F056F82068806840F480402168886032E0EA686968206812
:20A8400009F028F95021206809F052F828E0EA686968206809F033F96021206809F048F888
:20A860001EE0EA686968206809F014F94021206809F03EF814E00021206809F039F80FE05B
:20A880001021206809F034F80AE02021206809F02FF805E03021206809F02AF800E000BF8F
:20A8A00000BF012084F83D0000BF002084F83C0000BF00BF71E7704710B5044620680069DB
:20A8C000C0F34000D8B12068C068C0F34000B0B16FF002002168086101202077206880697C
:20A8E00000F0030018B12046FFF7E5FF05E0204600F0D6F8204600F0ABF90020207720681A
:20A900000069C0F38000D8B12068C068C0F38000B0B16FF004002168086102202077206838
:20A92000806900F4407018B12046FFF7C4FF05E0204600F0B5F8204600F08AF9002020772A
:20A9400020680069C0F3C000D8B12068C068C0F3C000B0B16FF00800216808610420207772
:20A960002068C06900F0030018B12046FFF7A3FF05E0204600F094F8204600F069F90020CD
:20A98000207720680069C0F30010D8B12068C068C0F30010B0B16FF0100021680861082086
:20A9A00020772068C06900F4407018B12046FFF782FF05E0204600F073F8204600F048F9C8
:20A9C000002020772068006900F0010058B12068C06800F0010030B16FF001002168086101
:20A9E000204600F095F920680069C0F3C01058B12068C068C0F3C01030B16FF0800021687A
:20AA000008612046FFF75EFD20680069C0F3801058B12068C068C0F3801030B16FF0400066
:20AA200021680861204600F055FA20680069C0F3401058B12068C068C0F3401030B16FF08F
:20AA40002000216808612046FFF73DFD10BD00001FB504460E492068884218D140200090E1
:20AA6000022001900320039069460A48FEF792FC00BF0949486820F4406040F0E06040F4D0
:20AA80004060486000BF0021044800F00BF81FBD0004004000100140000001400813002062
:20AAA0007047000030B504460D4601222946206808F0F6FE0A492068884201D1012000E0DF
:20AAC000002028B12068406C40F40040216848642068006840F0010021680860002030BD81
:20AAE000002C014070B504460D46164600BF94F83C00012801D1022070BD012084F83C0021
:20AB000000BF022084F83D0036B1042E1BD0082E31D00C2E5ED145E02946206808F0F2FEF3
:20AB20002068806940F00800216888612068806920F00400216888612068806929690843B5
:20AB40002168886147E02946206808F00DFF2068806940F40060216888612068806920F465
:20AB600080602168886120688069296940EA0120216888612FE02946206808F02DFF206811
:20AB8000C06940F008002168C8612068C06920F004002168C8612068C06929690843216814
:20ABA000C86118E02946206808F04CFF2068C06940F400602168C8612068C06920F480609E
:20ABC0002168C8612068C069296940EA01202168C86100E000BF00BF012084F83D0000BF8C
:20ABE000002084F83C0000BF00BF85E710B504460CB9012010BD94F83D0028B9002084F88B
:20AC00003C00204600F00CF8022084F83D00211D206808F00BFE012084F83D000020E9E732
:20AC200008B5094A016891420DD100BF0749C96941F00201054AD1611146C96901F0020177
:20AC4000009100BF00BF08BD00040040001002407047000030B504460D4601222946206837
:20AC600008F01EFE0A492068884201D1012000E0002028B12068406C40F400402168486472
:20AC80002068006840F0010021680860002030BD002C014030B504460D460022294620688D
:20ACA00008F0FEFD19492068884201D1012000E0002090B100BF2068006A41F2111108406B
:20ACC00050B92068006A8910084028B92068406C20F400402168486400BF00BF2068006A8A
:20ACE00041F21111084050B92068006A8910084028B92068006820F001002168086000BF49
:20AD0000012084F83D00002030BD0000002C014038B5044660480088401C5F49088008469E
:20AD20000088B0F5967F01DB002008805B4840785B4B0090DA79997958795A4B1B7800F05E
:20AD40002BFE59480078401C574908700846007805280ADB55480068806840F001005349AB
:20AD60000968886000205049087051480068401C4F49086000F02AFA4D48C08842F6FF7153
:20AD800088420CDA4A480089494989880844484908810846C088898808444549C880444A88
:20ADA000917A108905F038FF424948804249434804F00EFD42480078424909784840FF289E
:20ADC0001AD13F4880793F4989794840FF2813D13B4880883B498988484080B24FF6FF715C
:20ADE000884209D13648408836494988484080B24FF6FF7188420AD0FEF76CFC32490968BD
:20AE0000401AC82807D902203049087003E0FEF761FC2D4908602D480078012802D00228D0
:20AE200037D132E02648807901282DD128480078012804D1FBF7A8FD00202549087020487F
:20AE40000078012813D0022804D0032804D0042818D100E000BF00BF154B1A89154BB3F9EF
:20AE60000210174BB3F90200FBF746FF0BE0104B1A89104BB3F90210114BB3F90400FBF779
:20AE80003BFF00E000BF00BF04E001201049087000E000BF00BF38BDDC030020CA00002008
:20AEA000400700208C030020D40300206C130020BC100020380600204401002060020020B5
:20AEC000CE000020D6000020D803002030000020D5030020704770472DE9F04704462068BE
:20AEE00005682068C668206847694FF00008C14605F00F08B8F1000F0AD105F0200038B10C
:20AF000006F0200020B1204609F0E4F9BDE8F087B8F1000F6DD007F0010018B906F490703A
:20AF2000002866D005F0010030B106F4807018B1E06B40F00100E06305F0040030B107F099
:20AF4000010018B1E06B40F00200E06305F0020030B107F0010018B1E06B40F00400E0630C
:20AF600005F0080030B107F0010018B1E06B40F00800E063E06B68B305F0200028B106F022
:20AF8000200010B1204609F0A5F920684069C0F38019E06B00F0080010B9B9F1000F22D09F
:20AFA000204609F028F92068406900F04000B0B12068406920F0400021684861606B50B1D0
:20AFC0001748616B4863606BFDF7F2FE10B1606B416B88470CE02046FFF77DFF08E02046D3
:20AFE000FFF779FF04E02046FFF775FF0020E0638CE705F0800030B106F0800018B120465E
:20B0000009F0AEFA82E705F0400030B106F0400018B1204609F0FFF878E700BF76E7000040
:20B02000A540010810B504460CB9012010BDA06900B100E000BF94F8390028B9002084F8C5
:20B040003800204600F028F8242084F839002068C06820F400502168C860204609F09CF990
:20B060002068006920F49040216808612068406920F02A00216848612068C06840F4005038
:20B080002168C8600020E063202084F8390084F83A000020CAE7000010B586B004462B4967
:20B0A000206888424FD100BF2948C06940F480202749C8610846C06900F48020019000BFFD
:20B0C00000BF0815029002200390012004900320059002A91F48FEF75DF94FF4006002904E
:20B0E000002003900120049002A91A48FEF752F900BF1949486820F0300040F0E06040F0EA
:20B100001000486000BF012211462720FEF7B1FB2720FEF7A1FB11480068C06840F4807071
:20B120000E490968C8600D480068406940F001000A490968486109480068C06840F02000EA
:20B1400006490968C86006B010BD000000480040001002400010014000000140C01A00201E
:20B160007047704710B500F011F9054931F8100041F255510844034908810020086010BDCC
:20B180000C7B0108BC10002000B585B000BF0D48806940F010000B4988610846806900F0A8
:20B1A0001000009000BF00BF4FF460700190002002900120039001A90348FEF7EBF805B0E5
:20B1C00000BD00000010024000100140F8B500F0DDF8064600F0DAF8044600F0D7F805463B
:20B1E000A64203D1AC4201D15E4805705E48007830B95C4800785B49487001205A490870FD
:20B200005848007857494978884210D0FEF762FA564908605648007828B155480078401C53
:20B220005349087017E001205249887213E0FEF751FA4E490968401AC8280CD900204D492D
:20B2400088724B4908704B498881C8814A4908700120484908744748807A10B900204749C7
:20B260000870404800783F494978454A515C884245D14048006840B13E48006842F6AA211F
:20B28000B1FBF0F03B49888002E00120394988803A480078401C39490870084600780228C9
:20B2A0000DDD3448006844F63E11B1FBF0F03149888100203049087001202E4908742F488C
:20B2C00000780F280CDA274800782E4931F8100041F255510844274908810020888009E013
:20B2E0000F20264908701F480078264931F810002049088100201F490860C88026E0194820
:20B300004078184909781E4A515C88421ED100201A4908701749888012480078194931F805
:20B32000100041F255510844124908814FF6FF70086011480078401CC0B20F49087005283C
:20B3400004DD0620087000200A490874054800680D49009003F0A0FB024800780149487092
:20B36000F8BD0000F0020020F2020020F4020020F3020020BC100020F8020020F9020020A6
:20B38000FC7A01080C7B01084401002010B51E48C07AA8B94FF400711C48FEF789F904469A
:20B3A0004FF480711948FEF783F944EA4000C4B280211648FEF77CF944EA8000C4B220E016
:20B3C0004FF400711148FEF773F908B9012000E0002004464FF480710C48FEF769F908B933
:20B3E000012000E0002044EA4000C4B280210748FEF75EF908B9012000E0002044EA80007C
:20B40000C4B204F0070010BDBC1000200010014007E0044804F019F9002005F0EDFEFBF786
:20B4200005F8F6E7FC00002070B50446204609F042FEA1890122A068FEF746F90120FAF76D
:20B44000D0FFA1882068FEF733F90546A1890022A068FEF739F90120FAF7C3FF012D01D1B1
:20B46000012070BD0020FCE71FB50446A06809F09FFD206809F09CFDA08900900120039039
:20B48000112001906946A068FDF784FFA0880090012003901120019069462068FDF77AFFEA
:20B4A0001FBD2DE9F04704460F464FF000084FF08009204609F0FFFD00251CE0A1890122EC
:20B4C000A068FEF701F93220FAF78BFFA1882068FEF7EEF80646012E03D149FA05F040EA6B
:20B4E0000808A1890022A068FEF7EEF83220FAF778FF681CC5B2082DE0DB87F80080012048
:20B50000FAF76FFFBDE8F08710B50446204609F0DAFDA18801222068FEF7D6F80120FAF7C2
:20B5200060FFA1890122A068FEF7CEF83220FAF758FFA1890022A068FEF7C6F8A1880022B0
:20B540002068FEF7C1F80120FAF74BFF10BD10B50446204609F0B7FDA1890122A068FEF720
:20B56000B3F8A18801222068FEF7AEF83220FAF738FFA18800222068FEF7A6F83220FAF78E
:20B5800030FFA1890022A068FEF79EF810BD10B50446204609F097FDA18800222068FEF706
:20B5A00093F8A1890122A068FEF78EF83220FAF718FFA18801222068FEF786F83220FAF74C
:20B5C00010FFA18800222068FEF77EF8A1890022A068FEF779F810BD2DE9F04104460D46B3
:20B5E000A8468026204609F06EFD002736E006EA0800C0B1A18801222068FEF765F83220CF
:20B60000FAF7EFFEA1890122A068FEF75DF83220FAF7E7FEA1890022A068FEF755F831209E
:20B62000FAF7DFFE17E0A18800222068FEF74CF83220FAF7D6FEA1890122A068FEF744F89C
:20B640003220FAF7CEFEA1890022A068FEF73CF83120FAF7C6FE7610781CC7B2082FC6DBED
:20B66000A18801222068FEF72FF80120FAF7B9FEBDE8F08101480249086070470030000810
:20B6800008ED00E0012023490978052910D12149103109789B290BD11E4914310978522944
:20B6A00006D11C4918310978052901D1032030E018490978042910D1164910310978C32954
:20B6C0000BD1144914310978B42906D11149183109780B2901D102201BE00E49097881B95E
:20B6E0000C491031097810290BD10A4914310978042906D10749183109780A2901D10120C1
:20B7000007E005490968054A914201D1042000E000207047D0FF0FE0002004E010040313C8
:20B7200000B585B000BF2B48806940F01000294988610846806900F01000009000BF00BF24
:20B74000254826490860401488800846808801900020029001200390086801A9FDF71AFED6
:20B7600000201E4988714872C860C87108721A481B4908604FF48040888008468088019094
:20B780000020029001200390086801A9FDF702FE0020134988714872C860C87108720E48D5
:20B7A000104908604FF4004088800846808801900020029001200390086801A9FDF7EAFDFB
:20B7C0000020084988714872C860C871087205B000BD00000010024000100140E81100203C
:20B7E000FC110020101200202DE9F04104460F4616469846069DB8F1000F04D10121204602
:20B8000009F03AFC03E00221204609F035FCE07900F0010020B101206072FDF75BFFE060C7
:20B82000607A01281BD1207A50B9FDF753FFE060FDF750FF206100206072012028700EE093
:20B84000FDF748FFE168401AB84208D9FDF742FFE060002060722870FDF73CFF20612878E0
:20B8600068B966B1FDF736FF2169401AB04206D9FDF730FF20610020607201202870BDE8BE
:20B88000F0812DE9F04105460E4617469846B8F1F10F13D100240EE0BC4201D1012300E0A3
:20B8A00000231A4605EBC403998855F83400FDF70BFF601CC4B2B442EEDB0DE0002409E003
:20B8C00005EBC402918855F834000022FDF7FCFE601CC4B2B442F3DBBDE8F08110B586B041
:20B8E00000BF2A48806940F00400284988610846806900F00400019000BF00BF00BF084659
:20B90000806940F0080088610846806900F00800019000BF00BF002433E01D4A02EBC4028E
:20B9200091881B4A52F834000022FDF7CDFE184800EBC40080880290012003900220059016
:20B94000134951F8340002A9FDF724FD114A02EBC40291880F4A52F834000022FDF7B4FE88
:20B960000C4800EBC400808802900120039002200590084951F8340002A9FDF70BFD601CCE
:20B98000C4B2032CC9DB06B010BD00000010024090030020A80300202DE9F04707468946A2
:20B9A00092461C46DDF82080B9F1060F06D0B9F10C0F05D0B9F1FF0F06D103E0002505E02D
:20B9C000012503E0022501E0002500BF00BFBAF1060F06D0BAF10C0F05D0BAF1FF0F06D1F2
:20B9E00003E0002605E0012603E0022601E0022600BF00BF43462A4603217548FFF741FF90
:20BA0000072F43D2DFE807F04204436F7AA6AD004CB9F123324603216E48FFF732FF0020A6
:20BA20006D49088031E0B8F1F10F22D16B48408969490988884206DDF12332460321654852
:20BA4000FFF71FFF0FE06548808963490988884206DDF023324603215E48FFF712FF02E005
:20BA600000205D4908805C480088401C5A4908800BE0B8F1F00F08D1F0233246032155480D
:20BA8000FFF7FFFE0020544908809DE000BF04BB51480088B0F5167F06DAF1233246032188
:20BAA0004C48FFF7EEFE0EE04B480088B0F5966F06DAF023324603214648FFF7E2FE02E088
:20BAC00000204549088044480088401C4249088008E04346324603213E48FFF7D2FE002034
:20BAE0003D49088070E00CB9F12000E0F0200346324603213748FFF7C4FE65E004BB364884
:20BB00000088B0F5167F06DAF123324603213148FFF7B7FE0EE030480088B0F5966F06DA37
:20BB2000F023324603212B48FFF7ABFE02E000202949088028480088401C2749088008E014
:20BB4000F023324603212348FFF79BFE00202249088039E0F123324603211E48FFF791FE75
:20BB600032E01F4800881D490989884222DB1B48408919490988884206DDF1233246032189
:20BB80001448FFF77EFE0FE01448808912490988884206DDF023324603210E48FFF771FE80
:20BBA00002E000200C4908800B480088401C0A49088008E0002008490880F0233246032104
:20BBC0000448FFF75EFE00BF00BFBDE8F087000090030020A8030020C00300204007002065
:20BBE0003C0300202DE9FF4F89B08146FA4903C9CDE907010025AA460020049003901898A9
:20BC0000AA2823D1BDF85A0032281FDD0020F3490870BDF85A001E2801DA01200870BDF8A7
:20BC20005A00EF49498D4843C0F3CF20EB49488008464088BDF83010884203DABDF83000DC
:20BC4000E64948800120E749087067E0BDF85800E2494880E4480088B0F5C87F01DA6420DE
:20BC600002E0E148008880100590DC4841880598814204DBFDF72EFDDC4908600BE04FF406
:20BC8000FA6BFDF727FDD9490968401A584502D90120D2490870D64800883C2814DDD248F9
:20BCA0000088C82801DA96200CE0CF480088B0F52F7F02DD40F20D2004E0CB48008800EBF5
:20BCC00040008010069010E0C7480088C82801DA962009E0C4480088B0F52F7F02DD40F215
:20BCE0000D2001E0C04800880690BC4841880698814202DB0020B94908709DF82900012884
:20BD000002D09DF82A0010B90120B4490870BDF83000B24948800020B2490870AF48007889
:20BD200001281BD1AD48B0F9060007280CDC0020AA49C880AF4803F088FC0120AE490870DA
:20BD40000020AE490880F3E3A448C088C01F00B2A249C880A74803F06BFCF4E7A1480078F1
:20BD6000012837D19D48408804B203254FF0070A9B48408DA04202DA9948408D00E0204655
:20BD800004B29748C08D9E49097A48434FF47A714843401400EBC00101EB00104FF6FF7162
:20BDA00001EA80060123052296480188304602F0A3FA944908808A48408D40429249086191
:20BDC000002048618648408D8002404288610020C861F0E3179813287ED004DC112807D0CE
:20BDE00012287AD1EFE0142878D03328F9D1C7E38348C07B5A2804DC7948007A401EC5B224
:20BE00000AE07F48C07B6E2804DB7548007A401CC5B201E07248057A002D01DC012000E092
:20BE2000284605466E4890F809A09DF8280032282EDADFF8A8C1BCF80230DFF8A4C1BCF82D
:20BE40000220BCF80010BCF800C04FEA6C00F9F789F8624949884843800A04B26448B0F9D6
:20BE6000020040F22221884202DA5D48C0880DE05F48B0F9020000EB800080005B2190FB87
:20BE8000F1F0C4EB0411C90091FBF0F004B258E09DF82800322851DB9DF828005A284DDA31
:20BEA000DFF838C1BCF80230DFF834C1BCF80220BCF80010BCF800C04FEA6C00F9F752F813
:20BEC000464949884843800A04B24948B0F9020040F22221884202E076E1F3E35AE202DA95
:20BEE0003F48C08828E04248B0F9020040F2D73188420DDA3E48B0F9020000EB800080002F
:20BF00005B2190FBF1F1D820604390FBF1F013E09DF82800604300EB4000C0000A2190FB3D
:20BF2000F1F03349B1F9021001EB810189005B2291FBF2F190FBF1F004B202E02848C08849
:20BF400004B22F48807B6043642190FBF1F004B223488088A04202DD2148808800E0204684
:20BF600004B21F48C088A04202DA1D48C08800E0204604B21A4840892149097A48434FF40F
:20BF80007A714843401400EBC00101EB00104FF6FF7101EA8006012305221A48018830465D
:20BFA00002F0AAF9174908800D48C088404216490861002048610A48C088800240428861CD
:20BFC0000020C861B8E30E48407C5A281EDC0448007D401EC5B224E0505F0108E000002095
:20BFE0005408002018010020520100201001002038060020FC0000201A0100201C010020F6
:20C000002007002016010020C4050020FE48407C6E2804DBFD48007D401CC5B201E0FB4889
:20C02000057D002D01DC012000E028460546F74890F815A09DF8280032282EDADFF8D0C3B5
:20C04000BCF80230DFF8C4C3BCF80E20BCF80C10BCF80CC04FEA6C00F8F784FFEC4949884D
:20C060004843800A04B2EB48B0F9020040F22221884202DAE548408A0DE0E648B0F902003F
:20C0800000EB800080005B2190FBF1F0C4EB0411C90091FBF0F004B254E09DF828003228D3
:20C0A0004DDB9DF828005A2849DADFF864C3BCF80230DFF858C3BCF80E20BCF80C10BCF8BA
:20C0C0000CC04FEA6C00F8F74DFFD14949884843800A04B2CF48B0F9020040F222218842FD
:20C0E00002DACA48408A28E0CA48B0F9020040F2D73188420DDAC748B0F9020000EB8000B3
:20C1000080005B2190FBF1F1D820604390FBF1F013E09DF82800604300EB4000C0000A2146
:20C1200090FBF1F0BB49B1F9021001EB810189005B2291FBF2F190FBF1F004B202E0B348F1
:20C14000408A04B2B048007C6043642190FBF1F004B2AE48008AA04202DDAC48008A00E002
:20C16000204604B2A948408AA04202DAA748408A00E0204604B2A548C08AA349097A484344
:20C180004FF47A714843401400EBC00101EB00104FF6FF7101EA8006012305229E4801880A
:20C1A000304602F0A9F89C4908809848408A40429A490861002048619448408A800240421E
:20C1C00088610020C861B7E28F48C07C5A2805DC8E4890F82000401EC5B20CE08A48C07CD1
:20C1E0006E2805DB894890F82000401CC5B202E0864890F82050002D01DC012000E028465C
:20C200000546824890F821A09DF8280032282EDADFF8FCC1BCF80230DFF8F0C1BCF81A20B1
:20C22000BCF81810BCF818C04FEA6C00F8F79AFE774949884843800A04B27648B0F90200A5
:20C2400040F22221884202DA7048C08B0DE07148B0F9020000EB800080005B2190FBF1F09C
:20C26000C4EB0411C90091FBF0F004B254E09DF8280032284DDB9DF828005A2849DADFF863
:20C2800090C1BCF80230DFF884C1BCF81A20BCF81810BCF818C04FEA6C00F8F763FE5C495B
:20C2A00049884843800A04B25A48B0F9020040F22221884202DA5548C08B28E05548B0F944
:20C2C000020040F2D73188420DDA5248B0F9020000EB800080005B2190FBF1F1D8206043BD
:20C2E00090FBF1F013E09DF82800604300EB4000C0000A2190FBF1F04649B1F9021001EBC6
:20C30000810189005B2291FBF2F190FBF1F004B202E03E48C08B04B23B48807C60436421F4
:20C3200090FBF1F004B23948808BA04202DD3748808B00E0204604B23448C08BA04202DA83
:20C340003248C08B00E0204604B23048408C2E49097A48434FF47A7148434014304909784C
:20C36000484386B2012305222B480188304601F0C3FF294908802548C08B4042274908617D
:20C38000002048612148C08B8002404288610020C861D1E11C48407D5A2805DC1B4890F8C9
:20C3A0002C00401EC5B20CE01748407D6E2805DB164890F82C00401CC5B202E0134890F854
:20C3C0002C50002D01DC012000E0284605460F4890F82DA09DF8280032283DDADFF830C07C
:20C3E000BCF80230DFF824C0BCF82620BCF82410BCF824C04FEA6C00F8F7B4FD04494988BF
:20C400004843800A04B20DE02007002054080020E00000203806002016010020C405002023
:20C42000DE000020FE48B0F9020040F22221884202DAFC48408D0DE0F948B0F9020000EB1D
:20C44000800080005B2190FBF1F0C4EB0411C90091FBF0F004B254E09DF8280032284DDBD2
:20C460009DF828005A2849DADFF8BCC3BCF80230DFF8B0C3BCF82620BCF82410BCF824C05A
:20C480004FEA6C00F8F76EFDE74949884843800A04B2E348B0F9020040F22221884202DAE0
:20C4A000E048408D28E0DE48B0F9020040F2D73188420DDADA48B0F9020000EB800080000B
:20C4C0005B2190FBF1F1D820604390FBF1F013E09DF82800604300EB4000C0000A2190FB78
:20C4E000F1F0CF49B1F9021001EB810189005B2291FBF2F190FBF1F004B202E0C948408DC2
:20C5000004B2CA48007D6043642190FBF1F004B2C448008DA04202DDC248008D00E0204655
:20C5200004B2C048408DA04203DABE48408D01E000E2204604B2BB48C08DBC49097A48439C
:20C540004FF47A7148434014B9490978484386B201230522B7480188304601F0CDFEB54985
:20C560000880B048408D4042B349086100204861AC48408D8002404288610020C861DBE00C
:20C58000AA48C07D5A2805DCA64890F84400401EC5B20CE0A548C07D6E2805DBA14890F87D
:20C5A0004400401CC5B202E09E4890F84450002D02DC012001E0C0E028460546994890F8B1
:20C5C00045A09DF82800322822DA9748408840439449C98FB0FBF1F004B29148B0F902003E
:20C5E00040F22221884203DA8E48B0F842000DE08B48B0F9020000EB800080005B2190FB02
:20C60000F1F0C4EB0411C90091FBF0F004B249E09DF82800322841DB9DF828005A283DDAD8
:20C620008148408840437F49C98FB0FBF1F004B27B48B0F9020040F22221884203DA794839
:20C64000B0F8420028E07648B0F9020040F2D73188420DDA7248B0F9020000EB8000800044
:20C660005B2190FBF1F1D820604390FBF1F013E09DF82800604300EB4000C0000A2190FBD6
:20C68000F1F06749B1F9021001EB810189005B2291FBF2F190FBF1F004B203E06148B0F814
:20C6A000420004B26148807D6043642190FBF1F004B25C48B0F84000A04204DD5948B0F8FA
:20C6C000400001E034E0204604B25648B0F84200A04203DA5348B0F8420000E0204604B241
:20C6E0005048B0F846005149097A48434FF47A71484340144E490978484386B201230522D9
:20C700004C480188304601F0F7FD4A4908804548B0F8420040424849086100204861414841
:20C72000B0F842008002404288610020C86103E00025AA46002400BF00BF404800883B49AB
:20C740000090097901EB81014A003849097901EB8101480034230021FAF71CFC6043800AA8
:20C7600004B231488480B0F90400002802DC00202D498880314800882C49097901EB8101CF
:20C78000B0EB410F20DD2848B0F904002649B1F90610401A022806DD2348C088401C00B23D
:20C7A0002149C880A3E02048B0F904001E49B1F90610401AB0F1FF3F05DA1B48C0880A3803
:20C7C00000B21949C88092E000BF1D48007801286CD116484078032805D100201949088068
:20C7E0001749087083E011484078012805D14FF4967004901E20039003E0642004900A201B
:20C80000039010480088401C0E490880084601880498814244DC0448B0F90400024913E0DD
:20C820003806002054080020E000002020070020DE00002016010020C40500203C0300205A
:20C840001A0100201C010020B1F90610401A022814DD64480188039891FBF0F0C0F10A0034
:20C860006049098891FBF0F200FB121068BB5E48C088284400B25C49C88038E05A48B0F974
:20C8800004005949B1F90610401AB0F1FF3F2EDA5548C088A0EB0A0000B25349C88026E0DB
:20C8A0000020504908805149087020E04E48B0F904004D49B1F90610401A022806DD4A4893
:20C8C000C088284400B24849C88010E04648B0F904004549B1F90610401AB0F1FF3F06DA87
:20C8E0004148C088A0EB0A0000B23F49C8803E48B0F90600062801DA062002E03A48B0F9DF
:20C9000006003949C8803A4800883A49097901EB8101162202EB4101884208DD0120324918
:20C9200008700020C880344802F08FFE02E0324802F07EFE314A117B314AD088314A128863
:20C9400001F080FB80462F48A0F8008001231A462D480188404601F0CFFC2B490880254AE7
:20C96000517A274A907D01F05BFB029001231A4626480188029801F0BFFC24490880244873
:20C980000088642190FBF1F000B201901C480089C111204A019804F0E9FA1F4908801248F8
:20C9A000B0F90600184909884843871217480088784387121848B0F900003844471038B2B1
:20C9C000ADF81E0001208DF8220003208DF81C000798C9F800000898C9F804000DB0BDE8E1
:20C9E000F08F00001C010020E00000201A0100203C03002020070020FC00002060070020F7
:20CA0000380600201E010020200100202201002016010020C4050020140100202DE9FF4F3C
:20CA200085B081468A469346FE4903C9CDE90301002500200290DA4501DA584600E050469F
:20CA4000F949488008464088B0F5006F02DD4FF4006001E0F4484088F3494880089801286E
:20CA600006D0022852D0032873D0042872D1E7E0EE48C07B502801DC022506E0EB48C07BAF
:20CA8000782801DB042500E00325002D01DC012000E02846054607200290E3484088E4494C
:20CAA000C9884843C00A04B2E148C088A04202DADF48C08800E0204604B2DD484089DB496E
:20CAC000097A48434FF47A714843401400EBC00101EB00104FF6FF7101EA80060123052222
:20CAE000D4480188304601F007FCD2490880D048C0884042D049086100204861CC48C088FB
:20CB00008002404288610020C861E8E0C748407C502801DC022506E0C448407C782801DBA6
:20CB2000042500E00325002D01DC012000E02846054607200290BC484088BD49498A484317
:20CB4000C00A04B2BA48408AA04204DAB848408A02E02BE0BEE0204604B2B548C08AB34915
:20CB6000097A48434FF47A714843401400EBC00101EB00104FF6FF7101EA80060123052281
:20CB8000AC480188304601F0B7FBAA490880A848408A4042A849086100204861A448408A6F
:20CBA0008002404288610020C86198E09F48C07C502801DC022506E09C48C07C782801DBA6
:20CBC000042500E00325002D01DC012000E02846054607200290944840889549C98B484346
:20CBE000C00A04B29248C08BA04202DA9048C08B00E0204604B28E48408C8C49097A48432E
:20CC00004FF47A71484340148C490978484386B20123052287480188304601F06DFB8549AE
:20CC200008808348C08B404283490861002048617F48C08B8002404288610020C8614EE060
:20CC40007A48407D502801DC022506E07748407D782801DB042500E00325002D01DC01209F
:20CC600000E028460546072002906F4840887049498D4843C00A04B26D48408DA04202DA09
:20CC80006B48408D00E0204604B26948C08D6749097A48434FF47A7148434014674909781E
:20CCA000484386B20123052262480188304601F023FB604908805E48408D40425E49086178
:20CCC000002048615A48408D8002404288610020C86104E0002500200290002400BF00BF89
:20CCE0005748008851490090097901EB81014A004E49097901EB8101480034230021FAF771
:20CD000049F96043800A04B247488480B0F90400002802DC0020444988804948008843494E
:20CD2000097901EB8101B0EB410F20DD3E48B0F904003D49B1F90610401A022806DD3A48B9
:20CD4000C088401C00B23849C88032E03648B0F904003549B1F90610401AB0F1FF3F28DAFE
:20CD60003148C0880A3800B22F49C88021E000BF2D48B0F904002C49B1F90610401A0228A3
:20CD800006DD2948C088284400B22749C88010E02548B0F904002449B1F90610401AB0F1EF
:20CDA000FF3F06DA2048C1880298081A00B21E49C8801D48B0F90600062801DA062002E062
:20CDC0001948B0F906001849C8801D4800881749097901EB8101162202EB4101884208DD47
:20CDE0000120114908700020C880164802F02DFC02E0144802F01CFC134A117B134AD08879
:20CE0000134A128801F01EF980461148A0F8008001231A460F480188404601F06DFA0D4944
:20CE2000088019E0405F0108E0000020200700205408002000010020C4050020DE000020FE
:20CE40003C030020FC00002060070020380600200401002006010020204A517A204A907D7A
:20CE600001F0DEF8019001231A461E480188019801F042FA1B4908801B480088642190FB3A
:20CE8000F1F000B2009016480089C111174A009804F06CF8164908801648B0F90600164912
:20CEA0000988484387120F480088784387121048B0F900003844471038B2ADF80E000120F8
:20CEC0008DF8120004208DF80C000398C9F800000498C9F8040009B0BDE8F08F2007002025
:20CEE000380600200801002000010020C4050020FE000020E0000020060100202DE9FF4FF8
:20CF00008BB08246FE4903C9CDE909010025AB460020069005901A98AA2834D1BDF862003A
:20CF2000322830DDF748008864282CDDF5480088FA2808DBF3480088B0F5827F23DABDF849
:20CF40006000C8281FDA0020EF490870BDF862001E2801DA01200870BDF86200EB49C98E45
:20CF60004843C0F3CF20E849488008464088BDF83810884203DABDF83800E34948800120CF
:20CF8000E34908707BE0BDF86000DF494880E1480088C82801DA642002E0DE4800884010AD
:20CFA0000790D94841880798814204DBFCF792FBD949086020E0D348B0F90200C82807DD0B
:20CFC000D048B0F90200D54991FBF0F087B201E04FF49667B7F5FA7F02DA4FF4FA7000E01C
:20CFE00038460746FCF776FBCB490968401AB84202D90120C4490870C24800883C2814DDC1
:20D00000C4480088C82801DA96200CE0C1480088B0F52F7F02DD40F20D2004E0BD4800887C
:20D0200000EB40008010089010E0BA480088C82801DA962009E0B7480088B0F52F7F02DD00
:20D0400040F20D2001E0B34800880890AE4841880898814202DB0020AB4908709DF8310024
:20D06000012802D09DF8320010B90120A6490870BDF83800A44948800020A5490870A2488B
:20D08000007801281BD1A048B0F9060007280CDC00209D49C880A24802F0D7FA0120A1494F
:20D0A00008700020A0490880FEE39748C088C01F00B29549C8809A4802F0BAFAF4E7944869
:20D0C000007801283DD19048408804B297480088E62801DA032500E001254FF0070B8B48A9
:20D0E000C08EA04202DA8948C08E00E0204604B28648408F8E49097A48434FF47A714843CE
:20D10000401400EBC00101EB00104FF6FF7101EA80060123052287480188304601F0ECF8FF
:20D12000844908807948C08E404283490861002048617648C08E8002404288610020C861C9
:20D1400092E37048B0F90200B0F5FA7F23DD7B4800780F281FDB6C484088C8281BDD694858
:20D16000B0F90200642148437449097890FBF1F073490860734800680968C0EB01307149FC
:20D18000096801EBA0206F49086008460068C0F30F306D490880199804287DD006DC012837
:20D1A0000BD0022879D0032878D11AE1052876D0332875D04428F7D1E3E25D48C07B5A2844
:20D1C00004DC5248007A401EC5B20AE05848C07B6E2804DB4D48007A401CC5B201E04B48F6
:20D1E000057A002D01DC012000E028460546474890F809B0DFF810C1BCF802308446BCF810
:20D200000220BCF80010BCF800C04FEA6C00F7F7A9FE3D4949884843800A04B24448807BD1
:20D220006043642190FBF1F004B238488088A04202DD3648808800E0204604B23348C08816
:20D24000A04202DA3148C08800E0204604B22F4840893749097A48434FF47A714843401478
:20D2600000EBC00101EB00104FF6FF7101EA8006012305222F480188304601F03DF82D4983
:20D2800008802248C08840422B490861002048611E48C088800204E015E107E0DFE284E115
:20D2A000F5E1404288610020C861DCE22048407C5A2804DC1548007D401EC5B20AE01C48A3
:20D2C000407C6E2804DB1148007D401CC5B201E00E48057D002D01DC012000E028460546F7
:20D2E0000A4890F815B0DFF820C0BCF802308446BCF80E20BCF80C10BCF80CC026E00000F0
:20D30000585F010838060020E0000020540800202C010020520100202401002020550300F6
:20D32000FC0000202E010020300100203C030020200700202A010020C40500200C03002028
:20D34000380100203C010020960100204FEA6C00F7F708FEFE4949884843800A04B2FD489F
:20D36000007C6043642190FBF1F004B2FA48008AA04202DDF848008A00E0204604B2F64856
:20D38000408AA04202DAF448408A00E0204604B2F148C08AEF49097A48434FF47A71484381
:20D3A000401400EBC00101EB00104FF6FF7101EA800601230522E9480188304600F09CFF45
:20D3C000E6490880E448408A4042E549086100204861E148408A8002404288610020C86195
:20D3E00041E2DC48C07C5A2805DCDB4890F82000401EC5B20CE0D748C07C6E2805DBD648CC
:20D4000090F82000401CC5B202E0D34890F82050002D01DC012000E028460546CE4890F83A
:20D4200021B0DFF82CC3BCF802308446BCF81A20BCF81810BCF818C04FEA6C00F7F792FD2D
:20D44000C34949884843800A04B2C248807C6043642190FBF1F004B2BF48808BA04202DD01
:20D46000BD48808B00E0204604B2BB48C08BA04202DAB948C08B00E0204604B2B648408C82
:20D48000B449097A48434FF47A7148434014B5490978484386B201230522B04801883046F0
:20D4A00000F02AFFAD490880AB48C08B4042AC49086100204861A848C08B800240428861C6
:20D4C0000020C861CFE1A348407D5A2805DCA24890F82C00401EC5B20CE09E48407D6E28B0
:20D4E00005DB9D4890F82C00401CC5B202E09A4890F82C50002D01DC012000E02846054654
:20D50000954890F82DB0DFF848C2BCF802308446BCF82620BCF82410BCF824C04FEA6C0019
:20D52000F7F720FD8A4949884843800A04B28948007D6043642190FBF1F004B28648008D7E
:20D54000A04202DD8448008D00E0204604B28248408DA04202DA8048408D00E0204604B2CF
:20D560007D48C08D7B49097A48434FF47A71484340147C490978484386B2012305227748A7
:20D580000188304600F0B8FE744908807248408D404273490861002048616F48408D8002A4
:20D5A000404288610020C8615DE16A48407D5A2805DC694890F83800401EC5B20CE06548C8
:20D5C000407D6E2805DB644890F83800401CC5B202E0614890F83850002D01DC012000E033
:20D5E000284605465C4890F839B0DFF864C1BCF802308446BCF83220BCF83010BCF830C013
:20D600004FEA6C00F7F7AEFC514949884843800A04B25048007D6043642190FBF1F004B238
:20D620004D48808EA04202DD4B48808E00E0204604B24948C08EA04202DA4748C08E00E08F
:20D64000204604B24448408F4249097A48434FF47A714843401443490978484386B20123B9
:20D6600005223E480188304600F046FE3B4908803948C08E40423A4908610020486136483A
:20D68000C08E8002404288610020C861EBE03148C07D5A2805DC304890F84400401EC5B209
:20D6A0000CE02C48C07D6E2805DB2B4890F84400401CC5B202E0284890F84450002D01DCCD
:20D6C000012000E028460546234890F845B02048408840432049C98FB0FBF1F004B21D488D
:20D6E000807D6043642190FBF1F004B21A48B0F84000A04203DD1848B0F8400000E0204649
:20D7000004B21548B0F84200A04203DA1248B0F8420000E0204604B20F48B0F846000D4972
:20D72000097A48434FF47A71484340140D490978484386B20123052208480188304600F0AA
:20D74000DBFD064908800448B0F8420040420BE0E000002020070020540800202A01002069
:20D76000C4050020DE000020F049086100204861EF48B0F842008002404288610020C86100
:20D7800071E0EC48C07D5A2805DCE94890F85000401EC5B20CE0E748C07D6E2805DBE4488C
:20D7A00090F85000401CC5B202E0E14890F85050002D01DC012000E028460546DC4890F81B
:20D7C00051B0DD4840884043D949B1F84A10B0FBF1F004B2D748807D6043642190FBF1F0C1
:20D7E00004B2D348B0F84C00A04203DDD048B0F84C0000E0204604B2CD48B0F84E00A042AD
:20D8000003DACB48B0F84E0000E0204604B2C848B0F85200C749097A48434FF47A71484345
:20D820004014C6490978484386B201230522C4480188304600F060FDC1490880BC48B0F860
:20D840004E004042B949086100204861B848B0F84E008002404288610020C86103E0002590
:20D86000AB46002400BF00BFB64800880090B148007900EB80004200342300210846F9F72A
:20D8800089FB6043800A04B2AB488480B0F90400002802DC0020A8498880AA480088A549F6
:20D8A000097901EB810100E0C4E0B0EB410F20DDA148B0F90400A049B1F90610401A022849
:20D8C00006DD9D48C088401C00B29B49C8808EE09948B0F904009849B1F90610401AB0F166
:20D8E000FF3F05DA9448C0880A3800B29249C8807DE000BF94480078012857D18D48407882
:20D90000032805D10020914908808F4908706EE088484078012805D14FF4967006901E2042
:20D92000059003E0642006900A20059087480088401C8649088008460188069881422FDC49
:20D940007D48B0F904007C49B1F90610401A022814DD7E480188059891FBF0F0C0F10A0048
:20D960007A49098891FBF0F200FB121068BB7248C088284400B27049C88038E06E48B0F90D
:20D9800004006D49B1F90610401AB0F1FF3F2EDA6948C088A0EB0B0000B26749C88026E08D
:20D9A00000206A4908806849087020E06248B0F904006149B1F90610401A022806DD5E4815
:20D9C000C088284400B25C49C88010E05A48B0F904005949B1F90610401AB0F1FF3F06DA3A
:20D9E0005548C088A0EB0B0000B25349C8805248B0F90600062801DA062002E04E48B0F97D
:20DA000006004D49C8804F4800884A49097901EB8101162202EB4101884208DD01204649BA
:20DA200008700020C8804A4801F00FFE02E0484801F0FEFD474A117B474AD088474A1288E7
:20DA400000F000FB81464548A0F8009001231A4643480188484600F04FFC41490880354A6D
:20DA6000517A3D4A907D00F0DBFA0390314A527A0F3A91B2384A507D00F0D2FA0290DDE9B9
:20DA800002104843810A0491049988B201231A463449098800F030FC324908802E48C07B90
:20DAA000052801DC052007E02B48C07B0A2801DB0A2001E02848C07B2149098848434FF415
:20DAC0007A7190FBF1F000B2019023480089C111164A019803F04AFA234908801648B0F9BB
:20DAE00006001F49098848434FEAA0281D48008808FB00F04FEAA0281B48B0F9000040442A
:20DB00004FEA60080FFA88F0ADF8260001208DF82A0002208DF824000998CAF800000A9878
:20DB2000CAF804000FB0BDE8F08F0000C40500205408002020070020E0000020DE00002092
:20DB40002A0100203C0300202E01002030010020FC00002060070020380600203201002027
:20DB60003401002036010020280100202DE9FF5F82460E46874903C9CDE90201002700BFE5
:20DB80000025012E56D184484088400141F2883190FBF1F0C5B2012D01DA012000E02846EE
:20DBA00005467D48408840017C4909784843642190FBF1F00A387A494968884205D978486C
:20DBC000406828447649486026E0734840884001724909784843642190FBF1F00A30704955
:20DBE000496888420DD26E484068A84205D96C484068401B6A4948600EE00020684948602C
:20DC00000AE0654840884001644909784843642190FBF1F062494860624A1289D111624A92
:20DC2000127A4FF47A735A43D011604A03F09EF9044635E04FF000095B48C07F08B9872085
:20DC400001E05948C07F8146554840680A21C1EB4911884205D252484068401C5049486046
:20DC600010E04F4840680A2101EB4911884205D94B484068401E4A49486003E04FEA491013
:20DC800047494860474A1289D111474A127A4FF4FA735A43D011454A03F068F9044600BF07
:20DCA000404AB2F902103E4A5268520910B2404A03F05CF90746381907B2012E26D04FF031
:20DCC00000093948807F08B93C2001E03648807F814634480088A9F105018AB2009088B2CF
:20DCE00080230021F9F756F97843800A07B22D480088484506DD0020294948602D4801F016
:20DD0000A4FC02E02B4801F093FC02E0294801F08FFC214A117B234AD088274A128800F008
:20DD200091F980462448A0F8008001231A4623480188404600F0E0FA204908801A4A517A27
:20DD4000184A907D00F06CF9019001231A461C480188019800F0D0FA1949088017480088D9
:20DD600078434FEAA02B084600880BFB00F04FEAA02B0FFA8BF0ADF80C0001208DF80E002B
:20DD80008DF808000298CAF800000398CAF80400BDE8FF9F485F0108600700206B01002033
:20DDA000E800002038060020200700207C050020A0050020FC0000200A0100200C010020DC
:20DDC0000E01002070B504460D461646FBF782FC3C490968401A642870D3FBF77BFC39497C
:20DDE00008603948006828443749086037480078401C364908700846007808280ADB3248DF
:20DE00000068C0F3CF003249088000202F4908702D490860462C0BDA2D48008841F27071BF
:20DE2000884205DD2B480088401C2A49088002E0002028490880462C05DC2548008841F26E
:20DE40008831884207DA962E05DA23480088401C2149088002E000201F4908801D4800889B
:20DE6000B0F5967F05DD00201A49088001201B49087019480088642804DD002016490880A1
:20DE80001649087015480078012814D1462C0EDA04F11E001249087008460078642801DD58
:20DEA000642001E00E4800780D49087006E064200B49087002E06420094908700848007833
:20DEC00070BD00009C000020A0000020A4000020A6000020A8000020AA000020AC000020B1
:20DEE000AD0000202DE9FF4385B0074615469846DDE910944248827A08EA09012846069B47
:20DF000001F040FB06462078B04206D03D48007818B9052601203B490870062E5ED2DFE8E8
:20DF200006F05D144B2C035E05F00F0336480289BDF81A1003A8FEF771FD039820600498EE
:20DF4000606000202F49087056E030480078012807D12B48B0F9020040012C49486000202E
:20DF60000870394603A8FFF701FE03982060049860600020234908703EE025480079012862
:20DF800007D11F48B0F902004001214988600020087120480078CDE90150069800901A48F4
:20DFA0000EC803A8FDF71EFE03982060049860600020144908701FE05520CDE9015006984B
:20DFC000009011480EC803A8FEF798FF039820600498606000200B4908700DE000BF0E48E6
:20DFE00001F033FB0D48F7F7B7F9052020700020A0716080A08000BF00BF09B0BDE8F083DA
:20E0000038060020400100200C030020E8000020F000002020070020FC0000204401002032
:20E0200010B502464FF480608A4208DD01FB01F4A302B3FBF2F4B4FBF2F4A0B201E04FF4CA
:20E04000806010BDF0B503460E461546002100244FF48060182E04D0242E12D0302E34D15D
:20E0600021E0E721FC2401EBC10707EB0117B3EB870F02DD4FF4806701E0B3FBF1F73A4685
:20E0800025E04FF4A5714FF4B47401EBC10707EB0117B3EB870F02DD4FF4806701E0B3FB2D
:20E0A000F1F73A4613E040F2AD114FF4EA7401EBC10707EB0117B3EB870F02DD4FF4806779
:20E0C00001E0B3FBF1F73A4601E0642200BF00BF02FB02F74FF0640CB7FBFCF75743B7FBCE
:20E0E000FCF75743BF0242F2107CB7FBFCF2B2F54D7F02D24FF44D7700E017463A46AA427B
:20E1000001D290B200E0284604EBC40707EB0417B3EB870F01DD4FF48060F0BD2DE9F041AC
:20E1200005460E4617461C46002F7DD1552D66D14748007820BBFBF7CDFA45494968401A17
:20E14000B0F57A7F15D90120414908700020207040480078C043404908703E484078C0431B
:20E1600048703E48007820F00200801C3B49087018E03A48007820F002003849087011E051
:20E180000020207033480078C0433349087031484078C04348703148007820F00200801C5A
:20E1A0002E490870AA2E06D12C48007820F004002A49087023E02A480078C8B9FBF78AFAF2
:20E1C00027494968401AB0F57A7F0AD90120244908702248007820F00400001D1F4908704A
:20E1E0000DE01E48007820F004001C49087006E01A48007820F00400001D18490870194838
:20E200000078D8B9FBF766FA16494968401AB0F57A7F0CD90120134908701048007820F0E1
:20E220000100401C0D4900E00FE008700DE00B48007820F001000949087006E007480078A4
:20E2400020F00100401C05490870BDE8F081000074010020CA000020CC00002048010020A1
:20E260007C0100208401002001201549087000204860012013490870002048808880C88070
:20E280000120114908700020488001200871002088600E4908600E4908600E4908600E496D
:20E2A00008600E4908600E4908620E4908620E4908620E4908620E4908620E4908627047FA
:20E2C000E8000020E0000020F000002004000020080000200C00002010000020140000204A
:20E2E000340500201005002058050020C4050020A00500207C05002070B504461546661A7A
:20E3000032B2002A06DDAA4202DB4E19B0B20CE020460AE0002A07DA56429E4202DBCE1AF6
:20E32000B0B202E0204600E0204670BD70B505460E46144608216748FBF7BAF966490870FE
:20E340004FF400416548FBF7B3F96549087062480078644909784840634908705E480078AE
:20E36000604908705E480078604909784840604908705B4800785D4908705748007858499A
:20E38000097848405B490870FBF7A4F9B0F57A7F0CD2FBF79FF958490860FBF79BF9574994
:20E3A0000860FBF797F95649086070BD2088C0F38030002878D1B5F5966F7CDD462E7ADDF0
:20E3C0004948007800BBFBF785F94B490968401A42F2107188421BD9206820F4804000F5E6
:20E3E000804020600120474948800846F8F748FB00204549087045484088401C43494880B9
:20E40000022043490870D0E7FBF764F93A4908603748007800BBFBF75DF938490968401A9F
:20E4200041F2883188421BD9206820F4804000F5804020600220334948800846F8F720FBE3
:20E4400000203149087031484088401C2F49488002202F490870A8E7FBF73CF9274908602D
:20E460002448007810BBFBF735F925490968401A41F2883188422AD9206820F4804000F58A
:20E480008040206003201F4948800846F8F7F8FA00201D4908701D484088401C1B49488007
:20E4A00002201B49087080E711E004E0FBF712F9134908600BE0FBF70DF90F490860FBF7CC
:20E4C00009F90E490860FBF705F90D49086000BF6BE70000000C01405C02002000080140A8
:20E4E0005D02002045020020440200204D0200204C020020540200204802002050020020A1
:20E50000580200207C100020EC020020A0070020560100201FB53A48007890B93948807EF3
:20E5200055280ED1384A394800783949498889B2CDE9010200913749887837490EC900F065
:20E54000ABFE314931480078CDE902013249D1E90101324BCDE900011A78314B5988314B18
:20E5600018892D4B1B6800F02FFF274801902E488088ADF80000264B5B889AB2244B19890D
:20E58000224B9879284B1C6802949B88ADF80C30234600F0A1FD1E4A917D507D1A4A00F0DE
:20E5A0001DFD20498889184900F074FA1E48016802918088ADF80C00134ADDE9020100F0D7
:20E5C000D1FB114800F03CF80F48134A009011780F4A528890B2124A12680392134A13884D
:20E5E000039A00F093FC0848114900904A8911490878114B1149098800F00EFB1FBD0000FC
:20E60000C80000202007002044010020CE000020380600203C0300200C030020CA000020A2
:20E62000EE03002048130020FE030020960100205A1300206C010020C710002068010020DC
:20E6400010B50446FBF746F841F2883188420CD2FBF740F8EE490860FBF73CF8ED4908605A
:20E66000FBF738F8EC49086010BD2068C0F3804000286FD14FF40041E848FBF719F800BB39
:20E68000FBF728F8E3490968401A41F2883188421BD9206820F4802000F580202060012055
:20E6A000DF4948800846F8F7EBF90020DD490870DD484089401CDC4948810220DB49087095
:20E6C00003E0FBF707F8D3490860D9480088002847D1D8480078012843D1D7480078052860
:20E6E0003FD0D548807901283BD1D348B0F90400C82804DCD048B0F90200C82831DDCF4850
:20E70000807A40BBCE480089C82825DAFAF7E2FFC1490968401A41F28831884225D9206893
:20E7200020F4802000F5802020600220BC494880BF48008888800846F8F7A2F90020B94990
:20E740000870B9484089401CB74948810220B74908700AE08DE0FFE7FAF7BCFFAE49086070
:20E7600003E0FAF7B7FFAC490860FAF7B3FFA8490968401A14287CD3FAF7ACFFA4490860D7
:20E78000B048C088B04909680844AF490860AF480088AF4909680844AD490860AB484088D6
:20E7A000AC4909680844AB490860A8488088AA4909680844A8490860A8480078401CA74996
:20E7C00008700846007820287EDB002008709E4800684FF4FA71B1EB501F2FD89A4800686A
:20E7E000C900B1EB501F29D39948006841F28831B1EB501F22D8964800684EF66021B1EB68
:20E80000501F1BD39348006841F28831B1EB501F14D8904800684EF66021B1EB501F0DD385
:20E820008D48006841F28831B1EB501F06D88A4800684EF66021B1EB501F16D2206820F438
:20E84000802000F5802020600320754948800846F8F716F900207349087073484089401CDA
:20E86000714948810220714908707D480068C82100E0C2E0B1EBA02F36DA7A4800887249A9
:20E880000968C0EB511019282AD277480078401C75490870084600780A2828DD206820F45C
:20E8A000802000F58020206004205D49488066480068C0F34F1088800846F8F7E1F80020AB
:20E8C00058490870584800E01AE04089401C5649488102205549087000206349087006E0B6
:20E8E00000206149087002E000205F49087000205549086056490860564908605649086079
:20E900004F48407B00287AD14D484088002876D1FAF7E0FE55490968401A41F28831884278
:20E9200074D94848C0885249524A127821F812004648008850494F4A127821F8120043483E
:20E9400041884E484B4A127820F812103F4881884B48484A127820F8121046480078401C24
:20E96000444908700846007832284FDB0020087032213F48F8F741FD4249086032213E48DD
:20E98000F8F73BFD4049086032213C48F8F735FD3E49086032213A48F8F72FFD3C4908609B
:20E9A00038480068B0F5FA7F0DD83748006842F6E061884207D835480068884203D834485D
:20E9C0000068884222D9206820F4802000F5802020600520124948802A4800888880084621
:20E9E000F8F74EF800200F4908700F484089401C0D49488102200D49087007E0FFE700207A
:20EA00001C490870FAF766FE1849086000BF2BE6E8010020EC010020F001002000100140B3
:20EA20007C100020EC020020A0070020560100206001002030000020CE000020BC10002033
:20EA4000380600205A130020F8010020E6030020FC0100200002002004020020F40100202F
:20EA60000400002004040020F50100201C020020220E002008020020860E0020EA0E0020B0
:20EA80004E0F00200C0200201002002014020020180200207047000013B50C465448007844
:20EAA00060B9FAF717FE534908609DF8012006215148F5F706F801204D4908702078C0F359
:20EAC000C01000287ED19DF8000018B19DF80000072821D1FAF7FEFD46490968401AB0F5F0
:20EAE0007A7F1DD9206820F08000803020600120424948809DF8000088800846F7F7C0FFD3
:20EB000000203F4908703F48C08A401C3D49C88201203D4908701CBDFAF7DCFD3549086030
:20EB20009DF800009DF8011088425FD09DF80010364802780078401C344B18702E488154DE
:20EB400018460078062851DB00201946087006212948F6F7D1F928B92D480068401C2C49B0
:20EB6000086006E000202A490860FAF7B3FD2949086027480068322838D9FAF7ABFD254988
:20EB8000096801F5FA71884230D9206820F080008030206002201949488017480078000263
:20EBA0001549497800EB0110134989780844134988801148C07800020F49097900EB0110C4
:20EBC0000D4900E012E0497908440C49C8800846F7F756FF00200A4908700A48C08A401CEE
:20EBE0000849C88201200849087094E700BF92E72E02002030020020380200207C10002035
:20EC0000EC02002070070020560100203E02002040020020340200202DE9F04105460E46DA
:20EC200014469846069FFAF755FDB0F57A6F01D2BDE8F081FAF74EFD42F21071884220D290
:20EC40003868C0F3804000287CD1FAF743FD3E490968401A142875D3FAF73CFD3A49086010
:20EC600098F80000A8BB0DB1C82E0BDD40F2C270844207DD40F63E00844203DA0020334944
:20EC800008705FE031480078401C3049087008460078FA2856DB00200870386820F480207A
:20ECA00000F58020386008202949488005EB860088800846C480F7F7E3FE002025490870E0
:20ECC00025484089401C2449488102202349087038E0FFE70DB1C82E03DD002088F8000034
:20ECE00030E040F68B60844202DCB4F5BA7F26DA1B480078401C1A49087008460078FA2863
:20ED000020DB00200870386820F4802000F58020386009200E49488005EB860088800846CB
:20ED2000C480F7F7ADFE00200A4908700A484089401C0949488102200849087002E000208C
:20ED40000749087000BF73E7280200202C0200207C100020EC020020A00700205601002042
:20ED60002D02002037B514466048007801280CD0FAF7B0FC5E490860FAF7ACFC5D49086086
:20ED8000FAF7A8FC5C4908603EBD2068C0F30040002875D1BDF90000002801DB014600E00C
:20EDA000414244F62062914228DDFAF793FC50490968401AB0F57A7F24D9206820F4803071
:20EDC00000F58030206001204C494880BDF90000002801DB014600E04142484A9180104633
:20EDE000F7F74EFE0020464908704648C088401C4449C880022044490870C5E7FAF76AFC81
:20EE00003B490860BDF90200002801DB014600E0414244F62062914228DDFAF75BFC354946
:20EE20000968401AB0F57A7F24D9206820F4803000F580302060022030494880BDF90200E0
:20EE4000002801DB014600E041422C4A91801046F7F716FE00202A4908702A48C088401C04
:20EE60002849C8800220284908708DE7FAF732FC20490860BDF90400002802DB014601E083
:20EE800031E0414244F62062914228DDFAF722FC19490968401AB0F57A7F24D9206820F4D7
:20EEA000803000F580302060032014494880BDF90400002801DB014600E041420F4A918063
:20EEC0001046F7F7DDFD00200D4908700D48C088401C0C49C88002200B49087054E7FAF776
:20EEE000F9FB0549086000BF4EE7000030000020D0010020D4010020D80100207C10002099
:20EF0000EC020020A0070020560100202DE9FF4105460E461F460A9C2068C0F38050002872
:20EF20004DD1FAF7D7FB27490968401A142846D3FAF7D0FB23490860B5F5FA7F3CDD0F2E57
:20EF40003ADBBDF80800C82836DDBDF80A00322832DA40F2DC5087422ADD1B480088401C42
:20EF60001949088008460088FA2828DB00200880206820F4800000F5800020600120134976
:20EF80004880BDF808008880BDF80A00C8800846F7F776FD00200E4908700E4890F824003D
:20EFA000401C0C4981F8240001200B49087006E000200549088002E0002003490880BDE8BF
:20EFC000FF81000020020020240200207C100020EC020020700700205601002070B50446F2
:20EFE0000E461546FAF776FB41F28831884201D35A2C08DDFAF76EFB31490860FAF76AFB79
:20F000002F49086070BD2888C0F34020002855D1052C01DBBE2C22DDFAF75CFB28490968B2
:20F02000401A41F2883188421DD9286820F4007000F5007028600120224948800846848023
:20F04000C680F7F71DFD00201F4908701F48408B401C1E49488301201D490870D2E7FAF7F9
:20F0600039FB17490860052E01DBBE2E22DDFAF731FB18490968401A41F2883188421DD9A5
:20F08000286820F4007000F50070286002200D49488008468480C680F7F7F2FC00200A4948
:20F0A00008700A48408B401C08494883012008490870A7E7FAF70EFB0649086000BFA1E7D3
:20F0C000C80100207C100020EC0200207007002056010020CC0100200FB42DE9F04105463D
:20F0E0000E4617460B9C2088C0F30020002877D1012D76D141F28830864272DDB7F5FA7F31
:20F10000FBDDBDF92400002801DB014600E04142B1F5967F2CDAFAF7DDFA58490968401A9A
:20F1200041F28831884227D9206820F4807000F580702060012052494880BDF924000028A2
:20F1400001DB014600E041424D4A91801046F7F797FC00204B4908704B48008B401C4A4971
:20F160000883012049490870BDE8F0015DF814FBFAF7B0FA41490860BDF92600002801DB72
:20F18000014600E04142B1F5967F2BDAFAF7A2FA3F490968401A41F28831884226D92068E8
:20F1A00020F4807000F580702060022034494880BDF92600002801DB014600E04142304A7B
:20F1C00091801046F7F75CFC00202E4908702E48008B401C2C49088301202C490870C3E75E
:20F1E0003CE03CE0FAF776FA29490860BDF92800002801DB014600E04142B1F5967F29DA52
:20F20000FAF768FA23490968401A41F28831884231D9206820F4807000F580702060032090
:20F2200017494880BDF92800002801DB014600E04142134A91801046F7F722FC00201149D0
:20F2400008701148008B401C0F49088301200F49087089E7FAF73EFA0E4908600BE0FAF7EE
:20F2600039FA06490860FAF735FA09490860FAF731FA0849086000BF76E70000BC010020FC
:20F280007C100020EC0200207007002056010020C0010020C40100202DE9FF410646DDE978
:20F2A0000A870C9C00252078C0F34010002878D1052F08D1FAF70EFA3B490860FAF70AFAFD
:20F2C0003A4908606DE0012F01D0042F32D1B8F1320F2ADD4EBB364890FBF8F085B242F269
:20F2E0001070854200DA00E028460546FAF7F2F92D490968401AA84253D9206820F0200069
:20F300002030206001202B4948800846F7F7B8FB0020294908702948408A401C27494882F6
:20F32000012027490870BDE8FF81FAF7D3F91E49086036E09DF8040005282EDB9DF8050094
:20F3400058BB56BB9DF804001E4991FBF0F085B242F21070854200DA00E028460546FAF707
:20F36000B9F912490968401AA8421AD9206820F020002030206002200E4948800846F7F7D3
:20F380007FFB00200C4908700C48408A401C0B49488201200A490870C5E7FAF79BF9034905
:20F3A000086000BFBFE70000A4010020A801002048F13E007C100020EC020020700700202A
:20F3C00056010020D8B805000FB42DE9F047044688461746DDE90E95FAF77CF941F28831E1
:20F3E000884207D2FAF776F94C490860FAF772F94B490860FAF76EF94A490968401A1428C3
:20F400007ED3FAF767F947490860002607E04649701C31F8100021F81600701C86B2182EB8
:20F42000F5D3414804862878C0F38010002872D119213D48F7F7E1FF3C490860222F3AD0CE
:20F4400007F00F00B0B3B8F5FA7F34DA9DF82C001E2830DD9DF82D0060BBB9F1020F2AD168
:20F46000084600680A2826D2FAF734F92B490968401A43F69821884221D9286820F04000B9
:20F480004030286001202A4948802848008888800846F7F7F5FA0020264908702648808A6E
:20F4A000401C25498882012024490870BDE8F0075DF814FBFFE7FAF70DF918490860322C6E
:20F4C00003DB40F6D270844221DDFAF703F914490968401AB0F57A7F1DD9286820F0400089
:20F4E0004030286002201249488008468480F7F7C7FA00200F4908700F48808A401C00E041
:20F5000009E00D49888201200C490870CEE7FAF7E1F80349086000BFC8E70000AC01002046
:20F52000B0010020B8010020F00D0020B40100207C100020EC020020700700205601002067
:20F5400010B50C49487B01F02BFC0A49487B05F0AFF9094803F0F0FB0748F5F7FDFE07484F
:20F560000189074804F0BAFC01F01AFE012001F043FE10BD200700204401002048130020B8
:20F580005C1100202DE9FF4104460D461746052621480068002831D1012D2AD1FAF79AF8BC
:20F5A00040F6B831884224D900BFFCB1222C01D101261AE004F0F000102816D0022617482F
:20F5C000008864280FDABDF80E00C8280BDD14480078022802D11348807A18B110480078D4
:20F5E000012800D101260E48067001E0052600BF00E00526012001F0FFFD08E00526002007
:20F600000949087008460078C04308490870304604B0BDE8F081000044010020380600208B
:20F62000FD000020BC100020CA000020CC00002010B50446207838B9F7F7C0F9FBF792FD2B
:20F64000F7F754FB0120207010BD10B5044601F0C1FEF7F739FBFEF707FE0020207010BD97
:20F660002DE9F04107460D46144605EB4500C0F34F06207800F0010050BBB74203DAFAF7B1
:20F6800029F81C490860FAF725F81A490968401A41F2883188422AD9206820F00100401C92
:20F6A000206002201449488008468680F7F7E8F900201249087012480089401C104908814C
:20F6C000012010490870FAF705F80F4908600EE0FAF700F80C490968401A41F288318842DD
:20F6E00005D90A48006820F0010008490860BDE8F0810000900200207C100020EC02002026
:20F70000700700205601002094020020440100201CB528492848808B10B940F6B83001E03B
:20F720002548808B254CCDE90001237B244C247814B9244C248801E0234CE4882246224C04
:20F74000E17B1F4C207800F0F7F91C4A117B2246127812B91B4A128801E01B4AD2881046C6
:20F76000144A00F0FFF8194A917A174A1089114A00F060F90F48104C0090A37A124CA27D5B
:20F78000617DE07D00F04EF822461189D088094A00F094FA084A127A02EB4203C3EBC2123B
:20F7A0004FF6FF7303EAC20122461089014AFFF757FF1CBD4401002020070020600700203E
:20F7C00084010020B806002038060020BC10002070B504460D46207868B900200F490870F1
:20F7E0000F480078C0B90E480078401C0C490870F7F7CAF810E00020094908700748007879
:20F80000012802DB0020207001E0F6F70FFE03480078401C0149087070BD0000980200208F
:20F82000990200202DE9F04180460E4617461C46069DF9F74FFF40F6B831884207D2F9F75A
:20F8400049FF40490860F9F745FF3F4908602878C0F3001000283DD13C48C07A58B9A4F14E
:20F860001900B04215DD601D874212DAF9F732FF344908600DE0A4F12300B04209DD601D59
:20F88000874206DA1938404503DDF9F723FF2D490860F9F71FFF2B490968401A41F28831E0
:20F8A00088424CD9F9F716FF27490860286820F01000103028602648F7F7E2F80020254940
:20F8C00008702548008A401C2349088201202349087034E01D48C07AB8B9A4F12300B04294
:20F8E0002DDD0F30B8422ADDF9F7F4FE16490968401A1B49884222D9286820F01000286051
:20F90000F9F7E8FE0F49086019E0A4F12D00B04215DD1930B84212DD0A3840450FDDF9F7DD
:20F92000D9FE09490968401A0D49884207D9286820F010002860F9F7CDFE02490860BDE888
:20F94000F08100008002002084020020BC1000207C100020EC02002070070020560100203A
:20F96000E09304002DE9F04105460E4614460027182E04D0242E05D0302E09D105E047F60E
:20F980000C3707E04AF6C87704E04EF2844701E02F4600BF00BF2078C0F3800030BBBD4246
:20F9A00003DCF9F797FE1D490860F9F793FE1B490968401A41F28831884212D9206820F02C
:20F9C0000400001D20601648F7F75AF800201549087015488089401C13498881012013494E
:20F9E0000870F9F777FE1249086014E0A7F5FA70A84203DAF9F76EFE0D490860F9F76AFE34
:20FA00000B490968401A41F28831884203D9206820F004002060BDE8F08100006C02002075
:20FA20007C100020EC02002070070020560100207002002070B505460E4614462078C0F303
:20FA4000C000002848D1012E08D1F9F743FE30490860F9F73FFE2F49086014E040F6C41080
:20FA6000854208DAF9F736FE29490860F9F732FE2849086007E041F64C50854203DAF9F798
:20FA800029FE24490860F9F725FE21490968401AB0F5FA5F08D8F9F71DFE1E490968401A07
:20FAA00040F6B831884232D9206820F00800083020601948F6F7E4FF002018490870184870
:20FAC000C089401C1649C881012016490870F9F701FE154908601AE0F9F7FCFD124909687D
:20FAE000401A41F28831884211D91048007870B90F4800880A280ADA0D4840880A2806DAEF
:20FB00000C48807818B9206820F00800206070BD74020020780200207C100020EC02002091
:20FB200070070020560100207C020020CA000020EE0300200C0300202DE9F0470746884687
:20FB400015469A46DDE908940026BAF1180F06D0BAF1240F07D0BAF1300F11D10AE0C9EB1B
:20FB6000C90086B20EE009EB89004FF6FF7101EA400607E009EB890000EBC90086B201E002
:20FB80002E4600BF00BF002F48D12078C0F3400058BBB8F1010F05DBB54203DBF9F79AFD98
:20FBA00040490860F9F796FD3E490968401A41F28831884214D9206820F00200801C206026
:20FBC000394845808780F6F75BFF00203749087037484089401C3649488101203549087076
:20FBE000F9F778FD344908605AE0B8F1010F03DB06F57A70854203DAF9F76CFD2E49086029
:20FC0000F9F768FD2C490968401A41F28831884246D9206820F00200206041E02078C0F3F4
:20FC2000400040BBB54203DBF9F754FD1D490860F9F750FD1B490968401A41F28831884283
:20FC400014D9206820F00200801C2060164845808780F6F715FF00201449087014484089BC
:20FC6000401C13494881012012490870F9F732FD1149086014E006F57A70854203DAF9F7C1
:20FC800029FD0D490860F9F725FD0B490968401A41F28831884203D9206820F002002060A3
:20FCA000BDE8F087640200207C100020EC0200207007002056010020680200202DE9F04109
:20FCC0000746884614460026F9F704FD2B490968401A642850D3002507E02949681C31F87F
:20FCE000100021F81500681C85B2092DF5D3244847820A21F7F781FB06462068C0F340403C
:20FD000090BBB8F1320F2BDAB6F57A7F28D91D480078322830DD206820F4003000F50030CF
:20FD20002060C6F30F20184948800A211448F7F7D9FA154988800A211148F7F7E4FA1249D9
:20FD4000C8800846F6F79CFE00201049087010480089401C0E49088102200E4908700BE09C
:20FD600000200849087007E0FFE7B6F57A7F03D8206820F400302060BDE8F0818802002042
:20FD8000E80500208C0200207C100020EC020020A00700205601002010B5F9F79BFC9D497E
:20FDA0000968401AC8287DD3F9F794FC994908609948008900EBC00101EB00119748007A02
:20FDC00064225043B1FBF0F09349888008468088142801DA002001E08F4880888E4988806E
:20FDE0008F48407808738F4800881C2190FBF1F08949C8728C48007848738B484078887358
:20FE00008A48007800F0010068B10846C08800EBC00080008649097B90FBF1F084B2204672
:20FE2000F4F794FA01E08348407A7B49C8730846C07B88B17D48007800F0010010B14EF6EF
:20FE4000EE6006E07C48C08A08B9012001E07A48C08A714908820BE07448007800F001003D
:20FE600010B14EF6EE6001E07348C08A6A4908826A48807EEE2818D170488078012826D18D
:20FE80006E48806844F62061B1FBF0F06C49096808446B490860084600686421B0FBF1F028
:20FEA000664900E0B5E0C86011E05C48807EAA280DD15B4840685949897948435749C97957
:20FEC000B0FBF1F03221B0FBF1F05C49C8605348007B524991F91B10084442F2107191FBF7
:20FEE000F0F05649C968574A1268891A884206D80120554908705148C06852490860524857
:20FF00000078012838D100204F4908704F480068401C4E49086008468068401C88600846E5
:20FF200080684B49884203D9002048498860C8603948008B401C38490883444800680A214B
:20FF4000B0FBF1F03449488242480078401C41490870084600781E280EDB3F4B30224C2130
:20FF60003E4803F07AF8394B1022D6213B4803F074F8002037490870274800881E281ADBBD
:20FF800037480078401C3649087008460078052814DB0020087033480088401C314908803C
:20FFA0001D48408B401C1C4948832F480078401C2D49087002E00020294908702A48007876
:20FFC0003C280BDB00202849087020484068401C1E4948600846C068401CC8602148008868
:20FFE000B0F5167F0EDB00201E4908801A4B30224C211A4803F031F8144B1022D621174846
:020000040801F1
:2000000003F02BF80C48808A0A2190FBF1F00249087510BD6C00002038060020200700200F
:200020000C030020EE030020CA0000204801002060070020B80600209C0200203C030020AB
:200040007C0000207000002074000020A80800209F86010080000020700700207C03002014
:2000600075000020780000207600002010B50446F9F730FB10490968401A4EF660218842E0
:2000800018D3F9F727FB0C4908602068401C20600A480078401C09490870084600780A285A
:2000A00008DB074B30224C21064802F0D6FF00200249087010BD0000B8000020BC000020D3
:2000C000700700207C03002001B511480078022800D108BD0098A0B1F9F7FCFA0D4909680D
:2000E000401AB0F5FA7F10D9F9F7F4FA094908606B4641F204120C214FF4E26003F044F82C
:2001000003E0F9F7E7FA0349086000BFE1E700005D0000208400002010B50446012C13D1AF
:20012000F9F7D8FA0B490968401AC82810D30A4B4FF481520C214FF4E26003F025F8F9F7EE
:20014000C9FA0449086003E0F9F7C4FA0149086010BD0000880000203806002010B5FBF75A
:2001600013F8FAF7FFFFF4F703FD03F077F9FBF7D7FA05480189054803F0F8FE0248818913
:200180000348F7F711F810BD481300205C110020C40300201CB50446F9F79CFA40490968C6
:2001A000401AB0F5FA7F7AD33E480088401C3D49088008460088142837DB3B48007800F0F3
:2001C000010010B900203949487437480088C0F3002010B900203549087433480078C0F394
:2001E000801010B90020314908812F480078C0F3C01010B900202D4948812B480078C0F34B
:20020000001010B900202949888127480078C0F3401010B900202549C8814FF48051244860
:20022000F9F74EFA00201F4908802248007868B900204FF408430C2240F2FF7100901E48FF
:2002400002F0EEFF01201B49087024E019480078012820D100200190184801780078401C6D
:20026000164A107005290CDC01A841F20133162240F2FF710090104802F0D2FF0A20F8F7DA
:2002800043FF41F214030C2240F2FF710A48009402F0C6FF00BFF9F71DFA014908601CBD14
:2002A00094000020980000206001002040080020001001405D000020BC0400209A00002081
:2002C00070B504464D48007880BB08214C48F9F7EFF94C4908704FF400414B48F9F7E8F9DD
:2002E0004A49087080214A48F9F7E2F9494908704FF480714648F9F7DBF9474908704FF41A
:2003000000514348F9F7D4F94449087004214448F9F7CEF943490870002020816081A08110
:20032000E081207460740120344908703E48C08860803D488088A0804FF40060E0803A48FE
:200340000089208008212E48F9F7B2F905462D480078A84202D02089401C208129480570BA
:200360004FF400412848F9F7A3F9054627480078A84202D06089401C608124480570802167
:200380002348F9F795F9054622480078A84202D0A089401CA0811F4805704FF480711C4871
:2003A000F9F786F905461C480078A84202D0E089401CE081184805704FF400511448F9F710
:2003C00077F9054615480078A84202D0207C401C20741248057004211148F9F769F905465B
:2003E00010480078A84202D0607C401C60740D4805704FF47A70608270BD000092000020AD
:20040000000C01408C000020000801408D000020001001408E0000208F000020900000208F
:2004200000140140910000205A13002010B5F9F751F942F21071884204D2F9F74BF9414917
:20044000086010BDF9F746F93E490968401A41F28831884274D3F9F73DF93A4908603A4856
:20046000407D3A4991F82310884207DA3648407D364981F823000020354908703248407D32
:20048000324991F82210884207DD2F48407D2F4981F8220000202E4908702B48807D2B493E
:2004A00091F82910884207DA2748807D274981F829000020264908702348807D234991F8ED
:2004C0002810884207DD2048807D204981F8280000201F4908701C48C07D1C4991F82B10FD
:2004E000884207DA1848C07D184981F82B000020174908701448C07D144991F82A10884234
:2005000007DD1148C07D114981F82A0000201049087010480088401C0E4908800846008882
:200520000C280DDD0A48007850B900200880012007490870054B30224C21074802F08DFD5F
:2005400000BF7EE7C00000203806002070070020C6000020C40000207C03002010B5074825
:20056000007850B9F9F7B6F804494968401AB0F5FA6F02D901200149087010BD6C010020DE
:2005800000B587B0012003900320049003A90E48F8F700FF0D480068806820F001000B490A
:2005A0000968886000200090082001900720029069460648F7F7D6F920B140F28F2104A0AF
:2005C00004F0BAFC07B000BD000801406C1300202E2E5C436F72655C5372635C6164632E9E
:2005E000630000000EB550485049086081154F4881600021C16041614FF46021C161002044
:200600004A494860092149480161F7F78DFC18B1582147A004F090FC0A20009001200190F6
:200620000720029069464148F7F79CF918B162213FA004F081FC0B20009002200190072015
:20064000029069463948F7F78DF918B16C2138A004F072FC0C2000900320019007200290AB
:2006600069463248F7F77EF918B1762130A004F063FC0D2000900420019001200290694695
:200680002A48F7F76FF918B1802129A004F054FC0520009001900120029069462348F7F71A
:2006A00061F918B18A2122A004F046FC07200090062001900720029069461C48F7F752F901
:2006C00018B194211AA004F037FC0E200090072001900120029069461448F7F743F918B194
:2006E0009E2113A004F028FC10200090082001900220029069460D48F7F734F918B1A82192
:200700000BA004F019FC11200090092001900720029069460548F7F725F918B1B22104A0A9
:2007200004F00AFC0EBD0000002401406C1300202E2E5C436F72655C5372635C6164632E79
:200740006300000000B589B02348244908608115224881600021C1604161C16100201F4999
:20076000486001211D480161F7F7DEFB18B1C6211BA004F0E1FB01200190029003200590EA
:20078000002003904FF480500890002007900690049001A91148F6F7DBFE18B1D52110A0E2
:2007A00004F0CAFB02200190029001A90B48F6F7CFFE18B1DE210AA004F0BEFB03200190B1
:2007C000029001A90548F6F7C3FE18B1E72104A004F0B2FB09B000BD002801409C1300201E
:2007E0002E2E5C436F72655C5372635C6164632E6300000010B50F480F490860302048604B
:2008000000210D488160C1604FF4403101610021416181610121C161002101624162816257
:20082000C162F7F7C1FF18B1542104A004F084FB10BD0000006400407C1800202E2E5C4372
:200840006F72655C5372635C63616E2E6300000008B500BF0A48406940F00100084948610D
:200860000846406900F00100009000BF00BF022211460B20F8F7FDFF0B20F8F7EDFF08BD26
:200880000010024000B585B000BF3A48806940F01000384988610846806900F01000009081
:2008A00000BF00BF00BF0846806940F0200088610846806900F02000009000BF00BF00BF77
:2008C0000846806940F0040088610846806900F00400009000BF00BF00BF0846806940F065
:2008E000080088610846806900F00800009000BF00BF002289142048F8F7E6FE4EF2203040
:2009000001900320029001A91B48F8F743FD40F6187001900320029001A91848F8F73AFD21
:200920004EF6024001900320029001A91448F8F731FD4FF480500190124802900020039085
:2009400001A90F48F8F726FD4FF480500190012002900220049001A90748F8F71BFD002255
:2009600011462820F8F785FF2820F8F775FF05B000BD00000010024000100140000801405C
:20098000000C01400000211010B50848084908600320486040F2E24105488160F8F7A0FE30
:2009A00018B13A2103A004F0C7FA10BD00300040040600202E2E5C436F72655C5372635C33
:2009C000697764672E63000000B595B03148324908600020486020212F4881604FF416616A
:2009E000C1600021016101214161F9F723FE4FF48050119011A92848F9F7C4FE2648FAF78F
:200A0000F5F870200F90802010900FA92248F9F79AFD4FF4006008904010099000200A90F3
:200A200039200B9000200C900D900E9008A91A48F9F74AFD6FF080001749096808616020E8
:200A400001904FF496600290002003900490059006900790002201A90F48FAF743F80422BC
:200A600001A90D48FAF73EF8082201A90A48FAF739F86020019040F65F100290002003900D
:200A8000082004900C2201A90348FAF72BF815B000BD0000002C01408812002000B587B0CE
:200AA00000200390049005900690019002904FF080401949086000204860002116488160B0
:200AC0004FF6FF71C1600021016141618161F9F7B1FD18B17E2111A004F02EFA4FF40050D3
:200AE0000390002004900590069003A90A48F9F749FE18B1862109A004F01EFA0020019079
:200B0000029001A90448F9F71EFD18B18C2103A004F012FA07B000BDC81200202E2E5C55AE
:200B20007365725C5372635C74696D2E6300000000B589B01C481D490860002048600021A7
:200B40001A4881604721C1600021016180218161FAF74CF820B14FF48F7115A004F0ECF9EC
:200B600000200790089007A91048F9F7ECFC20B140F225110EA004F0DFF96020009024203F
:200B80000190002002900490002269460748F9F7A9FF20B14FF4977105A004F0CDF9034800
:200BA000F9F756FF09B000BD00040040081300202E2E5C557365725C5372635C74696D2E4C
:200BC0006300000010B50C480C4908604FF416504860002109488160C16001610C214161E6
:200BE00000218161C161FAF71DFA18B1462104A004F0A2F910BD000000480040C01A002016
:200C00002E2E5C436F72655C5372635C75736172742E630000BFFEE730B504460A460021AF
:200C2000002329480078401C274D2870284600780F2841DB0020287024480089244D2D8834
:200C4000411B002907DA214800894FF6FF7528441F4D2D88411B44F62060814200DD00211F
:200C60001A4800891A4D28804FF47A70414319480068081A174D2D6805EB2020154D2860CB
:200C8000284600680314C3EB031040F35C0000B2114D28800D488089104D2D68C5EB8020BF
:200CA0000E4D2D6805EB60100C4D286028460068C0F38F20054DE88112B90020064D28802A
:200CC0000548B0F9000030BDFA020020BC100020FC02002000030020080300200403002096
:200CE0002DE9F04107460C46154629462046F6F779FA8046002606E0701C34F8100024F8C8
:200D00001600701C86B2681EB042F5DC24F810704046BDE8F081704702480068C0F302203A
:200D2000704700000CED00E010B5002807DA0A07140E054A00F00F031B1FD45403E00A077B
:200D4000130E024A135410BD18ED00E000E400E010B5F8F7BFFC40F6B831884216D90C48AE
:200D60000078012812D10020094908700948C07AAA280BD133200849087008460078C043E7
:200D80000649087004484078C043487010BD0000C700002020070020CA000020CC000020FC
:200DA00010B50446012C06D0022C23D0032C40D0042C7DD15CE024224E494F48F2F76FFE3D
:200DC00024224E494E48F2F76AFE24224D494E48F2F765FE24224D494D48F2F760FE242293
:200DE0004C494D48F2F75BFE24224C494C48F2F756FE7CE024224B493F48F2F750FE2422A1
:200E000049493F48F2F74BFE242248493E48F2F746FE242246493E48F2F741FE24224549A6
:200E20003D48F2F73CFE242243493D48F2F737FE5DE0242241493048F2F731FE2422404929
:200E40002F48F2F72CFE24223E492F48F2F727FE24223D492E48F2F722FE24223B492E482B
:200E6000F2F71DFE24223A492D48F2F718FE3EE0242238492048F2F712FE242236492048BE
:200E8000F2F70DFE242235491F48F2F708FE242233491F48F2F703FE242232491E48F2F721
:200EA000FEFD242230491E48F2F7F9FD1FE0FFE7242210491048F2F7F2FD24220F49104889
:200EC000F2F7EDFD24220F490F48F2F7E8FD24220E490F48F2F7E3FD24220E490E48F2F7E3
:200EE000DEFD24220D490E48F2F7D9FD00BF00BF10BD00005059010810050020745901085E
:200F0000340500209859010858050020BC5901087C050020E0590108A0050020045A0108D4
:200F2000C4050020285A01084C5A0108705A0108945A0108B85A0108DC5A0108005B010806
:200F4000245B0108485B01086C5B0108905B0108B45B0108D85B0108FC5B0108205C010860
:200F6000445C0108685C01088C5C01082DE9F04304460D46601B06B2B2F9000000FB06FC49
:200F8000908810B90020106212E0B2F9040000FB06F7106AC319D069984202DAD069106255
:200FA00006E09069984202DD9069106200E0136250889CFBF0F0B2F80690D2F8208098FB4D
:200FC000F9F800EB0801002906DA1069884203DD108A00B2BDE8F083002905DD506988420E
:200FE00002DC908A00B2F5E708B2F3E72DE9F34F83B00C46204602F0F5FF00901D48009920
:201000000160BDF90C001B49B1F9001000FB01F7FF13BDF90E001749B1F9021000FB01F8B6
:201020004FEAE8380FFA87FB0FFA88F001900198ABEB000000B2ADF80800BDF90C000D4914
:20104000B1F9021000FB01F5ED13BDF90E000949B1F9001000FB01F6F6130FFA85F90FFA88
:2010600086FA09EB0A0000B2ADF80A00029805B0BDE8F08F4C0000207047000030B50246CE
:20108000B2F900303F4CB4F90040A34202DD13883C4C2380B2F902303B4CB4F90040A3423D
:2010A00002DD5388384C2380B2F90430374CB4F90040A34202DD9388344C2380344B1B88DC
:2010C0005B1C1BB2324C23802346B3F90030B3F5FA7F56DB2B4BB3F900000023294C2380B7
:2010E000031E01DB1C4600E05C42B5256C43294D2D68C5EB8404274D2D6805EB6414254D64
:201100002C602B461B689B121BB20B801E4BB3F9000000231C4C2380031E01DB1C4600E0C8
:201120005C42B5256C431C4D2D68C5EB84041A4D2D6805EB6414184D2C602B461B689B125C
:201140001BB24B80114BB3F9000000230F4C2380031E01DB1C4600E05C42B5256C430F4D0C
:201160002D68C5EB84040D4D2D6805EB64140B4D2C602B461B689B121BB28B800023044C7B
:20118000238030BD380400203A0400203C0400203E0400204004002044040020480400200B
:2011A00000B585B000BF1148806940F004000F4988610846806900F00400009000BF00BF96
:2011C000002289140A48F8F77FFA4FF480500190012002900220049001A90548F8F7DAF8D1
:2011E00000200449087005B000BD00000010024000080140C203002010B50446012C0BD100
:201200000C480078A8B9012211030B48F8F75CFA0120084908700CE05CB9064800780128F8
:2012200007D1002201030448F8F74EFA00200149087010BDC20300200008014010B5044641
:2012400019480078012816D1B4F5D16F0FDB17480088401C80B21549088047F230518842F3
:2012600020DD0020114908800F4908701AE000200E49088016E0B4F5BC6F10DA0C48008816
:20128000401C80B20A4908803C280BDDF5F7CEF801200549087000200649087002E0002017
:2012A0000349088010BD0000500400204C0400204E0400209B01002038B5044600203149AA
:2012C0000870F020487008460078C0432E4908702C484078C04348702A4840782B4B0090FF
:2012E000DA79997958792A4B1B78FAF755FB29480078E0B928480068284908602648406826
:2013000048602548806888602348C068C8602448406808612822234801F03EFE042222A1E5
:201320002048083801F038FE01201A49087020A341F205320C214FF4E26001F025FF04B931
:2013400038BDF8F7C7F91C49086000201B49087012E0F8F7BFF918490968401A64280BD9EB
:20136000F8F7B8F91449086014480078401C134908701348F8F7DCF9104800780A28E8DB20
:2013800000BFDDE7CA000020CC000020400700208C030020AE000020A80800200008002018
:2013A0007007002008E80108464C4147000000005245414459000000B0000020B40000206A
:2013C0000406002010B50248F9F7CDF910BD00008812002010B500210B48F9F75BFC0421F2
:2013E0000948F9F757FC08210748F9F753FC00210548F9F7EFF804210348F9F7EBF80821F1
:201400000148F9F7E7F810BD8812002008B508490968C9084FF47A72B1FBF2F1414300910A
:2014200000BF00BF00994A1E00920029F9D108BD000000202DE9F04705460E46174698469C
:20144000F8F748F984490968401A052801D2BDE8F087F8F73FF9804908600FFA88F07F4907
:2014600048807F480088281AC8810846007801287ED1F8F72FF97949C969401AB0F5FA6F19
:2014800006D9F8F727F97549C8610120887601E0744886607148407E01281BD100206F4971
:2014A0004876002405E000206F4921F81400601CC4B2192CF7DB00206C4908806C490860DD
:2014C0006C4908706548408A20B16448408A0002694908606148C0890A2849DB60480560B0
:2014E0005E48807E00286FD15E4886600774C068002869D05B4880895A490989401A00B263
:201500005E4908800846B0F90000002803DD0846B0F9000000E00020584908800846B0F986
:2015200000001E2803DA0846B0F9000000E01E20524908800846008818B94A48007C64280F
:2015400042D049484949098830F8110048490968081A47490860084600684849B1F900106F
:201560000844434908604548008881B23F4800E06FE002880088401C3C4B18803A4820F806
:20158000121018460088192807DB002019460880012038490870314908763548006840B32F
:2015A00034480078012810D1314800684FF47A7148436421484329498989FA225143B0FBA4
:2015C000F1F02649088217E03FE02848008800EB80004100214880894143254800684FF469
:2015E0007A72504364225043B0FBF1F01B49088202E00020194908821C480088A0B9174847
:20160000B0F810901C480068C0EB09201E2190FBF1F019490968084417490860084600689A
:20162000C0F30F200D4948820C48408A002808DD0C4880680949898AB0FBF1F00749C882B6
:2016400003E04FF6FF700549C882064880680549C86000BFFBE60000CC0200209C02002063
:20166000D0020020B40F0020C80F0020BC020020C0020020C4020020C8020020C602002026
:201680002DE9F04104460D4617469846069E002013490860886043F2C82048600020C860AE
:2016A0000DB90846866000200E49087048800520888000208860084684810020C8810882FE
:2016C00048824FF6FF70C88200200876487601208876F7F7FFFF0349C861BDE8F081000050
:2016E000B40F00209C0200202DE9F04106460F4606F00F0000287CD0052FFCD001208649F8
:2017000008700846007E01287CD1002008760846408A82490988884274D07F48408A002836
:201720006CD07D48408A7E490988401A642100FB01F57B48008895FBF0F004B214F11E0F13
:201740005CDBB4F5E47F59DA04F16400744909884843642190FBF1F06F49888271480588E8
:2017600004F164006843642190FBF1F06E4908806C48458804F164006843642190FBF1F0BF
:20178000694948806748858804F164006843642190FBF1F0644988806248C58804F1640019
:2017A0006843642190FBF1F05F49C8805D48858904F164006843642190FBF1F05A49888149
:2017C0005848058904F164006843642190FBF1F0554908815348458904F1640068436421CD
:2017E00090FBF1F0504948810B461022A2214F4802E082E006E001E001F02FFC4648408ABF
:20180000464908804A480078864203D14948007887427AD0042E29D006DC012E0BD0022EA8
:2018200012D0032E46D118E0052E28D0332E2FD0442E3FD135E03C4800883749488239488D
:201840000088374908803BE03748408832494882344840883249088032E0334880882E49FE
:201860004882304880882E49088029E02E48C088294948822B48C0882949088020E02A48F5
:20188000808925494882274880892549088017E02548008920494882224800892049088095
:2018A0000EE0214840891C4948821E4840891C49088005E00020184948821949088000BFE4
:2018C00000BF1548408A154908801348408A124988820846408A002807DD17488068898A34
:2018E000B0FBF1F00C49C88203E04FF6FF700A49C88201200849487607E00020064908708B
:20190000488288824FF6FF70C8820948067009480770BDE8F08100009C020020D60200209A
:20192000D80200200C600108B80800207C030020D4020020D5020020B40F00202DE9F043A0
:2019400099B0064688461546AD10002423E056F8240011A941F8240011A850F82400000E29
:2019600001AA02F8240011A850F82400C0F30741A000401C115411A830F82400C0F307213D
:20198000A000801C115411A810F82410A000C01C1154601CC4B2AC42D9DB56F82590A10098
:2019A00001A8F3F7C9F80746B9EB070008D1AA0001A94046F2F773F8002019B0BDE8F083D3
:2019C0004FF0FF30F9E7000010B5B0F900205243B0F9023003FB03210C4A914214D9091664
:2019E0003939CBB20A4C34F81320B0F9003003FB02F1CB131BB20380B0F9023003FB02F17F
:201A0000CB131BB2438000BF10BD0000400AC139B05C01082DE9F14181B0BDF90400DFF869
:201A20006880B8F9008000FB08F1C913BDF90600DFF85480B8F9028000FB08F2D2130EB289
:201A400017B2F01900B2ADF80000BDF90400DFF83880B8F9028000FB08F3DB13BDF9060041
:201A6000DFF82480B8F9008000FB08F4E4130FFA83FC25B2CCF10000284400B2ADF80200EB
:201A80000098BDE8FC8100004C00002010B504462078012808D10B4B30224C210A4801F01F
:201AA000DCFA002020700AE02078022807D1074B1022EC21044801F0D0FA002020700020B4
:201AC00010BD0000700700207C030020A00700204FF055301F4A106040001F4A10601D4821
:201AE0000168B1F1553F01D0002070471A480168B1F1AA3F01D00020F7E74FF0AA30154A02
:201B000010604008144A106012480168B1F1AA3F01D00020E9E710480168B1F1553F01D068
:201B20000020E2E74FF055300A4A106040000A4A106008480168B1F1553F01D00020D4E795
:201B400005480168B1F1AA3F01D00020CDE70120CBE70000000600201006002001200C49FA
:201B60000968B1F1EE3F00D0002009494968B1F1CC3F00D0002006498968B1F1BB3F00D0E9
:201B800000200349C968B1F1DD3F00D000207047481F002010B5214800780D282FD2DFE819
:201BA00000F0070A0D101316191C1F2225282B00F1F704FB24E0F1F735FB21E0F1F771FB98
:201BC0001EE0F1F7B3FB1BE0F1F7F6FB18E0F1F73AFC15E0F1F77EFC12E0F1F7C2FC0FE0A9
:201BE000F1F707FD0CE0F1F74DFD09E0F1F78EFD06E0F1F7CFFD03E0F1F710FE00E000BF6D
:201C000000BF06480078401C04490870084600780C2801DD0020087010BD0000CC040020F1
:201C200010B5F1F7CBFAF1F7FDFAF1F73AFBF1F77DFBF1F7C1FBF1F706FCF1F74BFCF1F731
:201C400090FCF1F7D6FCF1F71DFDF1F75FFDF1F7A1FDF1F7E3FD10BD10B53B480068B0F18C
:201C6000AA3F70D138480068384909684840401C002866D136490860C043364908603448D0
:201C80000068801C32490860FFF784FF31480068801E304908602E4800680D302C4908608C
:201CA000FFF75CFF08B9F5F741F92A4800680D3828490860264800680B302549086000F01D
:201CC000C5FC044634B1012C0AD0032C04D0042C05D100E007E006E0F5F728F903E000BFA8
:201CE000F5F724F900BF00BF1A4800680B381949086017480068C01C1549086000F044F8F1
:201D000008B9F5F713F913480068C01E114908600F480068401D0E490860FFF7D9FE08B93E
:201D2000F5F704F90B480068401F0A490860222003F080FA08B9F5F7F9F8002002490860C5
:201D400001E0F5F7F3F810BD101B0020341B0020001B0020241B002010B500F047FC00F0C2
:201D600055FC00F001F810BD4FF0EE30054908604FF0CC3048604FF0BB3088604010C860DC
:201D800070470000481F0020F0B55527552F01D00020F0BDAA27AA2F01D00020F9E74FF008
:201DA0005531B1F1553F01D00020F2E74FF0AA31B1F1AA3F01D00020EBE74FF47A714A00BD
:201DC0008C1840F6B830844201D00020E1E74FF0FF3102228C18012C01D00020D9E74FF46A
:201DE0007A73F94D5E1916F57A7F01D00020D0E76FF0004301255E19B6F1004F01D0002067
:201E0000C7E76FF0004302255E19981C864201D00020BEE76FF0004303255E19D81C8642C5
:201E200001D00020B5E74FF4FA614A108C1AB4F57A7F01D00020ACE74FF4FA614A1C8C1AA7
:201E4000601C08B10020A4E7002101228C1A601C08B100209DE74FF47A735D005E1B16F5CE
:201E60007A7F01D0002094E7002301255E1B701C08B100208DE74FF0004301255E1B581ECB
:201E8000864201D0002084E74FF47A71491C0846814201D000207CE74FF0FF31491C09B198
:201EA000002076E70021491C012901D0002070E74FF47A735B1C1846834201D0002068E7A3
:201EC00000235B1C012B01D0002062E76FF000435B1CB3F1004F01D000205AE74FF0004342
:201EE0005B1C1846834201D0002052E74FF47A71491E0846814201D000204AE70021491ECE
:201F0000481C00B145E74FF0FF31491E881C00B13FE74FF47A735B1E1846834201D0002072
:201F200037E74FF000435B1E1846834201D000202FE76FF000435B1E1846834201D000202F
:201F400027E700235B1E581C00B122E764210A2201FB02F4B4F57A7F01D0002019E76FF014
:201F60007041112201FB02F49848844201D000200FE74FF0FF31012201FB02F4601C08B145
:201F8000002006E76421002201FB02F40CB10020FFE64FF47A710A22B1FBF2F4642C01D08C
:201FA0000020F6E601210A22B1FBF2F40CB10020EFE600210A22B1FBF2F40CB10020E8E609
:201FC0004FF47A710022B1FBF2F40CB10020E0E64FF0FF310122B1FBF2F4601C08B1002003
:201FE000D7E602214C00042C01D00020D1E602210C02B4F5007F01D00020CAE60221CC07ED
:202000000CB10020C5E64FF6FF714C084810844201D00020BDE64FF6FF710C0AFF2C01D0B6
:202020000020B6E64FF6FF71CC0F0CB10020B0E6012109B90020ACE6002109B10020A8E6C2
:20204000FF2109B90020A4E664210A22914201D800209EE664216422914201D9002098E69D
:202060000A216422914201D9002092E64FF0FF310022914201D800208BE66FF00043DD0716
:20208000AB4201DC002084E60A216422914201D300207EE664216422914201D2002078E6E1
:2020A00064210A22914201D2002072E600214A1E914201D300206CE64FF000435D1EAB42C5
:2020C00001DB002065E664210A22914201D200205FE664216422914201D2002059E60A21C2
:2020E0006422914201D3002053E64FF0FF310022914201D200204CE66FF00043DD07AB425E
:2021000001DA002045E60A216422914201D900203FE664216422914201D9002039E664217A
:202120000A22914201D8002033E600214A1E914201D900202DE64FF000435D1EAB4201DD5D
:20214000002026E664216422914201D0002020E64FF0FF310A46914201D0002019E60021DB
:202160000022914201D0002013E64FF000431D46AB4201D000200CE600230025AB4201D0C5
:20218000002006E66FF000431D46AB4201D00020FFE564216422914201D00020F9E54FF080
:2021A000FF310A46914201D00020F2E500210022914201D00020ECE54FF000431D46AB425A
:2021C00006D00020E5E5000030F8FFFFEFFFFF0F00230025AB4201D00020DAE56FF0004396
:2021E0001D46AB4201D00020D3E50121002221B9022904D0032906D103E0921C04E0121D22
:2022000002E0083200E000BF00BF022A01D00020BFE502210022012904D0022904D0032915
:2022200006D103E0921C04E0121D02E0083200E000BF00BF042A01D00020AAE503210022B5
:20224000012904D0022904D0032906D103E0921C04E0121D02E0083200E000BF00BF082A2E
:2022600001D0002095E504210022012904D0022904D0032906D103E0921C04E0121D02E026
:20228000083200E000BF00BF0AB1002081E50021002211B10AB100207BE501B90AB1002090
:2022A00077E50021012211B10AB1002071E511B90AB900206DE50121012201B10AB90020B2
:2022C00067E511B90AB9002063E50121FF2201B10AB900205DE511B90AB9002059E5002197
:2022E000FF2211B10AB1002053E511B90AB900204FE54FF055310A4681EA02040CB10020A4
:2023000047E54FF055314A0081EA0204601C08B100203EE50021002281EA02040CB1002008
:2023200037E54FF0FF310A4681EA02040CB100202FE500214A1E81EA0204601C08B1002011
:2023400027E54FF05531CC43B4F1AA3F01D000201FE5E443B4F1553F01D0002019E50021AA
:20236000CC43601C08B1002013E5E4430CB100200FE501200DE5000008B500BF71488069D8
:2023800040F004006F4988610846806900F00400009000BF00BF00BF0846806940F0080001
:2023A00088610846806900F00800009000BF00BF00BF0846806940F01000886108468069A1
:2023C00000F01000009000BF00BF00BF0846806940F0200088610846806900F020000090E9
:2023E00000BF00BF5848F4F7F1FD08B9002008BD5648F4F7EBFD08B90020F8E75448F4F788
:20240000E5FD08B90020F2E75248F4F7DFFD08B90020ECE74B48806920F004004949886100
:202420000846806920F0080088610846806920F0100088610846806920F020008861464846
:20244000F1F7F2FE00BF3F48C06940F000703D49C8610846C06900F00070009000BF00BF01
:202460003E48F2F723FB08B90020C0E73548C06920F000703349C86100BF0846406940F096
:20248000010048610846406900F00100009000BF00BF3348F2F7F0FF08B90020A7E7294869
:2024A000406920F001002749486100BF0846806940F4007088610846806900F4007000909B
:2024C00000BF00BF00BF0846806940F4806088610846806900F48060009000BF00BF214809
:2024E000F1F7BAFD08B9002081E71F48F1F7B4FD08B900207BE71348806920F4007011498F
:2025000088610846806920F48060886100BF0846806940F4006088610846806900F40060C0
:20252000009000BF00BF114801F0DFFA08B900205DE70448806920F4006002498861012047
:2025400055E700000010024000080140000C014000100140001401400000014000640040CC
:20256000080002400024014000280140002C014010B5002419480068194909684840401C6D
:2025800048BB164800681749884210D316490846F1F77CF9012801D1042400E003241148D8
:2025A0004B380E490860C0430D49086014E00E490A480068F1F76AF901280AD1074800680D
:2025C00010300649086008460068C0430449086002E0032400E00124204610BD0005002030
:2025E000040500207B000020E004002004480549086008460068C0430349086070470000ED
:2026000030000020000500200405002010B50A480A490860C0430A4908600A480A4908607F
:202620000846F6F79CFB08480068806840F0010005490968886010BD003000081C1B0020F4
:20264000401B002000300240D404002010B502241F4800681F4909684840401C002834D1F1
:202660001B4800681C49884223D2002006E01849096851F82010194A1160401C18498908F8
:20268000174A9209B1FBF2F18142F0D814498908134A9209B1FBF2F10D4A126802EB81016F
:2026A0000B4A116011460968C9430A4A116000240CE00A48006808490968884201D104246B
:2026C00000E00324FFF7A2FF00E00124204610BD1C1B0020401B0020C08301080030024094
:2026E000C053010070B50A2050490870F7F734F800F03EFF00204E490860C0434D490860FF
:202700004B480068801C4A490860FFF789FA49480068801E47490860F0F704FD0C2043497F
:202720000870434800680B304149086042484349086008460068806840F00100096888605B
:202740003E48F6F70CFB002405E03D4951F8240039490860641C3B48B4EB900FF5D3364892
:20276000056839480068854201D0F4F7DFFB314800680B382F4908600E202C4908702C4813
:202780000068C01C2A490860FFF7FEFA08B9F4F7CDFB28480068C01E26490860102023498F
:2027A000087023480068401D21490860FFF790F908B9F4F7BBFB1F480068401F1D490860C2
:2027C00012201A4908701A480068C01D18490860FFF7D2FD08B9F4F7A9FB1420134908705F
:2027E000FFF7CAFD08B9F4F7A1FB12480068C01F1049086016200D4908701C2002F01AFD29
:2028000008B9F4F793FB1820084908704FF400510804F1F7B4F808B9F4F788FB00F012FF19
:20282000AA2005490871F0F761FC70BDD0040020001B0020241B002000300240D40400209E
:2028400000300008C0530100C083010810B5124800780A281EDB00200F4908704FF0AA3015
:202860000E49086040080E49086072B6FFF780FE044662B634B1012C08D0032C05D0042C76
:2028800002D100E005E004E000BF00BFF4F74EFB00BF00BF10BD000059000020101B0020FB
:2028A000341B0020002107E041F64C5100BF0A00A1F1010399B2FAD10200A0F1010398B277
:2028C000F2D17047002106E0072100BF0A00A1F1010399B2FAD10200A0F1010398B2F3D135
:2028E000704770472DE9F143BDF9000044F2F30100FB01F9BDF902004FF416514843C0F1AD
:202900000008444608EB09004710A8EB09004610002F0FDA002E03DA0520F749088018E0D8
:20292000002C03DC0420F449088012E00320F24908800EE0002E03DB0220EF49088008E007
:20294000002C03DC0620EC49088002E00120EA4908800020E9490870E748008807287BD2CE
:20296000DFE800F07A044D97E0FCFB0004F51650801B4FF4966101EBA040E1490880084667
:20298000008800EB6640488008464088A0EB6440888008460088C0F5166080B2E22803DDEC
:2029A00040F65F10C88029E0D5480088D4494988401A85B2B5F58B7F05DBD148008833385D
:2029C000CF49C8801AE0CE480088C0F5166080B28A2813DDCA480088E230C949C8800846AC
:2029E000C088B0F5166F09DB0120C4490870C448C088C0F59650401EC149C88074E107F5EB
:202A00001650801B4FF4966101EBA040BC4908800846008800EB6640488008460088A0EB92
:202A20006740888008464088C0F5166080B2E22803DD40F65F10C8802AE0B1484088B049D9
:202A40000988401A85B2B5F58B7F06DBAC4840883338AB49C8801BE045E1A9484088C0F5CD
:202A6000166080B28A2813DDA5484088E230A449C8800846C088B0F5166F09DB01209F4963
:202A800008709F48C088C0F59650401E9C49C8802AE1C4F5165038444FF4966101EBA040BD
:202AA0009749088008460088A0EB674088800846808800EB6440488008464088C0F51660B0
:202AC00080B2E22803DD40F65F10C88029E08C4840888B498988401A85B2B5F58B7F05DB3E
:202AE0008748408833388649C8801AE084484088C0F5166080B28A2813DD81484088E2308D
:202B00007F49C8800846C088B0F5166F09DB01207A4908707A48C088C0F59650401E7849E1
:202B2000C880E1E004F51650801B4FF4966101EBA040734908800846008800EB6640488019
:202B400008464088A0EB6440888008468088C0F5166080B2E22806DD01E078E02EE040F60B
:202B60005F10C88029E06648808865494988401A85B2B5F58B7F05DB614880883338604976
:202B8000C8801AE05E488088C0F5166080B28A2813DD5B488088E2305949C8800846C08809
:202BA000B0F5166F09DB0120544908705448C088C0F59650401E5249C88095E007F516503A
:202BC000801B4FF4966101EBA0404D4908800846008800EB6640488008460088A0EB6740FF
:202BE000888008468088C0F5166080B2E22803DD40F65F10C88029E041488088404909888F
:202C0000401A85B2B5F58B7F05DB3D48808833383B49C8801AE03A488088C0F5166080B2EA
:202C20008A2813DD36488088E2303549C8800846C088B0F5166F09DB012030490870304866
:202C4000C088C0F59650401E2D49C8804CE0C4F5165038444FF4966101EBA04028490880AF
:202C600008460088A0EB674088800846808800EB6440488040F65F10C88008460088C0F51F
:202C8000166080B2E22803DD40F65F10C88029E01B4800881A498988401A85B2B5F58B7F08
:202CA00005DB1748008833381549C8801AE014480088C0F5166080B28A2813DD104800887F
:202CC000E2300F49C8800846C088B0F5166F09DB01200A4908700A48C088C0F59650401E1F
:202CE0000749C88000E000BF00BF0448007848B9002000F005FB08E0340000203600002077
:202D000038000020022000F0FBFA40F64C100949C880088800F0DCFA0649488800F0DEFAEB
:202D20000449888800F0E0FA0249C88800F0E2FABDE8F883380000202DE9F04104460025D7
:202D400000260027F3F7B2FBA84618E000BF334800780128FBD100203049087030480088F1
:202D600005442F48408806442D48808807440C212C48F7F76FFF08F101001FFA80F8B8F188
:202D80000A0FE3DB0A20B5FBF0F0274908800A20B6FBF0F048800A20B7FBF0F08880084615
:202DA000008846F2A81188421DDB1F48008849F64041884217DC1C48408846F2A811884285
:202DC00011DB1948408849F6404188420BDC1648808846F2A811884205DB1348808849F6CA
:202DE0004041884216DD206820F4802000F58020206006200D4948800846F3F741FE002069
:202E00000B4908700B484089401C0A494881022009490870F3F74AFBBDE8F081EC03002012
:202E2000E003002088120020F20300207C100020EC020020A00700205601002008B50020EB
:202E4000009053480088072870D2DFE800F0933362630405320000BF4E480088404201B2BF
:202E600011F5004F04DA4FF40040ADF8000009E0B1F5004F04DB47F6FF70ADF8000001E008
:202E8000ADF8001043484088404201B211F5004F04DA4FF40040ADF8020009E0B1F5004FBA
:202EA00004DB47F6FF70ADF8020001E0ADF8021061E000BF37484088404201B211F5004F77
:202EC00004DA4FF40040ADF8020009E0B1F5004F04DB47F6FF70ADF8020001E0ADF8021042
:202EE0002C488088BDF80220801A01B2B1F5004F04DB47F6FF70ADF8000009E011F5004FCF
:202F000004DA4FF40040ADF8000001E0ADF8001031E000BF1F480088404201B2B1F5004F2C
:202F200005DB47F6FF70ADF800000AE022E011F5004F04DA4FF40040ADF8000001E0ADF893
:202F4000001014488088BDF80020801A01B211F5004F04DA4FF40040ADF8020009E0B1F5EF
:202F6000004F04DB47F6FF70ADF8020001E0ADF8021000E000BF00BFBDF900000011ADF86E
:202F80000000BDF902000011ADF80200009808BD34000020F80300202DE9F043C1B0814674
:202FA0000D4616463046F11706EB9171C1F38707002414E015F824000106A000401C285CDF
:202FC00001EB0041A000801C285C01EB0021A000C01C285C08444DF82400601CC4B2BC4252
:202FE000E8DB31462846F1F7A7FD80464DF827807A1C69464846F3F741FE41B0BDE8F083E6
:203000002DE9F04190B080460D4616463046F11706EB9171C1F38707002414E0A000C01C6D
:20302000285C0106A000801C285C01EB0041A000401C285C01EB002015F8241008444DF8BA
:203040002400601CC4B2BC42E8DB3A4669464046F3F714FE10B0BDE8F0812DE9F8438146FA
:203060000D4616461F46002000908046002420E02819C1B26A464846F3F74EFB401C18B950
:203080004FF0FF30BDE8F883385D9DF8001088420DD0385D00902819C1B29DF800204846A5
:2030A000F3F790FB401C10B94FF0FF30EAE7601CC4B2B442DCDB31463846F1F725FD8046D3
:2030C0004FEA28200090A819C1B29DF800204846F3F778FB401C10B94FF0FF30D2E708F0C7
:2030E000FF000090A819401CC1B29DF800204846F3F768FB401C10B94FF0FF30C2E70020C5
:20310000C0E7000070B505460C4664BB1A4800691A4948600B4630224C212846FFF79DFF41
:20312000401C28B9154B30224C212846FFF795FF11480068124908600F48406848600E48BA
:20314000806888600C48C068C8600B461022D6212846FFF782FF401C28B9094B1022D621E2
:203160002846FFF77AFF064800680A21B0FBF1F004494882002070BD0008002070070020E2
:20318000A8080020380600202DE9F04706468846174699460025FCB255201F490870AA206C
:2031A0004870084680F80280A01CC870380A08710846447122464946801DF0F770FC552001
:2031C00016490870AA20487030128870CE70221D1149891C1148001DF0F761FC04F1080128
:2031E0000E48F1F7A9FC0546280EA11D0A4A5054C5F30741E01D1154C5F30721401C1154B2
:20320000401C1554F021401C1154421C02493046F1F7AEFBBDE8F087C60A0020C50B00206B
:203220002DE9F047CCB081460E4690461F46DDF850A1982126A8F0F74BFC98216846F0F7A6
:2032400047FC0025FCB255208DF89800AA208DF89900300A8DF89A00F0B28DF89B008DF83E
:203260009C80A01CC0B28DF89D00380A8DF89E008DF89F402246514628A8F0F710FC04F162
:20328000080226A96846F0F70AFC04F108016846F1F752FC0546280E04F1080126AA5054E5
:2032A000C5F3074104F109001154C5F30721401C1154401C1554F021401C1154401CC2B2A3
:2032C00026A9484601F059F84CB0BDE8F087000001490968486370478812002001490968A5
:2032E000886370478812002001490968C86370478812002001490968086470478812002083
:2033000008490968096A21F40051064A1268116204490968096A41EA0031024A126811620F
:2033200070470000881200202DE9F04705460C4616461F46DDE90889F6F7CCF91949096895
:20334000401A32282BD3F6F7C5F91649086005FB06F090FBF7F000FB08F000EBC000000142
:2033600042F2107190FBF1F0208020880E49096808440D4908600D480078401C0B4908701D
:203380000846007808280ADB0020087006480068C0F3CF00A9F80000002003490860BDE868
:2033A000F0870000540300205C0300205803002070B504460D461646F6F78CF924490968B7
:2033C000401A322841D3E07828B9F6F783F9214908600120E070F6F77DF91E490968401AAB
:2033E000B0F57A6F04D90020A0704FF6FF70A060208980B24FF6FF71884202D10020A07021
:2034000001E00120A070A078012812D1A06810B94FF0FF30A0604FF4B4707043A168B0FB69
:20342000F1F0208020880A220B49FDF759FC288007E00020208028800A210748F0F77BFFC8
:2034400070BDF6F747F90249086000BFF8E7000060030020640300204811002000B585B054
:2034600000BF1048806940F020000E4988610846806900F02000009000BF00BF04200190B2
:20348000094802900120039001A90848F5F782FF002202210820F6F7ECF90820F6F7DCF905
:2034A00005B000BD0010024000001110001401402DE9F04104460D4617461E46F6F70AF93D
:2034C00028490968401A32284AD3E07828B9F6F701F9254908600120E070F6F7FBF8224987
:2034E0000968401A4FF47A6191FBF6F1884201D90020A070A078012822D1A06810B94FF058
:20350000FF30A0604FF4B4707843B0FBF6F0A168B0FBF1F0208020880A221449FDF7E0FB94
:203520002880F6F7D7F86168411AA068B1EB400F12D940F20E41A0684843800AA0600BE09C
:203540000020208028800A210848F0F7F4FE4FF0FF30A060BDE8F081F6F7BCF801490860D8
:2035600000BFF7E74C030020500300203411002010B594B009200A904FF480300B900020ED
:203580000C9001200E90109002201190C10312914FF4E01113910AA8F6F74AFC18B1CD2192
:2035A0001AA001F0C9FC0F20059002200690002007904FF48060089000200990022105A824
:2035C000F6F7F4FA18B1DB2110A001F0B5FC022001908003039001A8F6F750FA18B1E22184
:2035E0000AA001F0A9FCF6F7B3FB4FF47A71B0FBF1F42046F6F748FF0420F6F739FE00222E
:203600001146501EF6F735F914B010BD2E2E5C53656C6654657374557365725C7372635FB5
:203620006D6964646C6577617265735C73746D33326678785F535455737461727475702EF2
:203640006300000010B590B00220069001200A9010200B9000200D9006A8F6F7E9FB20B1B7
:2036600040F2031114A001F067FC0F2001900020029003904FF4806004900020059000216A
:2036800001A8F6F793FA20B140F211110AA001F053FCF6F75DFB4FF47A71B0FBF1F420468F
:2036A000F6F7F2FE0420F6F7E3FD00221146501EF6F7DFF810B010BD2E2E5C53656C66546E
:2036C000657374557365725C7372635F6D6964646C6577617265735C73746D333266787800
:2036E0005F535455737461727475702E6300000010B5F6F725F8F6F7E1FE03480078401C11
:203700000149087010BD00005900002010B594B009200A904FF480300B9000200C9001206A
:203720000E90109002201190C10312914FF4E01113910AA8F6F77CFB20B14FF4BE711CA034
:2037400001F0FAFB0F20059002200690002007904FF48060089000200990022105A8F6F71F
:2037600025FA20B14FF4C57111A001F0E5FB022001908003039001A8F6F780F920B140F283
:2037800091110BA001F0D8FBF6F7E2FA4FF47A71B0FBF1F42046F6F777FE0420F6F768FD53
:2037A00000221146501EF6F764F814B010BD00002E2E2F436F72652F5372632F6D61696E09
:2037C0002E6300001148006840F001000F490860084640680E4908400C494860084600685E
:2037E0000C490840094908600846006820F4802008600846406820F4FE0048604FF41F008E
:203800008860C8030449086070470000001002400000FFF8FFFFF6FE08ED00E010B502486A
:20382000F7F74AF810BD00008812002000220268184B984208D0B0F1804F05D0164B9842B0
:2038400002D0164B984203D122F070024B681A43104B984208D0B0F1804F05D00E4B98426E
:2038600002D00E4B984203D122F44072CB681A4322F080024B691A4302608B68C3620B6885
:203880008362044B984201D10B6903630123436170470000002C01400004004000080040F6
:2038A00030B50023012404FA01F3046A9C430462046A02FA01F52C43046230BD30B500230C
:2038C000042404FA01F3046A9C430462046A02FA01F52C43046230BD30B50C4600218168B8
:2038E00021F47F4142EA032525432943816030BD0A460021816821F0700142F00703194389
:203900008160704730B5002400220023056A25F001050562026A4368846924F0700424F030
:2039200003040D682C4322F002028D682A430D4DA84206D100BF22F00802CD682A4322F07A
:203940000402084DA84207D123F4807323F400734D692B438D692B43436084614D68456349
:20396000026230BD002C014030B5002400220023056A25F010050562026A4368846924F41F
:20398000E04424F440740D6844EA052422F020028D6842EA05120F4DA84207D100BF22F010
:2039A0008002CD6842EA051222F04002094DA84209D123F4806323F400634D6943EA8503C0
:2039C0008D6943EA8503436084614D688563026230BD0000002C014030B50024002200230B
:2039E000056A25F480750562026A4368C46924F0700424F003040D682C4322F400728D689B
:203A000042EA05220E4DA84207D100BF22F40062CD6842EA052222F48062094DA84209D165
:203A200023F4805323F400534D6943EA05138D6943EA05134360C4614D68C563026230BD06
:203A4000002C014030B5002200230024056A25F480550562036A4468C26922F4E04222F455
:203A600040720D6842EA052223F400538D6843EA0533074DA84204D124F480444D6944EA35
:203A800085144460C2614D680564036230BD0000002C014030B50B46144600210022026AAA
:203AA000056A25F001050562816921F0F00141EA041122F00A021A438161026230BD30B556
:203AC0000B46144600210022056A25F0100505628169026A21F4704141EA043122F0A002C8
:203AE00042EA03128161026230BD0146002240F205100860086882B240F20510824201D0BA
:203B00000020704740F28A200860086882B240F28A20824201D00020F3E70020086045F2BC
:203B200055504860486882B245F25550824201D00020E6E742F6A8204860486882B242F632
:203B4000A820824201D00020DBE70020486045F255508860886882B245F25550824201D005
:203B60000020CEE74AF6A2208860886882B24AF6A220824201D00020C3E70020886045F2C2
:203B80005550C860C86882B245F25550824201D00020B6E742F6AA20C860C86882B242F600
:203BA000AA20824201D00020ABE70020C86045F255508861886982B245F25550824201D051
:203BC00000209EE74AF6AA208861886982B24AF6AA20824201D0002093E70020886145F2AF
:203BE0005550C861C86982B245F25550824201D0002086E74AF6AA20C861C86982B24AF6BC
:203C0000AA20824201D000207BE70020C86141F255500862086A82B241F25550824201D025
:203C200000206EE742F6AA200862086A82B242F6AA20824201D0002063E70020086245F23B
:203C400055504862486A82B245F25550824201D0002056E74AF6AA204862486A82B24AF687
:203C6000AA20824201D000204BE70020486245F255508862886A82B245F25550824201D06C
:203C800000203EE74AF6AA208862886A82B24AF6AA20824201D0002033E70020886245F2AB
:203CA0005550C862C86A82B245F25550824201D0002026E74AF6AA20C862C86A82B24AF657
:203CC000AA20824201D000201BE70020C86255200863086B82B2552A01D0002011E7AA2060
:203CE0000863086B82B2AA2A01D0002009E70020086345F255504863486B82B245F2555028
:203D0000824201D00020FCE64AF6AA204863486B82B24AF6AA20824201D00020F1E60020BA
:203D2000486345F255508863886B82B245F25550824201D00020E4E64AF6AA208863886BA7
:203D400082B24AF6AA20824201D00020D9E60020886345F25550C863C86B82B245F255505C
:203D6000824201D00020CCE64AF6AA20C863C86B82B24AF6AA20824201D00020C1E60020BA
:203D8000C86345F255500864086C82B245F25550824201D00020B4E64AF6AA200864086CF3
:203DA00082B24AF6AA20824201D00020A9E60020086441F215508864886C82B241F21550B1
:203DC000824201D000209CE640F60A208864886C82B240F60A20824201D0002091E600208C
:203DE0008864086101208CE62DE9F04104460E4690461F4630480078012812D12F480178CF
:203E00000078401C2D4A10702D4820F811601046007832281CDB00202749087011460870E3
:203E200016E0322226493046FCF75AFF05462088A84209DDF5F74EFC22490968401AB0F533
:203E40007A7F05D9258003E0F5F744FC1D49086040F6340008FB00F0642190FBF1F0C0F506
:203E600080502188884203DBF5F734FC16490860F5F730FC14490968401A42F2107188427F
:203E800017D9386820F040004030386003200F494880208888800846F2F7F2FD00200C49AC
:203EA00008700C48808A401C0A49888201200A490870BDE8F0810000690300206A03002058
:203EC00074110020700300206C0300207C100020EC02002070070020560100202DE9F04706
:203EE00004460F46E7824FF0090841462046F3F779F9C01B0FFA80F919F1780F2ADDB9F182
:203F0000780F27DA002606E0701C34F8100024F81600701CC6B2A8F10100B042F4DC24F897
:203F2000107041462046F3F7DDF905B2608AA84200DA658241462046F3F7E5F905B2A08A72
:203F4000A84200DDA582064B18227E210548FFF784F802E0002004490870BDE8F0870000A7
:203F60005C1100207C0300206803002003B50246002006E002EB4001BDF804300B80411C85
:203F8000C8B20C28F6D30CBDF0B504460D46671B39B2178892F802C007FB0CF74FF0640C93
:203FA00097FBFCF7BBB29778C7EBC70707EB4706002901DA002014E0994206DA4FF4B677FE
:203FC0004F4397FBF3F7B8B20BE0CF1A4FF4D96C07FB0CF7A6EB030C97FBFCF707F5B677BA
:203FE000B8B2F0BD08B5024602F5004081B20846CB1701EB936399114FF6FE70014001F496
:20400000407038B3B0F5807F36D0B0F5007F03D0B0F5407F40D10DE0C8B2214B33F81000E1
:20402000ADF80200C8B2C0F1FF0033F81000ADF8000032E0C8B2C0F1FF00194B33F81000F4
:20404000ADF80200C8B233F81000404200B2ADF8000022E0C8B2124B33F81000404200B2E3
:20406000ADF80200C8B2C0F1FF0033F81000404200B2ADF8000010E0C8B2C0F1FF00084BEE
:2040800033F81000404200B2ADF80200C8B233F81000ADF8000000E000BF00BF009808BDF5
:2040A0003E5D010870B505466C6A0020E085E0842046F6F710FF70BD2DE9F04106460D46B8
:2040C0001446002025490870F5F704FB2349486005F0FF08A5F50040083830B1A0F6FA708A
:2040E000B8B1B0F5545F2DD108E0424621461C48EFF7D5FC00201B4908702BE023462A462F
:20410000314640F21560FFF73FF801201649087020E02178627801EB02218FB2002007E092
:20412000124931F81010B94200DD03E0411CC8B20B28F5D300BF00F14901CAB20C4981F80A
:20414000252007E023462A46314640F21560FFF71BF800BF00BFBDE8F08100006C01002012
:20416000600100206A0100205D000020346001085806002010B50A46C37893421EDBC36852
:204180001B68DB6823F02003C4682468E360C3789B1AC370C3681B68DB6843F02003C46892
:2041A0002468E360114683780B4499B203788B4202DC0378CB1A99B281701BE0C3681B68D9
:2041C000DB6823F02003C4682468E360C1780023C370C3681B68DB6843F02003C4682468DD
:2041E000E3608378194403788B4202DC0378CB1A99B2817010BD0168C96821F4907102687B
:20420000D1600168496921F0010102685161202180F83A10704710B504462068C06820F09A
:2042200040002168C860202084F839002046F6F798FF002010BD00BFC27803789A42FBD0A6
:20424000C2681268D26822F08002C3681B68DA60C2788AB9C26812681268C2F3C0125AB1D7
:20426000C26812685160C2681268D26842F08002C3681B68DA60704743788268D154427834
:20428000521CD2B2427003789A4201D100224270C278521CC270C2681268D26842F0800211
:2042A000C3681B68DA6000BFE5E710B502460B461946D4789C4209DB94780C44A1B2147885
:2042C0008C4204DC14780C1BA1B200E000219468605C10BD70B5044694F83A0022284AD10A
:2042E000A068B0F5805F13D1A56A206940B920684068C0F308002880A06A801CA06219E089
:2043000020684068C0B22880A06A401CA06211E0206938B920684068C1B2A26A501CA06263
:20432000117007E02068406800F07F01A26A501CA0621170E08D401E80B2E085C8B920680F
:20434000C06820F020002168C8602068C06820F480702168C8602068406920F00100216824
:204360004861202084F83A002046F6F7F9FE002070BD0020FCE70220FAE7F0B507460D46BC
:204380001646002405E0295D3846FFF754FF601CC4B2B442F7DBF0BD2DE9F041044600254E
:2043A0002068006920F44050E1680843216808612169A06808436169084305432068C068F8
:2043C00041F20C61884328432168C8602068406920F44070A1690843216848615F492068AA
:2043E00088425CD1F5F7CAFC00EBC00101EB001061688900B0FBF1F6F5F7C0FC00EBC00134
:2044000001EB001061688900B0FBF1F06421B0FBF1F000EBC00101EB0010A6EB80003221A5
:2044200001EB00106421B0FBF1F000F0F006F5F7A5FC00EBC00101EB001061688900B0FB57
:20444000F1F06421B0FBF1F006EB0016F5F796FC00EBC00101EB001061688900B0FBF1F758
:20446000F5F78CFC00EBC00101EB001061688900B0FBF1F06421B0FBF1F000EBC00101EB99
:204480000010A7EB8000322101EB00106421B0FBF1F000F00F003044216888605BE0F5F78F
:2044A0005DFC00EBC00101EB001061688900B0FBF1F6F5F753FC00EBC00101EB001061686B
:2044C0008900B0FBF1F06421B0FBF1F000EBC00101EB0010A6EB8000322101EB0010642129
:2044E000B0FBF1F000F0F006F5F738FC00EBC00101EB001061688900B0FBF1F06421B0FB74
:20450000F1F006EB0016F5F729FC00EBC00101EB001061688900B0FBF1F7F5F71FFC00EB23
:20452000C00101EB001061688900B0FBF1F06421B0FBF1F000EBC00101EB0010A7EB800015
:20454000322101EB00106421B0FBF1F000F00F00304421688860BDE8F08100000038014088
:20456000014691F8390021282CD18868B0F5805F0FD10A6A1088C0F308000B685860086935
:2045800018B9086A801C086209E0086A401C086205E00B6A581C086218780B685860C88C6A
:2045A000401E80B2C88458B90868C06820F080000B68D8600868C06840F040000B68D86088
:2045C000002070470220FCE710B5054800F00EF8044800F040F80448F6F77EFC10BD000003
:2045E000AC040020BC040020C01A002008B5C26812681268C2F3401262B3C26812685268BC
:20460000D1B2C268126812680022B2B943788268D1544278521CD2B2427003789A4201DB11
:2046200000224270C278521CD2B2C27003789A4203DD0278C2700122027100BF002200925C
:20464000C268126812680092C26812685268009200BF00BF08BDC16809680968C1F3C011E7
:2046600039B3C1680968C96801F0800109B36FF08001C26812681160C17891B1C178491E45
:20468000C17082788168895CC268126851608178491CC9B28170027891420ADB00218170BE
:2046A00007E0C1680968C96821F08001C2681268D160704710B50248F3F74CFF10BD000019
:2046C0007C18002010B54FF4FA71024800F004F810BD0000AC0400202DE9F34F83B00398BA
:2046E000C0780D2873DB00210398FFF7DEFD01906B490198087001210398FFF7D6FD8146CF
:20470000674981F80190019855287DD1B9F1AA0FFBD102210398FFF7C8FD6149887003210D
:204720000398FFF7C2FD5E49C87004210398FFF7BCFD06465A490E71112E03D0162E01D046
:204740000C2E7DD105210398FFF7AFFD07465448477107210398FFF7A8FD834606210398E4
:20476000FFF7A3FD0BEB00201FFA80F84FEA18204B49887181F8078007210398FFF795FDB3
:204780000446381B02287AD10398C17807F10B0081421DDA43480078012806D1F4F79AFFEF
:2047A0004149086000203F490870F4F793FF3E490968411A0498814206D9F4F78BFF3A49E1
:2047C000086001203749087005B0BDE8F08F64E001203449087000250FE005F10800C1B2A0
:2047E0000398FFF762FD314948550846415D05F108002B4A1154681C85B2A542EDDB04F18F
:204800000800C1B2039800E043E0FFF74EFD4FEA006B04F10900C1B20398FFF746FD0BEB5F
:20482000004B04F10A00C1B20398FFF73EFD0BEB002B04F10B00C1B20398FFF736FD00E0B7
:2048400022E05844029004F108011548F0F774F982460298B0EB0A000CD1144A414630463A
:20486000FFF72AFC07F10B00C1B20398FFF782FCAAE704E001210398FFF77CFC0DE00121E8
:204880000398FFF777FC08E001210398FFF772FC03E001210398FFF76DFC00BF94E70000D2
:2048A0005A0D0020A00100209C010020C40C0020012806D002282AD003285FD004287DD10C
:2048C00084E05749574A13680B6053684B6092688A60554A1368CB6053680B6192684A61F2
:2048E000524A13688B615368CB6192680A620A464F490B6853624B6893628968D1624D49F6
:204900000B68D3634B6813648968516485E0444A49490B6813604B68536089689160114614
:20492000464A1368CB6053680B6192684A61444A13688B615368CB6192680A62414A13682D
:204940004B6253688B629268CA620A463E490B6813634B6853638968916311463B4A136877
:20496000CB6353680B6492684A640A4638490B6893644B68D364896811654EE0284A35498D
:204980000B6813604B6853608968916032490B68D3604B6813618968516130490B6893611E
:2049A0004B68D3618968116211462D4A13684B6253688B629268CA622A4A00E02CE013680D
:2049C000CB6353680B6492684A6426E01449264A13680B6053684B6092688A60234A1368EC
:2049E000CB6053680B6192684A61214A13688B615368CB6192680A621E4A13684B62536856
:204A00008B629268CA620A461B490B68D3634B6813648968516400E000BF00BF7047000041
:204A2000540800204A60010856600108626001086E6001087A600108866001089260010819
:204A40009E600108AA600108B6600108C2600108CE600108DA600108E6600108F2600108CE
:204A6000FE6001080A61010816610108226101082E6101083A6101084661010800BFFEE7BF
:204A800000B587B00020B2490860B24908800720B14908701821B148EFF71AF81821B04830
:204AA000EFF716F81821AF48EFF712F81022AE49AE48EEF7F4FFAE48AE490A680260496879
:204AC00041601022ACA1B148EFF70DF81022B0A1AE481030EFF707F82022B2A1BA48EFF7B7
:204AE00002F800BFB9A207CA04AB07C3BAA207CA01AB07C39DF81A0030389DF81910303977
:204B000001EB810100EB4100AF4988760322B5A104A8EFF70AF818B90120AB49C87670E082
:204B20000322B1A104A8EFF700F818B90220A649C87666E00322ADA104A8EEF7F6FF18B944
:204B40000320A149C8765CE00322A9A104A8EEF7ECFF18B904209C49C87652E00322A5A12E
:204B600004A8EEF7E2FF18B905209749C87648E00322A1A104A8EEF7D8FF18B906209249E6
:204B8000C8763EE003229DA104A8EEF7CEFF18B907208D49C87634E0032299A104A8EEF7E8
:204BA000C4FF18B908208849C8762AE0032295A104A8EEF7BAFF18B909208349C87620E077
:204BC000032291A104A8EEF7B0FF18B90A207E49C87616E003228DA104A8EEF7A6FF18B9EE
:204BE0000B207949C8760CE0032289A104A8EEF79CFF18B90C207449C87602E0002072496E
:204C0000C8769DF8151030399DF81400202801D1002002E09DF81400303800EB800001EB06
:204C20004000694908779DF8051030399DF80400202801D1002002E09DF80400303800EB4F
:204C4000800001EB4000604948779DF8081030399DF80700202801D1002002E09DF80700D6
:204C6000303800EB800001EB4000574988779DF80B1030399DF80A00202801D1002002E0C2
:204C80009DF80A00303800EB800001EB40004E49C87700BF5F48007828B930213B482038B5
:204CA00080F82A102CE05B480078012805D131213648203880F82A1022E056480078022800
:204CC00005D132213148203880F82A1018E051480078032805D133212C48203880F82A104C
:204CE0000EE04C480078042805D134212748203880F82A1004E030212448203880F82A103F
:204D0000102245A121482038EEF7EDFE102247A11E481038EEF7E7FE082249A14B48EEF7CC
:204D2000E2FE08224AA149480830EEF7DCFE08224AA146481030EEF7D6FE4B484B4B0ECB58
:204D40000EC000F0BBF800F093F807B000BD0000440100206001002048010020C8060020B6
:204D600008070020F0060020605F0108E006002049010020705F01085144303037482E201C
:204D8000202020202020202000000000780600205632723172365F32303233303930362E7F
:204DA0000000000054433033333030312D4D53323330332D563072332E202020202020203A
:204DC0002020202000000000980600204A756E20313720323032340031363A35383A34324A
:204DE000000000004A616E00466562004D617200417072004D6179004A756E004A756C00CB
:204E000041756700536570004F6374004E6F760044656300940100205653373530302E2070
:204E2000202020202020202000000000303030303030303030303030303030300000000072
:204E40004D4F54494E4F564100000000B0070020575548414E2E2020000000003230323158
:204E6000303930310000000028080020E8F7FF1F10B5302209490A48EEF711FE10220949E8
:204E80000948EEF70CFE0948094C1ECC1EC0102208490948EEF703FE10BD0000CC5F0108A9
:204EA00070070020FC5F0108A0070020A80800201C6001080C600108B808002010B50C2293
:204EC0000EA11248EEF70FFE114812490A68026049684160104811490968016020221049DE
:204EE0001048EEF7DCFD20220F491048EEF7D7FD10220F490F48EEF7D2FD10BD30303030CF
:204F000030303030303030300000000034080020570100202C60010852010020B85F010815
:204F2000785F010820070020985F010840070020BC5F01086007002088B004460D4631E052
:204F40001948FAF782FB0020FCF756F9F1F76EFA20216846EEF7BCFD2046EEF7D0FD0646DF
:204F6000324621466846EEF79AFD2046EEF7C7FD694608440DA10A88028089788170204604
:204F8000EEF7BDFD69460844C0F803506B464FF620720C214FF4E260FEF7F6F8C820F4F77C
:204FA000B3F800BFCCE70000FC000020202C200008B52B4988420DD100BF2A49896941F01E
:204FC0000401284A91611146896901F00401009100BF43E0244988420DD100BF2149896986
:204FE00041F008011F4A91611146896901F00801009100BF32E01D4988420DD100BF194948
:20500000896941F01001174A91611146896901F01001009100BF21E0154988420DD100BFA8
:205020001049896941F020010E4A91611146896901F02001009100BF10E00E4988420DD1EF
:2050400000BF0849896941F04001064A91611146896901F04001009100BF00BF08BD00004B
:205060000008014000100240000C014000100140001401400018014070B504460E46A1885D
:205080002068F4F715FB28B9A07908B9012506E0002504E0A07908B9002500E00125012E89
:2050A00004D1207A68402840E07102E0207A6840E071257270BD10B50446A1880122206804
:2050C000F4F702FB10BD00BF704702E008C8121F08C1002AFAD170477047002001E001C1D3
:2050E000121F002AFBD1704700F0010181F31388704700000149086070470000DC040020B1
:2051000010B50A46437993421EDB1E4B1B685B6923F002031B4C2468636143799B1A43714C
:20512000184B1B685B6943F00203164C24686361114603790B4499B283788B4202DC8378CD
:20514000CB1A99B201711BE00E4B1B685B6923F002030C4C24686361417900234371094B6D
:205160001B685B6943F00203064C246863610379194483788B4202DC8378CB1A99B20171F2
:2051800010BD00007C18002010B502460B46194654799C4209DB14790C44A1B294788C4238
:2051A00004DC94780C1BA1B200E000219468605C10BD00007FB50646002404E0305D18498D
:2051C0000855601CC4B2082CF8DB3823154A02A9304600F07FFB00241EE0002504E002A85F
:2051E00000F0A0FA681CC5B20F48005DA842F6DC40230E4A694602A800F06CFB002507E043
:205200001DF805000A4901EBC4014855681CC5B2082DF5DB601CC4B2102CDEDB7FBD0000B0
:20522000E402002014680108EC6A01084C680108FA0F002001460120064A12688A4206D1C9
:20524000044A1268044B1B685A40521C02B1002070470000001B0020241B00202DE9F04F33
:2052600087B082460F469046994600250AE0785D3A49495D884203D03846FFF79BFF072541
:20528000681CC5B2082DF2DB4023354A05A9504600F020FB012536E0002405E005A8005D91
:2052A00003A90855601CC4B2082CF7DBB8F1000F04D1681E2B4901EBC00B04E0C5F1100005
:2052C000284901EBC00B002406E003A9201D085C05A90855601CC4B2042CF6DB01AA05A9F8
:2052E000584600F043F8002409E003A8005D01A9095D484005AA211D5054601CC4B2042C85
:20530000F3DB681CC5B2112DC6DB9DF814609DF818008DF814008DF818609DF815609DF8FA
:2053200019008DF815008DF819609DF816609DF81A008DF816008DF81A609DF817609DF8C7
:205340001B008DF817008DF81B604023064A494605A800F0BFFA07B0BDE8F08FE40200201D
:2053600054670108FA0F002094670108F0B587B005460E4617464023104A05A9304600F093
:20538000A9FA002410E005A8005D295D484000F03F0003A908550A4800EB8410095D405C33
:2053A00001A90855601CC4B2082CECDB2023054A394601A800F08EFA07B0F0BD8C68010866
:2053C000EC680108CC6801081CB5F6F753F9F6F759F9B0490870F4F7BFF9FEF797F9F6F764
:2053E0007DFAFBF74FFAFBF7EFFAFBF757FBFBF79FFBFBF72DFAFBF7F5F8FBF7A3F9FBF7D8
:20540000F9F9FBF7DFFBFCF7A7FCEEF7F1FD1420F3F77AFEA048F5F797F9FFF731FBFBF757
:20542000B3FAFAF79BFE9D48F1F7A8F8F1F72AFA9A48F1F75BF8F1F771FA994908700846A4
:2054400001789648FDF75EFE96499748F1F744FAFAF776F80020954908701AE1944800789D
:20546000401C9349087008460078C82801DD0020087090480088F1F7C5FEFBF769FCEFF708
:20548000DFFCFFF71FF98C4A51788C4AD07A8C4B8C4A1278F8F742FEFBF760F88748807EE7
:2054A000AA2841D18848007BC0B18748B0F902000B2190FBF1F084B283498048007B7F4A2C
:2054C00092F91B20104480B2CDE900017B48C37982797E492046FDF727FF46E07A48B0F9F7
:2054E00002000B2190FBF1F07749897A884206DD7548B0F902000B2190FBF1F001E0724807
:20550000807A84B270496D48007B6C4A92F91B20104480B2CDE900016848C37982796B491E
:205520002046FDF701FF20E06448807EEE280AD16248007B6149C97E0844C2B2624963484A
:20554000FDF736FF11E05D48007B5C49C97E0844C2B25A48007E08B9012001E05748007E65
:20556000034659495948FDF7A3FF5948F1F72CFE5848EEF7A9FF00BF5748007818BB5748E1
:20558000007828B1F4F7A6F842F21071884229D94D48C0880A2190FBF1F084B25048808866
:2055A000464A0090127B454D95F91B502A4490B24C4A137B494A11782246FCF761F80120EE
:2055C000454908700EE0404C2389454C627AA1883E4CE068FBF72EFF434A1178384A1078F8
:2055E000FCF782F800BFFAF7D7FB4048FAF73EFDFAF71CFF344B9A7D1989987AF8F7E2FBE6
:205600003B4908703848807910B93A48F1F75AF93548807930B938493848F1F7F5F93848D9
:20562000FCF734FA37480078E8B93748006837490860354840684860334880688860324850
:20564000C068C8602948001F40680861282216480830FDF7A1FC04222DA11348FDF79CFC0D
:20566000012028490870F8F755FFFAF751F82A480068FAF729FD13480078FAF74DFD274835
:20568000FAF788FDFDF7E2F8FCF7E6FA2448F4F74FF8E3E694010020C81200207C0300203E
:2056A00074030020FFEF010800E801085C0000205A0000209801002049010020200700200B
:2056C000CA000020C8000020380600203C0300208D0300208C0300205B00002084010020BC
:2056E000B806002060070020CE00002074070020DE00002075030020EC0200207C1000206C
:20570000560100209B010020A808002000080020464C414700000000440100204008002077
:20572000040600200CB5002104E0425C0DF801204A1CD1B20829F8DB002112E0425C5206BF
:20574000120E425406290ADA4A1C1DF8022002F08002802A03D1425C42F0010242544A1C22
:20576000D1B20729EADB9DF8002002F0800222B1C27842F01002C27003E0C27822F01002C4
:20578000C2709DF8032002F0080222B1827942F00102827103E0827922F0010282710CBD7E
:2057A0002DE9F04106460F46EEF77AFA04000D4618BF0120284320F00040C0F17F6000F11D
:2057C000E040C00F0ED0301C18BF0120384320F00040C0F17F6000F1E040C00F04BF012099
:2057E000FFF788FC20462946BDE8F08130B502460023002952D03348007890B13248334C7C
:20580000247830F81400324C2468201A304C206020460068104420602B482C4C247820F82F
:2058200014202A480078401C284C2070204600781E280FDB002020702248007818B9012058
:20584000204C207006E01F480078012802D102201C4C20701B480078022806D11C480068C9
:205860001E24B0FBF4F083B211E01648007801280CD11648007808B9134608E014480068B9
:20588000124C2478B0FBF4F083B200E01346052093FBF0F0904212DD134610E0002005E06F
:2058A0000024094D25F81040441CE0B21E28F7DB0020064C2070064C2060024C20701846E7
:2058C00030BD000038030020E410002030030020340300202DE9F04104461D46154E00204B
:2058E00000BF4FF000080746401C01F807800828F7DB002000BF12F8013B04EBE3073F78C2
:2059000003F0070C16F80CC007EA0C0767B101EBE0073F7800F0070C16F80CC047EA0C07E0
:2059200001EBE00C8CF80070471C3846AF42E2DBBDE8F081FC6A0108000000000000000087
:2059400001020304060708090000000001020304204E000403000004000000040000000098
:205960009CFFFFFFFF7F0000000000FE00FCFF0100000000204E0004030000040000000499
:20598000000000000080FFFFFF7F0000000000FE00FCFF01000000004000000403000004C6
:2059A00000000004000000000000FCFF00000000000000F000000000000000003075000152
:2059C0002C0100040000000400000000CCF7FFFF000000000030DFFF0000000000000000C3
:2059E000001000040100000400000004000000009CFFFFFF1A0400000088FAFF00780500D5
:205A000000000000307500042C0100040000000400000000E6FBFFFF000000000098EFFF43
:205A20000000000000000000204E00040300000400000004000000009CFFFFFFFF7F0000D2
:205A4000000000FE00FCFF0100000000204E00040300000400000004000000000080FFFF51
:205A6000FF7F0000000000FE00FCFF0100000000400000040300000400000004000000005F
:205A80000000FCFF00000000000000F00000000000000000307500012C0100040000000440
:205AA00000000000CCF7FFFF000000000030DFFF00000000000000000010000401000004FE
:205AC00000000004000000009CFFFFFF1A0400000088FAFF00780500000000003075000464
:205AE0002C0100040000000400000000E6FBFFFF000000000098EFFF00000000000000000C
:205B0000204E00040300000400000004000000009CFFFFFFFF7F0000000000FE00FCFF01F7
:205B200000000000204E00040300000400000004000000000080FFFFFF7F0000000000FEEE
:205B400000FCFF0100000000400000040300000400000004000000000000FCFF00000000FF
:205B6000000000F00000000000000000307500012C0100040000000400000000CCF7FFFF99
:205B8000000000000030DFFF000000000000000000100004010000040000000400000000DA
:205BA0009CFFFFFF1A0400000088FAFF0078050000000000307500042C0100040000000452
:205BC00000000000E6FBFFFF000000000098EFFF0000000000000000204E000403000004E7
:205BE00000000004000000009CFFFFFFFF7F0000000000FE00FCFF0100000000204E00041E
:205C00000300000400000004000000000080FFFFFF7F0000000000FE00FCFF010000000083
:205C2000400000040300000400000004000000000000FCFF00000000000000F0000000002A
:205C400000000000307500012C0100040000000400000000CCF7FFFF000000000030DFFF9A
:205C60000000000000000000001000040100000400000004000000009CFFFFFF1A04000050
:205C80000088FAFF0078050000000000307500042C0100040000000400000000E6FBFFFF49
:205CA000000000000098EFFF0000000000000000657F367E107D807C657B527A467940781A
:205CC0004177C476CE75DF74F47310739F72C271EA701770486F7D6E1A6E566D966CDA6BF9
:205CE000216B6D6A136A6469B8680F68696718677666D8653D65A4640E64C4633263A2621C
:205D000015628A614561BE603960B55F345FB55E765EFA5D805D085D915C1C5CE25B705B30
:205D2000FF5A905A235AED5981591859AF584858E357B1574D57EB568A562B56CC550000C2
:205D4000C90092015B022403ED03B6047F0548061107D907A2086A09330AFB0AC40B8C0C29
:205D6000540D1C0EE30EAB0F72103A110112C8128F1355141C15E215A8166E173318F91861
:205D8000BE19821A471B0B1CCF1C931D571E1A1FDD1F9F2061212322E522A6236724282594
:205DA000E825A82667272628E528A329612A1F2BDC2B992C552D112ECC2E872F4130FB30A5
:205DC000B5316E322633DF3396344D350436BA366F372438D9388C39403AF23AA53B563C6C
:205DE000073DB83D683E173FC53F73402141CE417A422543D0437A442445CD4575461C47B8
:205E0000C34769480F49B449584AFB4A9D4B3F4CE04C814D204EBF4E5D4FFB4F9750335142
:205E2000CE51685202539B533254C9546055F5558A561D57B0574258D3586459F359825A9F
:205E40000F5B9C5B285CB35C3E5DC75D4F5ED75E5D5FE35F6860EB606E61F0617162F16256
:205E60007063EE636C64E8646365DD655666CF664667BC673268A66819698B69FD696D6ABC
:205E8000DC6A4A6BB76B236C8E6CF86C616DC96D306E966EFB6E5E6FC16F22708370E27015
:205EA00040719D71F9715472AE7207735E73B5730A745F74B27404755575A575F37541766D
:205EC0008D76D87622776B77B377FA773F788478C77809794A798979C879057A417A7C7AB1
:205EE000B67AEE7A267B5C7B917BC57BF87B297C597C887CB67CE37C0E7D397D627D897D9E
:205F0000B07DD57DFA7D1D7E3E7E5F7E7E7E9C7EB97ED57EEF7E097F217F377F4D7F617FC0
:205F2000747F867F977FA67FB47FC17FCD7FD87FE17FE97FF07FF57FF97FFD7FFE7F0000FC
:205F400005000000000000000500000000000000050000000000000005000000000000002D
:205F6000A02824000000000000000000000000000455000000000000AA02640019030E0999
:205F80000F87A555DB006464646464646464646401025500B80B3C870000000055020C0C61
:205FA00000000000000000000000000000000000000000000000000090016400FA00B0043E
:205FC000C8000A000A00A08C24000000010000000000000000000000000000000000000094
:205FE00000000000000000000000000000004141000000004141414100000000000000001B
:206000000000000000000000000000005A008700B400E100C800B4000E010000000000007F
:2060200000000000000000000000000041564F4E49544F4D7401E8025C04D1054507B90851
:206040002D0AA20B160D8A0EFF0F880100006400200302010002120300006400E803020117
:20606000AE021D05BC026400140503016603AC07480364003408050100040000F4016400A5
:206080003408040100048001000064004803020156015A0300006400B00402010002490569
:2060A000BC02640036060301AE025D07480364003A070401630332094803640034080501E3
:2060C00000040000F40164003408040100040000EE026400340804016303DC013002000014
:2060E000A903020152017604BC020000E2040302E9016F0748030000B3050402AE02290B2E
:20610000D40300003408050300040000B00400003408040200040B02300264006703010157
:20612000EB00AE04BC0264001F0402014B01B00648036400B805030100022D0BD403640093
:2061400034080502000400003A076400340804010004000000002110422063308440A5502F
:20616000C660E770088129914AA16BB18CC1ADD1CEE1EFF13112100273325222B5529442B3
:20618000F772D662399318837BB35AA3BDD39CC3FFF3DEE36224433420040114E664C7746F
:2061A000A44485546AA54BB528850995EEE5CFF5ACC58DD55336722611163006D776F66633
:2061C0009556B4465BB77AA719973887DFF7FEE79DD7BCC7C448E5588668A778400861186F
:2061E00002282338CCC9EDD98EE9AFF9488969990AA92BB9F55AD44AB77A966A711A500AB3
:20620000333A122AFDDBDCCBBFFB9EEB799B588B3BBB1AABA66C877CE44CC55C222C033C6E
:20622000600C411CAEED8FFDECCDCDDD2AAD0BBD688D499D977EB66ED55EF44E133E322E32
:20624000511E700E9FFFBEEFDDDFFCCF1BBF3AAF599F788F8891A981CAB1EBA10CD12DC1A8
:206260004EF16FE18010A100C230E3200450254046706760B9839893FBA3DAB33DC31CD3B2
:206280007FE35EF3B1029012F322D2323542145277625672EAB5CBA5A89589856EF54FE56E
:2062A0002CD50DC5E234C324A01481046674476424540544DBA7FAB79987B8975FE77EF732
:2062C0001DC73CD7D326F2369106B01657667676154634564CD96DC90EF92FE9C899E9896E
:2062E0008AB9ABA94458654806782768C018E1088238A3287DCB5CDB3FEB1EFBF98BD89BB2
:20630000BBAB9ABB754A545A376A167AF10AD01AB32A923A2EFD0FED6CDD4DCDAABD8BAD6D
:20632000E89DC98D267C076C645C454CA23C832CE01CC10C1FEF3EFF5DCF7CDF9BAFBABF31
:20634000D98FF89F176E367E554E745E932EB23ED10EF01E00000000B71DC1046E3B820925
:20636000D926430DDC7604136B6BC517B24D861A0550471EB8ED08260FF0C922D6D68A2F38
:2063800061CB4B2B649B0C35D386CD310AA08E3CBDBD4F3870DB114CC7C6D0481EE093452C
:2063A000A9FD5241ACAD155F1BB0D45BC2969756758B5652C836196A7F2BD86EA60D9B63CE
:2063C00011105A6714401D79A35DDC7D7A7B9F70CD665E74E0B6239857ABE29C8E8DA19171
:2063E000399060953CC0278B8BDDE68F52FBA582E5E66486585B2BBEEF46EABA3660A9B7C0
:20640000817D68B3842D2FAD3330EEA9EA16ADA45D0B6CA0906D32D42770F3D0FE56B0DDD9
:20642000494B71D94C1B36C7FB06F7C32220B4CE953D75CA28803AF29F9DFBF646BBB8FBD5
:20644000F1A679FFF4F63EE143EBFFE59ACDBCE82DD07DEC77708634C06D4730194B043DB7
:20646000AE56C539AB0682271C1B4323C53D002E7220C12ACF9D8E1278804F16A1A60C1B9F
:2064800016BBCD1F13EB8A01A4F64B057DD00808CACDC90C07AB9778B0B6567C699015718B
:2064A000DE8DD475DBDD936B6CC0526FB5E6116202FBD066BF469F5E085B5E5AD17D1D5765
:2064C0006660DC5363309B4DD42D5A490D0B1944BA16D84097C6A5AC20DB64A8F9FD27A5D4
:2064E0004EE0E6A14BB0A1BFFCAD60BB258B23B69296E2B22F2BAD8A98366C8E41102F8327
:20650000F60DEE87F35DA9994440689D9D662B902A7BEA94E71DB4E0500075E4892636E9F8
:206520003E3BF7ED3B6BB0F38C7671F7555032FAE24DF3FE5FF0BCC6E8ED7DC231CB3ECF6C
:2065400086D6FFCB8386B8D5349B79D1EDBD3ADC5AA0FBD8EEE00C6959FDCD6D80DB8E60BD
:2065600037C64F643296087A858BC97E5CAD8A73EBB04B77560D044FE110C54B3836864676
:206580008F2B47428A7B005C3D66C158E4408255535D43519E3B1D252926DC21F0009F2C3A
:2065A000471D5E28424D1936F550D8322C769B3F9B6B5A3B26D6150391CBD40748ED970A8C
:2065C000FFF0560EFAA011104DBDD014949B93192386521D0E562FF1B94BEEF5606DADF8EF
:2065E000D7706CFCD2202BE2653DEAE6BC1BA9EB0B0668EFB6BB27D701A6E6D3D880A5DEFE
:206600006F9D64DA6ACD23C4DDD0E2C004F6A1CDB3EB60C97E8D3EBDC990FFB910B6BCB447
:20662000A7AB7DB0A2FB3AAE15E6FBAACCC0B8A77BDD79A3C660369B717DF79FA85BB49293
:206640001F4675961A163288AD0BF38C742DB081C330718599908A5D2E8D4B59F7AB085481
:2066600040B6C95045E68E4EF2FB4F4A2BDD0C479CC0CD43217D827B9660437F4F4600725D
:20668000F85BC176FD0B86684A16476C93300461242DC565E94B9B115E565A158770191899
:2066A000306DD81C353D9F0282205E065B061D0BEC1BDC0F51A69337E6BB52333F9D113EA3
:2066C0008880D03A8DD097243ACD5620E3EB152D54F6D4297926A9C5CE3B68C1171D2BCC52
:2066E000A000EAC8A550ADD6124D6CD2CB6B2FDF7C76EEDBC1CBA1E376D660E7AFF023EAE5
:2067000018EDE2EE1DBDA5F0AAA064F4738627F9C49BE6FD09FDB889BEE0798D67C63A8066
:20672000D0DBFB84D58BBC9A62967D9EBBB03E930CADFF97B110B0AF060D71ABDF2B32A6AA
:206740006836F3A26D66B4BCDA7B75B8035D36B5B440F7B139312921191109013B332B23B6
:206760001B130B033D352D251D150D053F372F271F170F0738302820181008003A322A2225
:206780001A120A023C342C241C140C043E362E261E160E0627072F0F37173F1F26062E0E31
:2067A00036163E1E25052D0D35153D1D24042C0C34143C1C23032B0B33133B1B22022A0AD9
:2067C00032123A1A210129093111391920002808301038182122232425262728292A2B2C8B
:2067E0002D2E2F303132333435363738393A3B3C3D3E3F400102030405060708090A0B0C09
:206800000D0E0F101112131415161718191A1B1C1D1E1F2038302820181008003931292122
:20682000191109013A322A221A120A023B332B233E362E261E160E063D352D251D150D0560
:206840003C342C241C140C041B130B0300000D04100A1700000002091B0E05140000160750
:20686000120B031900000F01061A130C00002836331E242E00001D2F27322C2000002B343F
:206880003026372100002D1F2931231C00001F040001020300000308040506070000070C08
:2068A00008090A0B00000B100C0D0E0F00000F141011121300001318141516170000171C44
:2068C00018191A1B00001B001C1D1E1F1F0E272C3C173724041E2E350C253E15050F2F1D2A
:2068E0003F360614261C3D0D2D1607340E040D01020F0B08030A060C05090007000F07046D
:206900000E020D010A060C0B0905030804010E080D06020B0F0C0907030A05000F0C08027C
:2069200004090107050B030E0A00060D0F01080E060B03040907020D0C00050A030D040771
:206940000F02080E0C00010A06090B05000E070B0A040D0105080C060903020F0D080A0142
:20696000030F04020B06070C00050E090A00090E06030F05010D0C070B0402080D0700092A
:206980000304060A0208050E0C0B0F010D060409080F03000B01020C050A0E07010A0D000C
:2069A00006090807040F0E030B05020C070D0E030006090A010208050B0C040F0D080B05DA
:2069C000060F00030407020C010A0E090A0609000C0B070D0F01030E05020804030F0006D4
:2069E0000A010D080904050B0C07020E020C0401070A0B060805030F0D000E090E0B020C98
:206A000004070D0105000F0A030908060402010B0A0D07080F090C050603000E0B080C0787
:206A2000010E020D060F00090A0405030C010A0F09020608000D03040E07050B0A0F04026D
:206A4000070C090506010D0E000B0308090E0F0502080C030700040A010D0B060403020C50
:206A600009050F0A0B0E01070600080D040B020E0F00080D030C0907050A06010D000B071C
:206A80000409010A0E03050C020F080601040B0D0C03070E0A0F060800050902060B0D08FF
:206AA00001040A070905000F0E02030C0D020804060F0B010A09030E05000C07010F0D08E7
:206AC0000A0307040C05060B000E0902070B0401090C0E0200060A0D0F03050802010E07D3
:206AE000040A080D0F0C09000305060B01010202020202020102020202020201804020102A
:206B000008040201381000001A1002001910060018100A0017100E001610160015101E00DD
:206B2000141022001310360012103A0011104600101056000F105E000E106E000D108200D5
:206B40000C108E000B10A6000A10B2000910C2000810DA000710F2000610020105101E01DB
:206B60000410360103104E0102106E010110820100109E01FF0FBE01FE0FD601FD0FEE01F8
:206B8000FC0F0E02FB0F3202FA0F5602F90F7E02F80F9602F70FB202F60FE202F50F020368
:206BA000F40F2203F30F4E03F20F7E03F10FA203F00FDA03EF0FFE03EE0F2E04ED0F5A04CF
:206BC000EC0F8E04EB0FB604EA0FEE04E90F2A05E80F5E05E70FAE05E60FE205E50F220667
:206BE000E40F6E06E30FBE06E20F0A07E10F5E07E00FAA07DF0FEE07DE0F5208DD0F9608CD
:206C0000DC0FDE08DB0F4E09DA0F9E09D90F020AD80F7A0AD70FD20AD60F420BD50FA60BEA
:206C2000D40F2E0CD30FA20CD20FF60CD10F720DD00FE20DCF0F3A0ECE0FBE0ECD0F320FAB
:206C4000CC0F860FCB0FFE0FCA0F6E10C90FBA10C80F3211C70F9611C60FD611C50F421269
:206C6000C40F9212C30FD612C20F2E13C10F7213C00FBE13BF0F0E14BE0F5214BD0F861453
:206C8000BC0FD214BB0F1A15BA0F4A15B90F9215B80FC215B70FFE15B60F3616B50F7216DF
:206CA000B40FA216B30FDE16B20F0E17B10F3617B00F6E17AF0FA617AE0FCA17AD0F02187D
:206CC000AC0F3618AB0F5618AA0F9218A90FC218A80FE218A70F1A19A60F4A19A50F72199D
:206CE000A40FA219A30FD219A20FF219A10F261AA00F561A9F0F761A9E0FAE1A9D0FD21A73
:206D00009C0FFE1A9B0F261B9A0F4E1B990F721B980F9E1B970FC21B960FE61B950F161C1F
:206D2000940F361C930F621C920F8A1C910FB61C900FD61C8F0F021D8E0F261D8D0F461D58
:206D40008C0F781D8B0F961D8A0FBE1D890FF01D880F101E870F361E860F621E850F861EA1
:206D6000840FAA1E830FDA1E820FF61E810F1E1F800F4E1F7F0F7A1F7E0F961F7D0FCA1FE2
:206D80007C0FE61F7B0F06207A0F2820790F5620780F7820770F9620760FC820750FE62092
:206DA000740F1421730F3621720F5A21710F8621700FA8216F0FD0216E0FF8216D0F202214
:206DC0006C0F48226B0F66226A0F9822690FB622680FE822670F0823660F3223650F562370
:206DE000640F8423630FB023620FC823610FFC23600F28245F0F48245E0F80245D0FA02473
:206E00005C0FBC245B0FF8245A0F1225590F3E25580F6425570F9025560FB425550FE8257C
:206E2000540F0626530F3426520F5826510F8426500FA8264F0FD8264E0F00274D0F2C2762
:206E40004C0F64274B0F84274A0FB827490FD827480F0828470F2C28460F7028450F90288E
:206E6000440FC028430FE828420F1829410F4C29400F7C293F0FA4293E0FD4293D0FFC2954
:206E80003C0F282A3B0F482A3A0F8C2A390FB02A380FDC2A370F082B360F3C2B350F702B27
:206EA000340FA82B330FCC2B320FF82B310F382C300F642C2F0F882C2E0FCC2C2D0FF42C29
:206EC0002C0F282D2B0F582D2A0F902D290FC42D280FF02D270F242E260F582E250F882EC3
:206EE000240FBC2E230FF42E220F1C2F210F582F200F942F1F0FBC2F1E0FEC2F1D0F2C3013
:206F00001C0F54301B0F90301A0FC830190FF430180F2831170F6431160F8C31150FC83131
:206F2000140FFC31130F2C32120F6C32110F9C32100FCC320F0F08330E0F3C330D0F6C3317
:206F40000C0FAC330B0FCC330A0F1034090F4434080F8034070FA834060FE434050F2035DE
:206F6000040F4835030F8035020FB435010FE835000F1C36FF0E5436FE0E8036FD0EB436E4
:206F8000FC0EF036FB0E1437FA0E4C37F90E7837F80EB437F70EE437F60E0C38F50E443854
:206FA000F40E7C38F30EAC38F20ED838F10E1439F00E3C39EF0E7039EE0EA439ED0EDC39D8
:206FC000EC0E043AEB0E403AEA0E643AE90E9C3AE80ECC3AE70E043BE60E243BE50E5C3B96
:206FE000E40E883BE30EB03BE20EE03BE10E143CE00E383CDF0E6C3CDE0E9C3CDD0EC03C14
:20700000DC0EF43CDB0E243DDA0E483DD90E7C3DD80E9C3DD70ECC3DD60E003ED50E303EDF
:20702000D40E543ED30E883ED20EAC3ED10EDC3ED00E083FCF0E2C3FCE0E603FCD0E8C3FE4
:20704000CC0EBC3FCB0EE03FCA0E0C40C90E3840C80E6040C70E8C40C60EAC40C50EDC402A
:20706000C40E1041C30E3841C20E5841C10E8441C00EB441BF0ED841BE0EFC41BD0E2C42BB
:20708000BC0E4C42BB0E7442BA0EA042B90EC442B80EEC42B70E1043B60E3C43B50E6043ED
:2070A000B40E9043B30EB043B20ED843B10E0044B00E2C44AF0E5044AE0E7044AD0EA0441B
:2070C000AC0EC044AB0EF044AA0E1045A90E3045A80E6045A70E8845A60EB045A50ED0457E
:2070E000A40E0046A30E2046A20E5446A10E7446A00E94469F0EC4469E0EE8469D0E1447AF
:207100009C0E44479B0E64479A0E8047990EB447980ED447970EF447960E2848950E4848ED
:20712000940E7848930EA448920EC048910EE448900E18498F0E3C498E0E68498D0E90490B
:207140008C0EB4498B0EE0498A0E0C4A890E304A880E504A870E804A860EA84A850ED04A15
:20716000840EF44A830E204B820E404B810E744B800E9C4B7F0EC84B7E0EFC4B7D0E204CFB
:207180007C0E504C7B0E704C7A0EA04C790EC04C780EF44C770E244D760E444D750E7C4D60
:2071A000740EA04D730ED04D720EF84D710E204E700E444E6F0E744E6E0EA44E6D0EC44EC6
:2071C0006C0E004F6B0E284F6A0E504F690E804F680EA84F670ED44F660E1050650E3850C5
:2071E000640E6050630E9050620EC450610EDC50600E08515F0E40515E0E70515D0E9C51B3
:207200005C0ED4515B0E08525A0E3052590E6052580E9452570EB852560EF052550E2053E2
:20722000540E4853530E8053520EB053510EE053500E14544F0E50544E0E70544D0EAC54E6
:207240004C0ED8544B0E10554A0E4855490E8055480EAC55470EE455460E1C56450E445631
:20726000440E8856430EC056420EE456410E3057400E64573F0E94573E0ED0573D0E0C58B4
:207280003C0E3C583B0E74583A0EB058390EE058380E2059370E5059360E8C59350ECC59EE
:2072A000340E105A330E385A320E805A310EC45A300EF05A2F0E405B2E0E705B2D0EB05B2B
:2072C0002C0EF45B2B0E305C2A0E685C290EB45C280EF05C270E2C5D260E705D250EB45D98
:2072E000240EF05D230E405E220E745E210EBC5E200E045F1F0E485F1E0E845F1D0ED05F27
:207300001C0E0C601B0E4C601A0E9860190EE060180E1C61170E7461160EBC61150EF46125
:20732000140E3C62130E8462120ED462110E2463100E70630F0EAC630E0E04640D0E50641A
:207340000C0E84640B0EE0640A0E1865090E6465080EB465070E0466060E5066050E9866D0
:20736000040EE866030E3867020E8867010ED867000E2468FF0D6868FE0DB868FD0D086994
:20738000FC0D5869FB0DC069FA0DF869F90D5C6AF80DB46AF70DF06AF60D446BF50D946B8A
:2073A000F40DE46BF30D346CF20D886CF10DC86CF00D186DEF0D686DEE0DB86DED0D086ED5
:2073C000EC0D6C6EEB0DA86EEA0DEC6EE90D606FE80DA06FE70DF86FE60D4870E50D9870B2
:2073E000E40DE870E30D4C71E20D8871E10DD071E00D3872DF0D7472DE0DCC72DD0D24736D
:20740000DC0D5C73DB0D9C73DA0D0074D90D4474D80D8874D70DF074D60D2875D50D68755C
:20742000D40DD075D30D0876D20D5876D10DA876D00DEC76CF0D3877CE0D8877CD0DD47756
:20744000CC0D2078CB0D7078CA0DA878C90DEC78C80D3C79C70D8479C60DCC79C50D1C7AEF
:20746000C40D4C7AC30D9C7AC20DDC7AC10D207BC00D5C7BBF0D9C7BBE0DE47BBD0D1C7CEE
:20748000BC0D6C7CBB0DA47CBA0DDC7CB90D2C7DB80D5C7DB70D9C7DB60DEC7DB50D147ECA
:2074A000B40D5C7EB30D8C7EB20DCC7EB10D147FB00D4C7FAF0D847FAE0DBC7FAD0DFC7F9B
:2074C000AC0D3080AB0D7480AA0D9C80A90DE480A80D0C81A70D4081A60D8481A50DAC815C
:2074E000A40DE481A30D2082A20D6082A10D8482A00DBC829F0DEC829E0D20839D0D5C8303
:207500009C0D90839B0DB4839A0DEC83990D1C84980D4884970D8484960DAC84950DDC8482
:20752000940D1085930D4885920D6C85910DA085900DCC858F0DF8858E0D2C868D0D5C8685
:207540008C0D84868B0DB4868A0DE086890D1087880D4087870D6C87860D9087850DD08716
:20756000840DF087830D1888820D4C88810D7C88800D9C887F0DCC887E0DEC887D0D1C891F
:207580007C0D44897B0D6C897A0D9489790DC089780DE089770D0C8A760D388A750D608AEC
:2075A000740D808A730DA88A720DD08A710DF08A700D188B6F0D388B6E0D608B6D0D848B6F
:2075C0006C0DB08B6B0DCC8B6A0DF08B690D148C680D308C670D548C660D708C650D948C9A
:2075E000640DBC8C630DE08C620DF88C610D1C8D600D388D5F0D588D5E0D808D5D0DA08D5A
:207600005C0DBC8D5B0DE08D5A0D048E590D1C8E580D408E570D608E560D788E550D9C8E60
:20762000540DB88E530DDC8E520DFC8E510D208F500D348F4F0D508F4E0D708F4D0D908FB5
:207640004C0DA88F4B0DD48F4A0DEC8F490D0C90480D2C90470D4490460D6090450D80903D
:20766000440D9C90430DB490420DD490410DF490400D0C913F0D38913E0D50913D0D6C9102
:207680003C0D90913B0DAC913A0DC891390DE491380D0892370D2892360D5092350D689262
:2076A000340D8092330DB492320DCC92310DF092300D14932F0D3C932E0D60932D0D90931A
:2076C0002C0DB4932B0DE8932A0D1494290D3C94280D6C94270D9094260DC094250DF494C4
:2076E000240D3095230D5095220D8095210DB895200DDC951F0D0C961E0D40961D0D64962F
:207700001C0D90961B0DC8961A0DEC96190D1C97180D5097170D7097160DA097150DD497F4
:20772000140DF497130D2498120D4C98110D7898100D9C980F0DD0980E0DF0980D0D209945
:207740000C0D44990B0D6C990A0D9099090DC099080DE899070D089A060D449A050D5C9A22
:20776000040D809A030DB89A020DD49A010DF09A000D289BFF0C449BFE0C609BFD0C949B70
:20778000FC0CB49BFB0CD09BFA0C009CF90C209CF80C409CF70C709CF60C889CF50CA89C63
:2077A000F40CC89CF30CEC9CF20C109DF10C2C9DF00C509DEF0C689DEE0C849DED0CA49D2F
:2077C000EC0CC89DEB0CDC9DEA0CFC9DE90C149EE80C309EE70C4C9EE60C649EE50C7C9E08
:2077E000E40C949EE30CAC9EE20CC09EE10CD89EE00CE89EDF0C049FDE0C189FDD0C289F2E
:20780000DC0C3C9FDB0C549FDA0C609FD90C749FD80C849FD70C989FD60CA49FD50CB89F70
:20782000D40CC49FD30CD49FD20CE49FD10CF49FD00C00A0CF0C10A0CE0C18A0CD0C28A0A8
:20784000CC0C34A0CB0C40A0CA0C4CA0C90C58A0C80C64A0C70C70A0C60C7CA0C50C84A098
:20786000C40C90A0C30C9CA0C20CA4A0C10CB0A0C00CB8A0BF0CC0A0BE0CCCA0BD0CD4A00C
:20788000BC0CDCA0BB0CE8A0BA0CF0A0B90CF8A0B80C04A1B70C0CA1B60C14A1B50C1CA1D4
:2078A000B40C24A1B30C2CA1B20C34A1B10C3CA1B00C44A1AF0C4CA1AE0C54A1AD0C5CA1DC
:2078C000AC0C64A1AB0C6CA1AA0C74A1A90C7CA1A80C84A1A70C8CA1A60C90A1A50C98A104
